:1000000000800020BD010000F9880000B1880000D8
:10001000B1880000B1880000B1880000B1880000FC
:10002000B1880000B1880000B1880000F9880000A4
:10003000F9880000B1880000A5800000A9810000B7
:10004000F9880000F9880000F9880000F9880000AC
:10005000F9880000F9880000F9880000F98800009C
:10006000F9880000F9880000F9880000F98800008C
:10007000F9880000F9880000F9880000F98800007C
:10008000F9880000F9880000F9880000F98800006C
:10009000F9880000F9880000F9880000F98800005C
:1000A000A9640000B5640000F9880000F988000028
:1000B000F9880000F9880000F9880000F98800003C
:1000C000F9880000F9880000F9880000F98800002C
:1000D000F9880000F9880000F9880000F98800001C
:1000E000F9880000F9880000F9880000F98800000C
:1000F000F988000099A80000F9880000C5A900004F
:10010000F9880000D1920000F9880000F988000009
:10011000F9880000F9880000F9880000F9880000DB
:10012000F9880000F9880000F9880000F9880000CB
:10013000F9880000F9880000F9880000F9880000BB
:10014000F9880000F9880000F9880000F9880000AB
:10015000F9880000F9880000F9880000F98800009B
:10016000F9880000ED950000F9880000F98800008A
:10017000F9880000F9880000F9880000F98800007B
:10018000F9880000F9880000F9880000F98800006B
:10019000F9880000F9880000F9880000F98800005B
:1001A000F9880000F9880000F9880000F98800004B
:1001B000F9880000F9880000F9880000564B4CF2DD
:1001C000205210B51A804DF628121A8000BF00BFC9
:1001D00008F096FB514B4FF010621A60504A9A603B
:1001E000504ADA60504A136813F4807304D14F49BF
:1001F0000B604FF4A85313604D4B1A78110703D5C9
:100200001A7842F008021A704A4B4B492A221A7097
:100210004A4A4B4B8B4204D252F8040F43F8040B6A
:10022000F8E7484B484900228B4202D243F8042B9E
:10023000FAE74649464A002352F8230041F82300D2
:1002400001336F2BF8D1434B434A802103F8011B44
:100250009342FBD1414B3D4A1A60414B8A221A70AE
:10026000A3F5805324225A70A0221A709A7992071B
:10027000FCD59A79D406FCD43A4A937903F00C035E
:10028000082B384BF9D103221A7140225A719A79FE
:100290009006FCD5334A9179324B4906FBD5324A58
:1002A000324911600221516020221A709A7902F0BD
:1002B0000C020C2AFAD12E4B2E4A1A602E4B2F4AD2
:1002C0001A6000225A60072243F8042C2C4AC3F813
:1002D0000C2D62B608F0C4FE144B1B68DA0705D576
:1002E000284808F091FC284B284A1A60284B1B78B4
:1002F0005B0609D5244C254B22689A4204D121483B
:1003000008F082FC002323600BF016FE08F0FEFAD2
:1003100008F02CFAFEE700BF0E20054030800440B4
:10032000823F04000100002B10D0034014D0034092
:1003300002D0074000E007401C99FF1F80E4000046
:100340004088FF1F1C99FF1FB49FFF1F0082FF1FE3
:100350000000000000E400E05FE400E008ED00E0E1
:100360000050064000400640448004400000030165
:1003700004800440C010050014E000E0FF76010096
:1003800000002020176F385D1CE00340A5C3945A7D
:1003900000F00740FFFFFFFFFFFFFFFFFFFFFFFF32
:1003A000FFFFFFFFFFFFFFFFFFFFFFFFFFFFFFFF5D
:1003B000FFFFFFFFFFFFFFFFFFFFFFFFFFFFFFFF4D
:1003C000FFFFFFFFFFFFFFFFFFFFFFFFFFFFFFFF3D
:1003D000FFFFFFFFFFFFFFFFFFFFFFFFFFFFFFFF2D
:1003E000FFFFFFFFFFFFFFFFFFFFFFFFFFFFFFFF1D
:1003F000FFFFFFFFFFFFFFFFFFFFFFFFFFFFFFFF0D
:10040000FFFFFFFFFFFFFFFFFFFFFFFFDEF9FFFF23
:1004100010B5054C237833B9044B13B10448AFF33E
:1004200000800123237010BD1C99FF1F00000000F5
:1004300084E40000084B10B51BB108490848AFF32D
:1004400000800848036803B910BD074B002BFBD0A0
:10045000BDE81040184700BF000000002099FF1FB2
:1004600084E400001C99FF1F0000000070B44C8859
:10047000A04220D901230133DBB21CB2660031F85F
:10048000144084421D46F6D3A04211D005F1004528
:10049000013D965B31F8151032F81530401AF21A0A
:1004A00000FB02F0641A90FBF4F4E01870BC704793
:1004B000905B70BC704702260125E5E700280CDA46
:1004C000064A434282FB0320DA17C2EB600000EBCE
:1004D0004000A3EB8000C0F10C007047ABAAAA2A31
:1004E0002DE9F84F0C2007F0E7FF0C2008F09CFCEA
:1004F000E049142008F0A8FC0221032008F03AFD8E
:100500000221042008F036FD0221052008F032FD0A
:100510000221062008F02EFD01210A2008F02AFD04
:100520000121092008F026FD01210D2008F022FDFF
:100530000121282008F01EFD0121142008F01AFDD9
:1005400002210B2008F016FD01210C2008F012FDFD
:1005500000210C2008F0FAFC002004F0F9F917281B
:10056000044600F258822021002003F0D3FF4FF40C
:10057000AF61022003F0CEFF04204FF47A6103F054
:10058000C9FF0B2008F0E8FC002800F0398240F693
:100590002821062003F0BEFF40F6E441082003F0C6
:1005A000B9FF4FF4AF610A2003F0B4FF40F6FC013D
:1005B0000C2003F0AFFF4FF49661222003F0AAFF56
:1005C0004FF41661242003F0A5FF7D212A2003F0BB
:1005D000A1FF202C00F007822021002003F09AFFC9
:1005E0000C210E2003F096FF0121102003F092FF52
:1005F0000221122003F08EFF0021142003F08AFF55
:100600000021162003F086FF0221182003F082FF4C
:1006100001211A2003F07EFF02211C2003F07AFF43
:1006200004211E2003F076FF1421202003F072FF26
:100630000121262003F06EFF0321282003F06AFF2A
:1006400004212C2003F066FF0F212E2003F062FF0F
:100650000021302003F05EFF0C21322003F05AFF0E
:100660000021342003F056FF0021362003F052FF12
:100670000021382003F04EFF00213A2003F04AFF0A
:1006800000213C2003F046FF00213E2003F042FF02
:100690000021402003F03EFF0021422003F03AFFFA
:1006A0001F21442003F036FF1321462003F032FFC0
:1006B0000E21482003F02EFF11214A2003F02AFFCB
:1006C0000A214C2003F026FF00214E2003F022FFD8
:1006D0000621502003F01EFF0221522003F01AFFD2
:1006E0000C21542003F016FF0021562003F012FFC6
:1006F0000021582003F00EFF01215A2003F00AFFC9
:1007000003215C2003F006FF0A215E2003F002FFB4
:100710000021602003F0FEFE022004F019F9564B80
:10072000564C1880042004F013F9554BDFF8B4A19F
:100730001880062004F00CF9524B534D1880082005
:1007400004F006F9514BDFF8A09118800A2004F05C
:10075000FFF84F4BDFF894B118800C2004F0F8F844
:100760004C4B4D4F18800E2004F0F2F84B4B4C4E82
:100770001880102004F0ECF84A4BDFF874811880E0
:10078000122004F0E5F8484B1880142004F0E0F83B
:10079000464B1880162004F0DBF8454B18801820D3
:1007A00004F0D6F8434B18801A2004F0D1F8424BDD
:1007B00018801C2004F0CCF8404B18801E2004F058
:1007C000C7F83F4B1880202004F0C2F83D4B18803A
:1007D000222004F0BDF83C4B1880242004F0B8F827
:1007E0003A4B1880262004F0B3F82080282004F02B
:1007F000AFF8374B18802A2004F0AAF8AAF80000B6
:100800002C2004F0A5F8334B18802E2004F0A0F81B
:10081000314B1880302004F09BF8304B1880322088
:1008200004F096F82E4B1880342004F091F82880BC
:10083000362004F08DF86880382004F089F8A8800C
:100840003A2004F085F8E8803C2004F081F8288103
:100850003E2004F07DF86881402004F079F8A881FA
:10086000422004F075F8A9F80000442004F070F864
:1008700040E000BF001B3746B699FF1F8299FF1F5B
:10088000869AFF1F409AFF1F5499FF1F2A9AFF1F45
:10089000509AFF1F0C9AFF1F6A89FF1F8099FF1F44
:1008A0007089FF1FB899FF1F6299FF1F1C9AFF1FD5
:1008B0004099FF1FEC99FF1F2E9AFF1F4C9AFF1FB4
:1008C000F699FF1F849AFF1F529AFF1FEE99FF1F90
:1008D000E499FF1F169AFF1F209AFF1F5099FF1FD0
:1008E0007C9AFF1F149AFF1FAE99FF1F449AFF1FA7
:1008F0006C89FF1FA94BAA4D1880462004F028F8E8
:10090000ABF80000482004F023F8ABF802004A20BE
:1009100004F01EF8ABF804004C2004F019F8ABF812
:1009200006004E2004F014F89E4B1880502004F06E
:100930000FF89D4B1880522004F00AF89B4B18804A
:10094000542004F005F83880562004F001F8984B44
:100950001880582003F0FCFF964B18805A2003F0B3
:10096000F7FF954B18805C2003F0F2FF934B188043
:100970005E2003F0EDFF3080602003F0E9FFBAF85D
:10098000003021882970A3F5AF7E8D498D4CB9F8D0
:100990000020208040F23A7303FB0EF381FB03E159
:1009A000DB17A3EB6113884C8848DFF858C28849ED
:1009B0003233C8F8003002F00203238002F004034F
:1009C000038002F008038CF80030824C824802F069
:1009D000100C02F02003A1F800C05A21238005F07A
:1009E00013FE18BBFEE7042008F0B6FA00287FF4D7
:1009F00093AE062008F0B0FA00283FF4EDAD8BE688
:100A00004FF49661062003F085FD4FF4FA6108204B
:100A100003F080FDC5E5042008F09EFA002859D0B7
:100A20004FF6FF739C427FF4D4AD9CE56B4A6C4853
:100A30001268DFF8D4B10023012105F0BDFE03F0F8
:100A400021FD0B2008F088FA011E0CBF01230023B2
:100A50008BF8003002D1112008F08CFADFF8889171
:100A6000604CDFF8A8810023C9F800302360C8F883
:100A700000304FF0010A11E007F052FD23681844DE
:100A800020600AF001010D2008F060FA0AF1010A65
:100A9000FA2008F097FABAF1050F22D00F2008F0DB
:100AA00083FCD8F8003003440E20C8F8003007F06B
:100AB00037FDD9F800309BF800100344C9F8003026
:100AC00015200029D8D1112008F06EFC23681844A5
:100AD0002060D6E7062008F03FFA00283FF443AD37
:100AE0009EE7D8F80030D9F800103F4A2068DFF8B8
:100AF00020E13688DFF81CC1002BB8BF0333002982
:100B0000B8BF0331891011603988384F9B10002815
:100B1000A3EB0102B8BF033019448010CEF80020C7
:100B20003960DFF8F4E0324FC8F800308219C6EBC4
:100B30000008002120600D203B60CCF80080CEF83A
:100B4000002008F003FAFA2008F03CFA01210D20F9
:100B500008F0FCF9FA2008F035FA00210D2008F021
:100B6000F5F904F07DF940F2DC5008F02BFA214B46
:100B7000012604201E6008F0EFF910B91E4B287002
:100B80001E701E4B1E4A1B781370184605F072F833
:100B900001210D20BDE8F84F08F0D8B9549AFF1F85
:100BA000699AFF1F7E99FF1F6489FF1FA889FF1F95
:100BB000829AFF1F289AFF1F7099FF1F6689FF1FE7
:100BC000B5814E1BB299FF1F4E9AFF1FDC99FF1F84
:100BD000049AFF1F429AFF1F349AFF1F7489FF1F58
:100BE000BC99FF1F9C99FF1F089AFF1F649AFF1F63
:100BF000FC99FF1F7499FF1FE699FF1FB899FF1F0B
:100C00002C9AFF1F689AFF1F789AFF1F8899FF1F71
:100C1000189AFF1FF099FF1F3C9AFF1FF0B40E882F
:100C200086420DD203F10043013B31F81350854257
:100C300002D9F0BCFFF71ABC32F81300F0BC7047C1
:100C40001088F0BC704700BF094B1B880C2B09D8DB
:100C5000084A80B252F8232028B143F6FE73984226
:100C600003D9108C7047108870470349FFF7FEBB0B
:100C7000169AFF1FE0CB0000C0CA000008B5214A49
:100C8000214B12881868824234DA204B1B88991A4B
:100C90008342A8BF0346B1F5F87FA3EB020321DA34
:100CA000C3EB031303EB431393FBF1F105310A206C
:100CB00007F0BCFF164B1978F1B1164B16491B68AB
:100CC00083F30703C3EB031303EB431381FB0321FC
:100CD0001944DB17C3EBA11105310920BDE8084019
:100CE00007F0A4BFC3EB43131B01013193FBF1F1E8
:100CF0000531DCE70021DAE70920BDE8084007F00C
:100D000095BF00BFB699FF1F109AFF1F869AFF1F5D
:100D1000569AFF1F309AFF1F09040281374A38494B
:100D20001088384AF8B5384B12881B68834248DB74
:100D30009342A8BF134698420B60C8BF002342DD10
:100D4000101AB0F5804FAABF9B03C3EB8333013069
:100D500093FBF0F0FFF778FF2C4B2D4F1C883B687E
:100D6000C0F3C61505FB04F47F2CA8BF7F249D4269
:100D7000064608D0274B1B88002B38D1264B1B88F2
:100D8000002B30D13D60254D2B689E4205D0214B74
:100D90001B885A1F032A1DD92E60214D2B689C42A7
:100DA0000ED0204B188848B11A4B1F4A1B88D35CC1
:100DB000834203D0C0B2E1B204F0A4FE2C60F8BDBF
:100DC000F8BD034608609A42D4BFC0EB0203C0EBF3
:100DD0000303B5E7144AD05C2030C0B206F07F01AF
:100DE00004F090FED8E7284604F000FFCAE70E4A58
:100DF0002946D05C04F086FEC0E700BFB699FF1F0D
:100E0000109AFF1F869AFF1F6499FF1F7099FF1F9A
:100E10004499FF1F6299FF1F1C9AFF1F6C99FF1FC7
:100E20003C99FF1F289AFF1F7889FF1F2DE9F04F7B
:100E3000172087B008F0B8FAA34B1860162008F006
:100E4000B3FAA24BA24A1B8810600C2B00F07D83E2
:100E5000DFF8C0A29F4ABAF800109F4B52F8214019
:100E600000221A709D4B9E4A1B889E491288013BA6
:100E700031F91350002A00F0A7809B4B1B78002B00
:100E800049D1112008F090FA984B0193D3F80090C3
:100E90000746B94549DD964B964E1B88012B00F05D
:100EA000CD82954B03933068944B00930AF0D2FDAA
:100EB0004FF07C510AF022FE914A009B1288D3F831
:100EC00000800292834620460AF0C4FD029A039BEA
:100ED00053F822100AF012FE014600200AF004FD29
:100EE0000AF0D2FFC5EB0805C9EB0502BD42B8BF49
:100EF0003D469042C9EB0505C0F2C98200FB05F5ED
:100F000095FBF2F00AF0A6FD7E4BDFF80C920393FE
:100F10004FF07C5149E0152007F002FB734B019321
:100F2000D3F800900746B945B5DC764B0393D3F868
:100F30000090B94580F2A5806D4B6E4E1B88012B49
:100F400000F038836C4A6D4B3068049200930AF0CD
:100F500081FD4FF07C510AF0D1FD6949009B098861
:100F6000029183462046D3F800800AF073FD02996F
:100F7000049A52F821100AF0C1FD0AF085FF454499
:100F8000BD42C9EB0502A8BF3D46C9EB050590422D
:100F9000BABF00FB055501324543DFF87C9195FB54
:100FA000F2F00AF057FD4FF07C51574B02930AF0D4
:100FB000A5FD59460AF09AFC0AF066FF534B0493CC
:100FC0003060D9F800B074E04F4B02931E460F20FA
:100FD00008F0EAF9D6F8008005904045C0F2A681F5
:100FE0004A4B0493D3F80080059B434540F3C982E4
:100FF0003F4B404E1B88012B00F017833E4A306860
:1010000001920AF027FD4FF07C510AF077FD3C4B2E
:1010100003901B88009320460AF01CFD009B019A58
:10102000DFF8F49052F82310D9F800B00AF066FD0A
:101030000AF02AFF059A5D449542C8EB0503A8BF54
:101040001546C8EB05059842BABF00FB05550133AC
:10105000454395FBF3F00AF0FDFC284B00934FF05D
:101060007C511D46214B01930AF048FD03990AF07B
:101070003DFC0AF009FF234B03933060D5F8008054
:1010800017E01E4B1B4E00931D461F4B306802930A
:101090001E4B04930AF0DEFC4FF07C510AF02EFD4B
:1010A0000AF0F2FEDFF87090D5F80080D9F800B0B1
:1010B000306017490988013903295BD8DFE811F04E
:1010C000D00014012E00F2004C99FF1F7C9AFF1FE4
:1010D000009AFF1F2889FF1F9499FF1F6489FF1F33
:1010E000B299FF1F84CC0000789AFF1FF099FF1F70
:1010F000829AFF1F7899FF1F38CC00009C99FF1F30
:10110000F699FF1F3C9AFF1F189AFF1F649AFF1F52
:10111000A889FF1F2E9AFF1F8899FF1F58460AF0C3
:1011200099FCAA490AF0EAFC054605980AF092FCE7
:10113000A7490AF0E3FC014628460AF0D7FB0AF06B
:10114000A3FE8346C9F800B040460AF083FC9F49DD
:101150000AF0D4FC054638460AF07CFC9C490AF0AB
:10116000CDFC014628460AF0C1FB0AF08DFE009B2B
:1011700080461860974898490788984B08881D68EA
:101180009749DFF8B0E20988C7EB0B0307EB0B02C6
:10119000029F3B60C0EB080700EB08030498026065
:1011A000019A1760039A8D421360BEF8002080F206
:1011B000AA810027C1EB020E8A4B7445186880F2A1
:1011C0009681631C884207FB03F70EF1010E97FB23
:1011D000FEF7C0F249828242A8BF0246521A03FBC0
:1011E00002F494FBFEF48D4200F35781884200F331
:1011F00054817D4C20680AF02DFC7C490AF07EFC6D
:101200007B490AF073FB0AF03FFEA0F5FF531C3B3D
:10121000082B98BF4FF40050336818440028206012
:10122000C0F26381B0F5804F80F27481714B1B78FE
:101230001BB1B0F5005F40F075816F4D2B78002B2E
:1012400040F078816D4D20682B68674C984204D03F
:1012500080B204F035FD23682B6007B0BDE8F08F45
:1012600058460AF0F7FB66490AF048FC054605981F
:101270000AF0F0FB63490AF041FC014628460AF0F7
:1012800035FB0AF001FE8346C9F800B040460AF07B
:10129000E1FB5B490AF032FC054638460AF0DAFB0E
:1012A00058495CE758460AF0D5FB50490AF026FC3D
:1012B000054605980AF0CEFB53490AF01FFC01468B
:1012C00028460AF013FB0AF0DFFD8346C9F800B098
:1012D00040460AF0BFFB45490AF010FC0546384677
:1012E0000AF0B8FB48493AE758460AF0B3FB4749C9
:1012F0000AF004FC054605980AF0ACFB44490AF0E4
:10130000FDFB014628460AF0F1FA0AF0BDFD8346CE
:10131000C9F800B040460AF09DFB3C490AF0EEFBDC
:10132000054638460AF096FB394918E7394B3A4EDC
:101330001B88012B00F05E81384A306801920AF068
:1013400089FB4FF07C510AF0D9FB354B04901B8888
:10135000009320460AF07EFB009B019ADFF8D890AC
:1013600052F82310D9F800B00AF0C8FB014600205B
:101370000AF0BAFA0AF088FD059AC5EB0B0595420A
:10138000C8EB0503B8BF1546C8EB05059842BABFC0
:1013900000FB05550133454395FBF3F00AF05AFB7A
:1013A000204B00931D46204B01934FF07C511F4B67
:1013B00003930AF0A3FB04990AF098FA0AF064FD7B
:1013C0001B4B04933060D5F8008072E6CDCC4C3FC7
:1013D000CDCC4C3E6A89FF1F7089FF1F4C99FF1FBF
:1013E000509AFF1F009AFF1F6089FF1F9A99193FAB
:1013F000CDCC4C45069BFF1F7D99FF1F2089FF1F09
:101400003333733FCDCC4C3DCDCCCC3E6666663F8E
:10141000CDCCCC3D829AFF1F7899FF1F38CC0000BD
:10142000F699FF1F9C99FF1FF099FF1F3C9AFF1F21
:10143000649AFF1F0C9AFF1F8899FF1F904B00931F
:101440003068904B03930AF005FB4FF07C510AF093
:1014500055FB8D4A8A4B1288D3F80080029283464E
:1014600020460AF0F7FA029A039B53F822100AF07A
:1014700045FB0AF009FDC5EB0805C9EB0502BD42B5
:10148000B8BF3D468242C9EB05057FF737AD00FB8B
:101490000555013295FBF2F034E5BAF80030002B27
:1014A0003FF4A7AE3B1B002BB8BF5B42092B48DDC6
:1014B00007F500500130001B0AF0CCFA7349744C58
:1014C0000AF01CFB054620680AF0C4FA71490AF0CC
:1014D00015FB014628460AF009FA0AF0D5FC3368E4
:1014E000184400282060BFF69DAE002214E0884218
:1014F00007FB04F7B8BF002397FBFEF780F2B68026
:1015000093FBFEF46FE69542D4BFC1EB0507C1EB38
:1015100002074FE643F6FF725F4B22601B78002BF9
:101520003FF48BAE00210D2007F010FD5B4B012234
:101530001A7087E601210D2007F008FD00232B70AB
:1015400080E64FF40050524C66E6012007F02CFF75
:10155000534B1B6898427FF77BACDFF85CA1514A84
:10156000BAF80010504B52F8210001221A700AF00C
:1015700071FA4FF07C510AF0C1FA0AF085FC04467A
:1015800070E43F4B494E00931D46494B3068019330
:10159000484B03930AF05EFA4FF07C510AF0AEFA22
:1015A0000AF072FCDFF81491D5F80080D9F800B089
:1015B00030607EE5334B04933068314B00930AF082
:1015C00049FA4FF07C510AF099FA2F4A009B128891
:1015D000D3F800800292834620460AF03BFA029A32
:1015E000049B53F822100AF089FA014600200AF001
:1015F0007BF9C2E4234A306801920AF02BFA4FF0DB
:101600007C510AF07BFA204B04901B880093204603
:101610000AF020FA009B019ADFF8A09052F82310FC
:10162000D9F800B00AF06AFAA4E6164A30680192C6
:101630000AF010FA4FF07C510AF060FA124B039056
:101640001B88009320460AF005FA009B019ADFF8F8
:101650006C9052F82310D9F800B00AF04FFA014606
:1016600000200AF041F9E3E40A46B7E59042D4BF0E
:10167000C1EB0003C1EB020304FB03F340E700BF2F
:101680009C99FF1F38CC0000F699FF1FCDCCCC3EB3
:101690006089FF1F9A99193F069BFF1F7D99FF1FC5
:1016A0006C89FF1F2889FF1F9499FF1F7899FF1FDE
:1016B000F099FF1F3C9AFF1F2E9AFF1F8899FF1F6A
:1016C00030B58DB06D460024E1B23E4804F060FFB5
:1016D00001340C2C45F8040BF6D13B4B1B88002B36
:1016E0004DD03A4B0A9A1B889A424BDA009A9342A1
:1016F00048DD029A934245DD049A934242DD344B21
:101700001978002946D03348334A34490088128872
:1017100009680244B1EB620F34DD00241C7004F050
:1017200099FA21460D2007F011FC322007F04AFCFF
:1017300001210D2007F00AFC322007F043FC21466E
:101740000D2007F003FC322007F03CFC01210D20A6
:1017500007F0FCFB322007F035FC21460D2007F096
:10176000F5FB322007F02EFC0D20012107F0EEFBE7
:101770004FF42F700DB0BDE8304007F023BC144A81
:10178000117809B90DB030BD13700DB0BDE830400F
:1017900004F060BA0F4C104A11482488128800687F
:1017A0002244B0EB620FEDDD01240D201C7007F028
:1017B000CDFB322007F006FC0D20214607F0C6FBCA
:1017C0003220D7E7349AFF1F049AFF1F149AFF1F95
:1017D000A699FF1F0C9AFF1F509AFF1F009AFF1F28
:1017E0004C99FF1F2DE9F0417B4C7C4D20680AF09D
:1017F00031F97B490AF082F90646102007F0D4FD42
:101800000AF028F977490AF079F931460AF06EF8BA
:101810000AF03AFB2B882060002B3FD0724F3A88A9
:1018200090423BDB01467148067836B94FF0010E15
:10183000042B80F800E000F0B380012B6AD0022B6B
:1018400000F0BC80032B36D1694B1B88092B32D0AA
:1018500023683C88674AA342128853DB9342D4BF73
:10186000C4EB0303C4EB0203141B7E2CDFF8888156
:10187000D5BFC3EB8313C3EBC3135B00013493FBEE
:10188000F4F4D8F800300134A34203D0E1B24A2086
:1018900004F038F9C8F80040BDE8F081534A1178E7
:1018A00049B10024012B147016D0022B1FD0032B3A
:1018B00003D0042B28D0BDE8F0814D4B1B88092BA9
:1018C000F9D04D4D2B68002BF5D021464A2004F06D
:1018D00019F92C60BDE8F081474D2A68002AEAD04A
:1018E0001846214604F00EF92C60BDE8F081424D07
:1018F0002B68002BDFD02146042004F003F92C6074
:10190000BDE8F0810023AFE721464020BDE8F0416B
:1019100004F0F8B8374B1B888B42D4BFC2EB0306E8
:10192000C2EB01069A1ADFF8D0807E2AD8BFC6EB38
:101930008616D8F80030C6BFC6EBC6160132760050
:1019400096FBF2F60136B34203D0F1B2012004F067
:10195000D9F82B88C8F80060022B7FF473AF236896
:101960003E88244AB34212882CDA0023961B7E2E2E
:10197000DFF88480D5BFC3EB8313C3EBC3135B00D5
:10198000013693FBF6F6D8F800300136B34220D08A
:10199000F1B2042004F0B6F82B88C8F8006051E7D3
:1019A0007F21402004F0AEF82B88012BD4D1216890
:1019B0003A88104B91421B88B4DBADE70D4A23688F
:1019C00012883E889A42D4BFC6EB0203C6EB0303DB
:1019D000CCE70223E1E700BF6C9AFF1F4C9AFF1F80
:1019E0009A99193FCDCCCC3E529AFF1F8499FF1F84
:1019F0006299FF1FEE99FF1F9899FF1F38B5184B8A
:101A00001B88D3B9174A184914880968174AA14294
:101A100012881DDA141B7F2CC6BFDB010134C3EB17
:101A2000C31393FBF4F4124D2B689C4203D0E1B234
:101A3000052004F067F82C6038BD0E4B0E490F4AA4
:101A40001B680C6812681C1BA41A84F30704EAE7DD
:101A50009142D4BFC4EB0103C4EB0203DAE700BF39
:101A6000B299FF1F409AFF1F609AFF1F2A9AFF1F1B
:101A7000309AFF1FFC99FF1F2489FF1F589AFF1FF0
:101A800010B50C4C236843B90B4B1B88022B0CD0B0
:101A90000A4A00231370236010BD0021052004F0C2
:101AA00031F8054B1B88022BF2D10021412004F0B4
:101AB00029F8EDE7309AFF1FEC99FF1F569AFF1F98
:101AC00010B5254B1B787BB1152006F029FD234A64
:101AD000234B1288186082B9224A12883ABB224BE3
:101AE0001B78002B33D110BD112007F05DFC1B4A81
:101AF0001B4B12881860002AEED00F2007F054FC10
:101B0000184B1A4A1B881060002BE8D0184A194954
:101B100012680968521A9042E1DC134C227892B99B
:101B2000022B0ED17F21412003F0ECFF09E0124986
:101B30001B6809889942D2DC0B4C23781BB9022A16
:101B4000F0D001232370BDE81040FFF757BFBDE878
:101B50001040FFF795BF00BF789AFF1FB299FF1F93
:101B6000609AFF1FEC99FF1F569AFF1F589AFF1F9C
:101B7000FC99FF1F2489FF1F409AFF1F2DE9F04F9A
:101B800091B004AD0024E1B2744804F001FD0134C9
:101B90000C2C45F8040BF6D1714B724CB3F800E0F5
:101BA0000C9B00227345227014DB0A9B9E4500F3B8
:101BB000C080089B6C4A9E4503DD1378002B40F0E3
:101BC000C880069B9E4540F3BA804FF0020C84F813
:101BD00000C009E0089B644A9E45CCBF4FF0060C4C
:101BE0004FF0050C84F800C00E9F059E07980999D8
:101BF00082F800C0BE45D4BF00270127B645D4BF38
:101C00000026012686450B9ADFF898810D9B0F9DD3
:101C1000DFF894A1DFF894918AF80060D4BF002027
:101C200001208E45D4BF0021012188F8001096457F
:101C30004E49DFF87CB14E4E89F80000D4BF002237
:101C400001229E45D4BF002301230A70AE45494AB4
:101C50008BF80070D4BF002501250120137035706A
:101C600007F0A2FB444B454A1D681188444BA8422B
:101C7000D4BF002201220B291A7001D90C2901D0EE
:101C8000A8424EDC002301933E4B9AF800E01F78F7
:101C900099F800C098F800209BF800303349367856
:101CA00091F800903349DFF80CA191F80080247876
:101CB000A7EB4E07CCEB070CA2EB8202C3EB8377BA
:101CC0006244C3EB8703134403EB4903434403EB30
:101CD0008606BAF800202C4F0C2313FB046632440E
:101CE000019B3E600C3A1344A8421946274AC4BFE0
:101CF000274B1E701368994217D0264B264C186844
:101D00000290029820601B680393244C039B248854
:101D100011601B1AA34284BF214B196011B0BDE8AA
:101D2000F08FA1F10C030193AEE71B48194B00683B
:101D3000E9E74FF0040C84F800C00B4A54E7049B19
:101D40009E45C6BF4FF0010C84F800C04FF0000C58
:101D50004AE74FF0030C84F800C045E7349AFF1FB0
:101D6000149AFF1F4999FF1FF499FF1F7E9AFF1FC6
:101D7000809AFF1FB499FF1F6C89FF1F7C9AFF1F79
:101D80004899FF1F5C89FF1F749AFF1F6899FF1F06
:101D90007F9AFF1F609BFF1F9099FF1F849AFF1F70
:101DA000A099FF1F7A9AFF1FAC99FF1F799AFF1F16
:101DB000B099FF1F8099FF1F2DE9F04F0E208FB0C3
:101DC00006F0AEFB09F046FE01469F489F4DA04F2E
:101DD00004F038FD9C4804F00BFD0AF055F880F340
:101DE0000C002860FFF7CAFE3E68012E7BD0022E51
:101DF000DFF8CCA200F06C81032E00F0E381954C5B
:101E0000954B01932368954E0A930A9B32689B1A5F
:101E1000022B1BD9924F3B78002B00F0A583914BEE
:101E20001A78002A0CBF012200221A7000F09F834A
:101E30003B78002B40F0A083FFF7D4FCFEF71EFF99
:101E4000FFF73EFC23680B930B9B33602368864EA1
:101E50000C930C9B32689B1A502B2CD82B68BAF829
:101E60000000019A8342128816DA101AB0F5805FDA
:101E70004FF000031ADAC3EB033393FBF0F0FEF7E5
:101E8000E3FE0146282006F0D1FE03F0CFFE03F06A
:101E9000FDFC0FB0BDE8F08F9342D4BFC0EB03034D
:101EA000C0EB0203101AB0F5805FE4DB1A030130C7
:101EB00092FBF0F0E3E702F0A7FD6C4B1B7823B92F
:101EC0006B4B1B78002B00F0DE810D2007F044F8EF
:101ED000B0FA80F149090D2007F038F823680D9316
:101EE0000D9B3360BAE7634B634A188813788342CB
:101EF00004D0C3B21846137003F0D4FDDFF8C481D8
:101F00005E4AB8F800001378834204D05C4C237812
:101F1000002B40F0DD81DFF8A8A12B68BAF8002083
:101F20004C4C9A4280F2A9812168564A0791079841
:101F30005549106002220B603A60544B1F88F7B974
:101F4000534B1B88DBB9534B1F680E2006F0E8FA91
:101F5000A7F21F37874202DC4F4B00221A704F4B0B
:101F60001B88002B40F00B83404E41484C494D4AA2
:101F7000337003700B701370374B019342E7DFF837
:101F800048B1DFF84891BBF80000B9F80030464985
:101F9000464A18440B684010984205DA1368984284
:101FA00002DA002F40F0BE833A4B02921F460E2009
:101FB0000391019306F0B4FA3F68029AA7F5487EB0
:101FC000704580F2958132480088002800F09081A9
:101FD0000399BBF800C0B9F800000B6812680CEB5D
:101FE00000014910994280F28A81914240F3878131
:101FF0002F480768791C002940F3BF85802900F32A
:10200000BB852C4E2C4A2D4B3688128801601868EF
:102010003244B0EB620FC0F2E987A7F148020F2A01
:1020200000F20684134B0021473F0D201F8006F06D
:102030008DFF962006F0C6FF01210D2006F086FFD9
:10204000019B1F6881E700BFBC99FF1F6499FF1FB8
:102050007499FF1F609BFF1F869AFF1F249AFF1F22
:10206000689AFF1F8699FF1FE899FF1F7C99FF1F41
:10207000A499FF1FB899FF1F2C9AFF1F699AFF1F91
:10208000E699FF1F3899FF1FE099FF1F4E9AFF1F27
:10209000DC99FF1F089AFF1F709AFF1F429AFF1FCB
:1020A000F899FF1FA799FF1F4C99FF1F009AFF1F68
:1020B000749AFF1F529AFF1FEE99FF1F6C9AFF1F21
:1020C000B699FF1F8299FF1F0C9AFF1F509AFF1F9E
:1020D0002E68BAF80030B34280F2EF80A24CA348D9
:1020E00022680892A24A089900681288091A914247
:1020F00002D8002A7FF484AE9E4A9F49126801915B
:10210000B242B8BF3246934208889C4940F3F485F6
:102110009B4A09881360002900F00783DFF8A48236
:1021200088F80010974EFEF7F9FD30687F2840F3DD
:10213000F085954B7F3883FB0032C317C3EB6203F6
:1021400003EB4303A0EB83007330904B03931B8896
:102150003060002B40F00E878D4B02931B78002BD4
:1021600000F06784DFF860B29BF80030002B00F0CD
:102170006084884B04944FF000094C4699460CE06B
:1021800003F17300C0B298F8001003F0E3FC9BF871
:1021900000300134A34240F34B84336859F8040FF4
:1021A000794A1844A0F17F0382FB032ED917C1EBB3
:1021B0006E0101EB41017F28A3EB8103E0DCFEF718
:1021C0007DF9DFE7D5F80080BAF80010414540F30B
:1021D000FD80714B1B78002B40F0F8806F4C20780D
:1021E0007F2840F32787A3F155337F3803F100435D
:1021F00083FB0032C317C3EB620303EB4303A0EB83
:1022000083007330614B03931B88C0B22070002B96
:1022100040F073875E4B02931B78002B00F0A28581
:10222000DFF8A4B19BF80030002B00F09B85594EDD
:10223000DFF854814FF000090BE003F17300C0B2E6
:1022400003F0B0FC9BF8003009F101094B4540F365
:10225000898556F8043F20781844A0F17F0388FB55
:102260000321DA17C2EB610202EB42027F28A3EBE3
:102270008203E2DCFEF722F9E1E7474A1278002AFE
:102280003FF45BAE50E6424B1B78002B7FF41DAE53
:10229000434B1B78002B7FF418AE3F4B1B78002B71
:1022A0007FF413AE0D2006F057FE00287FF416AE23
:1022B00001210D2006F04AFE10E6374A1278002A66
:1022C0007FF40CAF01233B602B4B274C019399E526
:1022D000C3B21846137003F0F3FB2D4B314A194675
:1022E0002F4B18460023137023700B70037012E6F7
:1022F000BBF80000B9F8001012680144491091427F
:10230000BFF623AE0E2006F00BF9019B1F68A7F560
:1023100048729042BFF619AE23480278002A7FF433
:1023200014AE224E327801210170002A40F04D8215
:102330001F4A1278002A40F0AF861E4A1278002AFF
:1023400000F013871C4B1B78002B7FF4FEAD1B4B5A
:102350001B78002B3FF4F9ADB8F80030184A0A3367
:10236000A8F800301170F0E5609BFF1F3899FF1F3F
:10237000209AFF1FE099FF1F869AFF1F4099FF1FB9
:10238000109AFF1FA099FF1FABAAAA2A7E99FF1FD0
:10239000F899FF1F8089FF1FA699FF1F1E9AFF1F34
:1023A000A799FF1FA499FF1F709AFF1F4999FF1F4C
:1023B000AC99FF1F799AFF1F7A9AFF1FB099FF1FF0
:1023C000E699FF1F8599FF1F6889FF1FBA4E306885
:1023D0007F2840F32981B94B7F3883FB0032C31734
:1023E000C3EB620303EB4303A0EB83007330B44CF5
:1023F0002778874200F04C85B24B1B88002B00F0F9
:102400001681B14B01937F2F40F36D84AB487F3F22
:1024100080FB0730FB17C3EB600000EB4000A7EB2D
:1024200080007330A94B02931B78C0B22070002B40
:1024300040F0CE83A64B04931B78002B40F0AA8576
:10244000A44B05931B78002B40F05E86A24B0393B0
:10245000059B1B78A3B3A14B22781B881344A3F1DF
:1024600018007F2840F3BE85944A973B82FB0321E6
:10247000DA17C2EB610202EB4202A3EB820303F123
:102480007300C0B203F08EFB954B964A19782378FF
:1024900032F811201344A3F118007F2840F39E85E1
:1024A000864A973B82FB0321DA17C2EB610202EBFB
:1024B0004202A3EB820303F17300C0B203F072FB8C
:1024C000029B1B78002B00F0E684039B824F198847
:1024D000002900F0568530687F2840F30984774B47
:1024E0007F3883FB0032C317C3EB620303EB430364
:1024F000A0EB830073303060002940F0F284029B2F
:102500001B78002B00F09881DFF810B29BF80030A8
:10251000002B00F09181744FDFF804824FF0000926
:102520000DE003F17300C0B298F8001003F012FB45
:102530009BF8003009F101094B4540F37D81336878
:1025400057F8040F5D4A1844A0F17F0382FB032172
:10255000DA17C2EB610202EB42027F28A3EB82038F
:10256000DFDCFDF7ABFFDEE7FEF7D8FB57E4FEF755
:102570005DFCFFF7A5FA65E4FEF7D0FB5CE4002004
:1025800006F012FF594B5A4F1A683978594E90424B
:10259000D4BF002301239942337040D090423EDDE6
:1025A000554A92F800C0BCF1000F00F0B784534ABE
:1025B00092F80080B8F1000F40F0AE845049434ECD
:1025C0004448097802964FF0010E059086F8008085
:1025D00080F8008082F800E0002940F0A985494A8F
:1025E0001278002A00F01685394A049210461278B3
:1025F000002A40F00C854449364E09783270012299
:102600000596027059B131493C4A0291002111707E
:10261000029A059E1170049A0120307011703B706F
:10262000294B0193FFF7EEBBFDF748FFDFE6374A82
:102630002548126801909142008805DC8242D4BF8F
:10264000C1EB0203C1EB0003411AB1F5804FC0F2A8
:10265000B6849B03481C93FBF0F0FEF7F5FAC0F339
:10266000C61009F0F7F92A4B8046188809F0F2F9EC
:1026700028498146404609F041FA0146484609F09A
:102680003DFA414609F032F94FF07E51804609F09B
:10269000D3FB002840F025851F49404609F0EAFB9E
:1026A000002840F0CB84404609F014FCC0B2DFF8AB
:1026B000708088F80000A6E6A099FF1FABAAAA2A9E
:1026C0001E9AFF1F4099FF1F869AFF1FF899FF1F50
:1026D000A799FF1F7C99FF1F7E99FF1F549AFF1F28
:1026E0005C9AFF1F449AFF1F8089FF1F6C89FF1FA0
:1026F0005D9AFF1FA599FF1FB099FF1FA499FF1FA7
:102700007E9AFF1FAC99FF1F4899FF1F109AFF1F69
:102710005099FF1FCDCCCC3D0000FE426889FF1FC1
:102720008599FF1FA84B019362E41A469042D4BFDB
:10273000C3EB0001C3EB0201C01AB0F5804FC0F239
:1027400057848A03013092FBF0F0FEF77DFAC0F364
:10275000C61009F07FF99D4B0646188809F07AF9F2
:102760009B498046304609F0C9F90146404609F0C8
:10277000C5F9314609F0BAF84FF07E51064609F026
:102780005BFB002840F0BD849249304609F072FBA3
:10279000002840F05684304609F09CFBC0B2DFF8B8
:1027A0008C8288F80000BDE48B4A1278002A7FF4FE
:1027B000CCAB8A4A8A481278243A82F347020260F4
:1027C000D1B25B2003F09EF93278032A30D1854ED6
:1027D0003178002940F01585834F3A78002A40F07F
:1027E0000385DFF8F48198F80020002A40F0EF8498
:1027F0007E4A1278002A40F0DD847D490A807D4AB5
:102800001278002A40F0C9847B4A7F2111803278F7
:1028100072B93A7862B998F800204AB9774E7F21A8
:102820000720328003F06EF97F210B2003F06AF954
:10283000019B1F68FFF789BB049B1B78002B49D0C5
:102840003368A3F10C007F2840F3C5836C4A8B3BAF
:1028500082FB0321DA17C2EB610202EB4202A3EB17
:10286000820303F17300DFF8C481C0B298F800104E
:1028700003F070F9029B1B7863B3DFF89CB19BF8FF
:1028800000303BB35F4F4FF000090CE003F17300E1
:10289000C0B298F8001003F05DF99BF8003009F120
:1028A00001094B4516DD336857F8042F54491A4483
:1028B000A2F18B0381FB0310D917C1EB6001A2F1D8
:1028C0000C0001EB41017F28A3EB8103DEDCFDF767
:1028D000F5FDDDE7059B1B78002B40D04A4A3368A5
:1028E00012881344A3F118007F2840F37183444AEF
:1028F000973B82FB0321DA17C2EB610202EB420233
:10290000A3EB820303F17300DFF82081C0B298F8D3
:10291000001003F01FF93D490B78022B9ABF5A1C97
:10292000D2B200220A703A49336831F812201344B7
:10293000A3F118007F2840F34883314A973B82FB7C
:102940000321DA17C2EB610202EB4202A3EB82031E
:1029500003F1730098F80010C0B203F0FBF8039B7A
:102960001B88002B00F0B782029B1B783BB9049BAD
:102970001B7823B9059B1B78002B00F00984254B9D
:102980001B78002B00F0228123490B78082B00F2E2
:102990001D81224832680068214E0133DBB25F1E80
:1029A000101A46F827000B70BAF80010D5F800800E
:1029B000227041451B4CBFF625AA22681A4B09928A
:1029C000099A1A60FFF71EBA089AFF1F5099FF1F55
:1029D000CDCCCC3D0000FE42B099FF1F7F9AFF1F77
:1029E000389AFF1FAC99FF1F7A9AFF1F799AFF1F31
:1029F0001C9AFF1F7E9AFF1F4099FF1F6299FF1FBD
:102A0000ABAAAA2A8089FF1F549AFF1F5C9AFF1F56
:102A1000449AFF1FA499FF1F6889FF1FA899FF1FF1
:102A20008489FF1F609BFF1F109BFF1F8599FF1F5D
:102A3000049CBA4B1B78002B40F05C823368B84A88
:102A40001278002A4AD0A3F10C007F2840F3D682E6
:102A5000B44A8B3B82FB0321DA17C2EB610202EB23
:102A60004202A3EB820303F17300C0B298F8001096
:102A700003F070F8029B1B787BB3DFF8E4B29BF89D
:102A8000003053B3A84B02944FF000094C469946CE
:102A90000BE003F17300C0B298F8001003F05AF88D
:102AA0009BF800300134A34216DD336859F8041F47
:102AB0009C4A1944A1F18B03D81782FB032EC0EB6B
:102AC0006E0EA1F10C000EEB4E0E7F28A3EB8E03D1
:102AD000DFDCFDF7F3FCDEE7029C3368934A1278F3
:102AE000002A3ED0924A10880344A3F118007F28A0
:102AF00040F38A828B4A973B82FB0321DA17C2EBB1
:102B0000610202EB4202A3EB820303F17300C0B245
:102B100098F8001003F01EF886490B78022B9ABF34
:102B20005A1CD2B200220A708349336831F812204D
:102B30001344A3F118007F2840F36382794A973B3E
:102B400082FB0321DA17C2EB610202EB4202A3EB24
:102B5000820303F17300C0B298F8001002F0FAFF8C
:102B60003368039A1288002A00F0CF817349032248
:102B70000B703A60FFF746B980267149714A0F8899
:102B800071491288096806603A44B1EB620FBFF6DA
:102B90004FAE6E4A1178002940F08B81B8F80020C2
:102BA0006B48B2423FF444AE6A4A068001260D20CB
:102BB000167006F0CBF9962006F004FA31460D2087
:102BC00006F0C4F9019B1F68FFF7BFB93268EBE656
:102BD000614B03931B88002B40F03283504B0493CE
:102BE000524B0593DFF878B19BF8003063B34E4F3A
:102BF000DFF830814FF000090AE003F17300C0B242
:102C000002F0D0FF9BF8003009F101094B451BDDB4
:102C100057F8043F20781844A0F17F0388FB032174
:102C2000DA17C2EB610202EB42027F28A3EB8203B8
:102C3000E3DCFDF743FCE2E73C4B059302F0B2FF17
:102C4000029B1B78002BCDD1049B1B78002B3FF4FB
:102C5000FFAB2378A3F10C007F2840F39881314A21
:102C60008B3B82FB0321DA17C2EB610202EB4202CB
:102C7000A3EB820303F17300C0B202F093FF029B47
:102C80001B78002B00F08F81DFF8D4B09BF8003068
:102C9000002B00F0C782244FDFF888804FF0000936
:102CA0000BE003F17300C0B202F07CFF9BF8003030
:102CB00009F101094B457FF7CBAB57F8043F227868
:102CC0001A44A2F18B0388FB0310D917C1EB6001F2
:102CD000A2F10C0001EB41017F28A3EB8103E0DCB2
:102CE000FDF7ECFBDFE73846FDF7E8FBFFF79ABBA3
:102CF000FDF7E4FBFFF7FFBB184E09888242A8BF2F
:102D00000246326000297FF409AA93423FF714ADCE
:102D10000CE5FDF7D3FBFFF718BA00BFA499FF1F1E
:102D2000A799FF1FABAAAA2A8089FF1F7C99FF1FC2
:102D3000549AFF1F5C9AFF1F449AFF1F1E9AFF1FA1
:102D4000EE99FF1F529AFF1F6C9AFF1F4899FF1FB1
:102D50008299FF1FE699FF1F7E99FF1F109AFF1FA0
:102D60006889FF1FB84B1B78002B43D02378A3F151
:102D70000C007F2840F3D081B44A8B3B82FB0321B7
:102D8000DA17C2EB610202EB4202A3EB820303F10A
:102D90007300C0B202F006FF029B1B7853B3DFF84A
:102DA000E0B29BF800302BB3A94EDFF8A0824FF0C1
:102DB00000090AE003F17300C0B202F0F3FE9BF8D1
:102DC000003009F101094B4514DD56F8043F207825
:102DD0001844A0F18B0388FB0321DA17C2EB6102D0
:102DE0000C3802EB42027F28A3EB8203E2DCFDF702
:102DF00065FBE1E7974B1B78A3B3974B22781B88C1
:102E00001344A3F118007F2840F38C818F4A973B2D
:102E100082FB0321DA17C2EB610202EB4202A3EB51
:102E2000820303F17300C0B202F0BCFE8B4B8C4AEC
:102E30001978237832F811201344A3F118007F2861
:102E400040F36D81814A973B82FB0321DA17C2EB85
:102E5000610202EB4202A3EB820303F17300C0B2F2
:102E600002F0A0FE039B1B88002B00F042817D4BEB
:102E70001B78002B40F038817B4B7C4A019200226A
:102E80001A600123BAF80010D5F800803B6090E585
:102E9000764B01938DE5049B1B78002B7FF415ABDB
:102EA000059B1B78002B7FF410AB039B1988FFF761
:102EB00012BB4B2E40F307811836802EB8F8002045
:102EC0006B49A8BF8026B2423FF4B2AC694A0E807B
:102ED000012600216BE6684B3078197802F03AFE43
:102EE00042E5DFF89481C0B298F8001002F032FE9B
:102EF000FFF705BB7F21402002F004FE5F49604AD6
:102F000033680B600021117099E5D8B298F8001071
:102F100002F020FE336829E600211170594A117829
:102F200041B1594A02921278002A00F0FE800298BC
:102F300000220270554A1278002A7FF455ABBCF18A
:102F4000000F67D1002965D151484F4E90F800E03D
:102F50003D4804903F4805903B48424A01703D4837
:102F60000296117031700170BEF1000F3FF457AB43
:102F7000FFF74CBBC0B298F8001002F0EBFDFFF772
:102F8000EBB8207802F00EFE3988FFF7A4BAFDF7FF
:102F900095FA71E63F4B03931B88002B7FF44CAEF0
:102FA0002C4B059355E6059B1B78002B7FF453AA09
:102FB000049B1B78002B3FF478AFFFF786BAC3EB76
:102FC000833393FBF1F0FFF748BBFDF777FAC1E4D9
:102FD000FDF774FA98E4FDF771FA44E4FDF76EFA30
:102FE000FFF76BBAFDF76AFAFFF74BBA0E46D0E56A
:102FF000C1EB813191FBF0F0FFF7A7BBFDF75EFA63
:1030000033E5FDF75BFAA6E5FDF758FA7FE504998D
:1030100000220A701E4A1278002A3FF400AB0D4AC3
:1030200005921278002A00F00481059900220A70A6
:10303000FFF7F5BAFDF742FAFFF7E4B87F20FFF794
:1030400036BB7F20FFF7ABBBA799FF1FABAAAA2A0D
:103050008089FF1F7C99FF1F549AFF1F5C9AFF1FF6
:10306000449AFF1FA499FF1F109AFF1F869AFF1F03
:103070008299FF1FE699FF1F8599FF1FA899FF1FDF
:103080006889FF1F7E9AFF1FF899FF1FAC99FF1FE9
:103090004899FF1F7E99FF1F6C4B1B78002B51D066
:1030A0006B4B1B78002B7EF450AF6A4B1B78002BC8
:1030B0003EF44BAFB8F80030674A0A3BA8F800303E
:1030C0001170FEF742BF243E002EB8F8002040F3F6
:1030D000A480B2423FF4ACABB6B25F4AA8F800603D
:1030E000F6E60120FFF7E3BA0021402002F00AFDD6
:1030F000C2E6207802F056FDB9E602F053FDFFF774
:1031000089B80120FFF74BBB544B03931B88002B5E
:103110007FF494ADFFF79CB9FDF7D0F939E6FDF7E0
:10312000CDF99CE6FDF7CAF97DE64D484D4A05907C
:10313000002616700298059A4FF0010E80F800E004
:103140001670F7E6424B1B78002B7EF4FEAE414B27
:103150001B78002B3EF4F9AEB8F800303E4A013B34
:10316000A8F800301170FEF7F0BE394A1278002A34
:103170007FF41AAB374B1B78002B3EF4E6AEB8F861
:103180000030354A0133A8F800301170FEF7DDBE7B
:10319000207802F007FDFFF7F2BB334A00201080D1
:1031A0007F21072002F0AEFC7F210B2002F0AAFC59
:1031B000FFF72DBB2D4A012010807F21072002F050
:1031C000A1FC7F210B2002F09DFCFFF718BB284AD1
:1031D000042010807F21072002F094FC00210B20A6
:1031E00002F090FCFFF704BB214A022010807F21EF
:1031F000072002F087FC7F210B2002F083FCFFF701
:10320000F0BA1B4800210280072002F07BFC7F21DE
:103210000B2002F077FCFFF7DFBA012A3FF408AB7E
:1032200001265AE7059B1B78002B7FF414A9FFF7B2
:103230004CB91049029110490A4A0491FFF7E6B9C6
:103240000D4B0493064B0593F8E400BF799AFF1FDA
:103250007A9AFF1FB099FF1FE699FF1F7E99FF1F03
:103260007C99FF1FA499FF1F4099FF1F1C9AFF1F05
:103270006299FF1FF899FF1FA799FF1F10B505F06E
:10328000EBF9064803F01CF900234FF07E52044886
:103290000121BDE8104003F071BA00BF349AFF1F4E
:1032A000BC99FF1F43682A20198801F033B900BF79
:1032B00010B5044622206368198801F02BF9E368F1
:1032C00024201988BDE8104001F024B910B5044647
:1032D0000A206368198801F01DF9E3680C20198839
:1032E000BDE8104001F016B910B504460620636829
:1032F000198801F00FF9E36808201988BDE810402B
:1033000001F008B910B5044602206368198801F07D
:1033100001F9E36804201988BDE8104001F0FAB80B
:1033200070B50E4C84B0122504220123064603908A
:10333000029320468DE824001423102104F060FB42
:103340000622092302930396019520460092142336
:10335000102104F055FB04B070BD00BFA09AFF1F00
:103360002DE9F041224D82B0012602B284B20092D2
:10337000284601967823192104F088FA04F10C02FA
:1033800012B28DE844002846A7197823192104F1C8
:10339000020804F07BFA3FB20FFA88F819233A4684
:1033A000284619460196CDF8008004F06FFA78237C
:1033B0003A4628461946CDF80080019604F10A07DE
:1033C0000B3404F063FA3FB224B278233A4628461D
:1033D00019468DE8500004F059FA192300943A4632
:1033E00001962846194604F051FA02B0BDE8F08172
:1033F000A09AFF1F2DE9F0411E4682B01446002A14
:103400006AD0099B4D4A00EBC305012C6F892989BD
:103410006868A7EB010382FB03E21A444FEAE373F7
:10342000C3EBA21302887BD0042C38D112FA83F3A9
:10343000994203DC9F423946A8BF1946089A018089
:10344000B6F90030BDF920803D48971D4FF0000EC1
:103450003FB2194642460097CDF804E004F016FA50
:1034600029896A896B68521A1B885C2AA3EB0103BD
:1034700059DD03EB43030132C3EB431393FBF2F338
:1034800003F11B0213B2012032801946424601901B
:1034900000972B4804F0FAF92A4B00221A702A4BA5
:1034A000022CB3F9001045D0082C31D100221A802B
:1034B00091422DD0089AB6F90030214806320124F5
:1034C00012B2009219460194BDF9202004F0DEF9F1
:1034D000204602B0BDE8F0811C4D1D4A2B681268E1
:1034E000CB1A93420F4617D9164A338811781448DD
:1034F000012918BF01241470089A06321BB212B2B7
:103500008DE814001946BDF9202004F0BFF92F60A2
:10351000012002B0BDE8F081204602B0BDE8F08194
:103520009BB2D31A84E75C2101FB03F393FBF2F215
:103530001B32A7E74A1C12B21A80B9E7C94216B279
:10354000A09AFF1F149BFF1F929AFF1F109BFF1F43
:1035500050D3000030B583B000230C4605B2009371
:1035600026225B231C210C4803F0E0FE29460123A0
:103570002622094803F0EAF9002C24B205DB214693
:1035800001232622044803F0E1F9044A044B158084
:103590001C8003B030BD00BFA09AFF1FAA89FF1F87
:1035A000AC89FF1F70B5944C237882B01BB1934B4C
:1035B0004FF6FF721A80924BB3F90030C3B9914AAB
:1035C0008E4B1068B3F9002080F30C005B2303FBE3
:1035D00000F000131C3082425AD04FF0FF31FFF749
:1035E000B9FF894803F006FF0023237002B070BDC5
:1035F000012B32D0022B6AD0032B4FD0042BF3D1F6
:10360000272200258DE8240076231C217E487F4E4A
:1036100004F03CF917E0B0F5AF7FA8BF4FF4AF70EE
:10362000323803FB00F386FB0321DB17C3EB611188
:103630001C3109B201231D442722734803F086F987
:103640000C2D00F08180E9B2714802F0A1FF312811
:103650004FF05B03DFDC1C21ECE76E4B1A68B2F520
:103660002F7F32DB41F25C239342A8BF1346A3F5C0
:103670002F735B22684802FB03F380FB0320DB17F8
:10368000C3EBA0201C305D4BB3F900308342A4D1C2
:10369000624BB3F9003001339FD1A5E7604B1B6843
:1036A000B3F5FA7F11DBB3F57A6FA8BF4FF47A63F5
:1036B000A3F5FA725B485B2303FB02F380FB032054
:1036C000DB17C3EB20201C30DDE71C20DBE7564B6B
:1036D0001B68B3F5FA7F33DBB3F57A6FA8BF4FF4FD
:1036E0007A63A3F5FA724F485B2303FB02F380FB76
:1036F0000320DB17C3EB20201C304C4B1B68B3F5B9
:10370000FA7F1FDBB3F57A6FA8BF4FF47A63A3F596
:10371000FA7244495B2303FB02F381FB0321DB17AD
:10372000C3EB21211C31354BB3F9003083427FF4C8
:1037300056AF3A4BB3F900308B427FF450AF53E7AA
:103740001C20DAE71C21EEE7012005F02DFE6FF4C6
:1037500095733238364A03FB00F082FB0023C01712
:10376000C0EB632303F5AF73312B3ADDB3F5AF7FC5
:10377000A8BF4FF4AF735B22323B244D02FB03F32F
:1037800085FB0325DB17C3EB65151C35002005F011
:103790000BFE6FF495733238254A03FB00F082FB71
:1037A0000023C017C0EB632303F5AF73312B1ADD81
:1037B000B3F5AF7FA8BF4FF4AF735B22323B134921
:1037C00002FB03F381FB0321DB17C3EB61111C3107
:1037D0000A4BB3F90030AB4207D02846FFF7BAFED8
:1037E000FFE61C25D2E71C21F2E70C4BB3F90030B1
:1037F0008B42F2D1F5E600BF889AFF1FAA89FF1F0E
:103800008E9AFF1F6499FF1FA09AFF1F4B48371B1A
:10381000349AFF1F609AFF1FD3058541AC89FF1FB3
:103820006C9AFF1F011FB8124C99FF1F009AFF1FCF
:1038300067BBCF462DE9F04FDFF8EC82B74CB8F903
:1038400000604D7854F8264087B08246039305B156
:103850000D78DFF8FCB2002A34D19BF800308BBB26
:10386000AF4EB6F90000002800F0CE80012800F02D
:103870002481012032232A46019000935146A94B0E
:103880002046FFF7B7FD00250746B6F90030022BAA
:1038900040F3F48000233380B8F90030A24A002BB3
:1038A000C0F2F880042BC4BF00231380039B002BBD
:1038B00040F0F680002D0CBF38464FF0FF3007B0C7
:1038C000BDE8F08F964EE36822689848049300277D
:1038D000059237808BF8007003F080FC1120FFF711
:1038E0003FFD4FF0010919232821CDF804900091E4
:1038F000242219468D4803F0C9FF78232821242269
:10390000CDF8049000918948194603F0BFFF49465D
:10391000864804F051FB02221921844804F048FB38
:10392000DDF81490484608F06BFE494602467F4891
:1039300004F042FC7D4804F055FC394614227B48D3
:1039400004F036FB03227A49784804F035FC7748C6
:1039500004F048FC39462322744804F029FB032272
:103960007449724804F028FC704804F03BFC049B46
:10397000002B72D10123704A18461370FFF7D0FC58
:10398000208963896768191A5C293A885BDC131AF5
:103990005C2202FB03F292FBF1F31B33674A63489C
:1039A000138001271BB21A2219468DE884001422C5
:1039B00003F06CFF049BDBB1218A638AE768581A25
:1039C0005C283A886FDD521A02EB4202C2EB4212C7
:1039D000431C92FBF3F31B33524A544813800127D4
:1039E00038221BB28DE884001946322203F04EFFC4
:1039F000534A544BB6F90000012111704FF6FF7283
:103A00001A8000287FF432AFDFF848914E4AD9F887
:103A100000301268C3EB0A0393424CD9464B1A7824
:103A2000012A18BF012018700127FFF779FCC9F897
:103A300000A0012D4ED0042D59D0022D60D0082DAC
:103A400064D0002521E7121A02EB4202C2EB4212B7
:103A50004B1C92FBF3F31B33A0E72F20FFF780FCF6
:103A600039463222314804F0A3FA032237492F485D
:103A700004F0A2FB2D4804F0B5FB7BE77FF40CAF0C
:103A8000E368002B3FF406AFB8F90030264A002B5C
:103A9000BFF608AF04231380039B002B3FF40AAF4B
:103AA000FFF780FD06E7511A5C2202FB01F292FB50
:103AB000F0F31B3390E70746BBE7002714238DE89C
:103AC00088002A4651461D4B2046FFF793FC3D4691
:103AD0000746DAE6B8F800308BF800500133A8F852
:103AE0000030636983B1002520469847CDE6B8F8D9
:103AF00000300122013BA8F800308BF80020F0E7ED
:103B0000012333800025C7E61D46BEE66369002217
:103B100032804FF0FF35002BE6D1BDE6B089FF1FA4
:103B2000929AFF1F8C9AFF1F8E9AFF1FA09AFF1F69
:103B300014CD000018CD0000149BFF1F8A9AFF1FB0
:103B4000889AFF1FAA89FF1F50D300001CCD0000D8
:103B5000909AFF1F109BFF1F064B074A10B41C884A
:103B6000064B0846002C14BF11461946042210BC0F
:103B700008F0B4BD4E9AFF1F38D400003CD40000BA
:103B8000064B074A10B41C88064B0846002C14BF8D
:103B900011461946042210BC08F0A0BDDC99FF1F95
:103BA00038D400003CD40000064B074A10B41C88EF
:103BB000064B0846002C14BF11461946042210BCBF
:103BC00008F08CBD049AFF1F38D400003CD40000DC
:103BD000064B074A10B41C88064B0846002C14BF3D
:103BE00011461946042210BC08F078BD429AFF1F06
:103BF00038D400003CD40000064B074A10B41C889F
:103C0000064B0846002C14BF11461946042210BC6E
:103C100008F064BD1C9AFF1F38D400003CD400009B
:103C200070B5284E05460FCE86B06C460FC496E898
:103C3000030044F8040B2320218004F071FC40F6BB
:103C4000B833984230DC204B40F6F50219889B7857
:103C5000ADF80D1090428DF80F302DDD00EB4000D7
:103C60001A4B1B491B4E00EB0010C21783FB00438D
:103C7000C2EB632381FB0314D917C1EBA40101EB51
:103C8000810186FB0040C2EB6030A3EB4103303082
:103C900030338DF811008DF813306946284616220E
:103CA00008F01CFD06B070BD0B4B1A889B78ADF870
:103CB0000D208DF80F30D1E7084B1868CDF81100B2
:103CC000EBE700BF50D4000040D40000976A3E2BC1
:103CD000676666668BAA30454CD4000044D4000069
:103CE000F8B5174C174E2278174D33782F888E462B
:103CF000003218BF012201467046FFF79BFD0023EA
:103D000098423370237015DB14BF012000202B88EC
:103D10009F420ED040F23A72A3F5AF730B490C4CA0
:103D200002FB03F381FB0312DB17A3EB62133233B5
:103D30002360F8BD0749012218460A702270E6E7A1
:103D4000E48AFF1F329BFF1F149AFF1FB5814E1B91
:103D50006C89FF1F989AFF1F08B500210D2005F000
:103D6000F5F8962005F02EF901210D2005F0EEF86A
:103D7000962005F027F900210D2005F0E7F89620A0
:103D800005F020F901210D20BDE8084005F0DEB85E
:103D9000014B187801F0D2BF8C99FF1F144BB3F977
:103DA000003070B583EAE375A5EBE375002BACB288
:103DB0001ADB012300E0034603EB83004000854249
:103DC000F9DA0C4E94FBF3F086FB03E503FB104499
:103DD000DB173030D3EBA503A4B201F8010BF1D10E
:103DE00005480B70106070BD2D230B700131E0E7AA
:103DF0007099FF1F6766666668D40000134BB3F9BD
:103E0000003030B583EAE374A4EBE374002BA0B276
:103E100018DB012300E0134603EB830252009442B7
:103E2000F9DA0B4D90FBF3F285FB03E403FB120080
:103E3000DB173032D3EBA40380B201F8012BF1D1B0
:103E40000B7030BD2D230B700131E2E7A889FF1FF5
:103E500067666666134BB3F9003030B583EAE374E6
:103E6000A4EBE374002BA0B218DB012300E013469F
:103E700003EB830252009442F9DA0B4D90FBF3F20C
:103E800085FB03E403FB1200DB173032D3EBA40302
:103E900080B201F8012BF1D10B7030BD2D230B70D6
:103EA0000131E2E76489FF1F67666666134BB3F969
:103EB000003030B583EAE374A4EBE374002BA0B2C6
:103EC00018DB012300E0134603EB83025200944207
:103ED000F9DA0B4D90FBF3F285FB03E403FB1200D0
:103EE000DB173032D3EBA40380B201F8012BF1D100
:103EF0000B7030BD2D230B700131E2E76A89FF1F83
:103F000067666666134BB3F9003030B583EAE37435
:103F1000A4EBE374002BA0B218DB012300E01346EE
:103F200003EB830252009442F9DA0B4D90FBF3F25B
:103F300085FB03E403FB1200DB173032D3EBA40351
:103F400080B201F8012BF1D10B7030BD2D230B7025
:103F50000131E2E76689FF1F67666666134BB3F9B6
:103F6000003030B583EAE374A4EBE374002BA0B215
:103F700018DB012300E0134603EB83025200944256
:103F8000F9DA0B4D90FBF3F285FB03E403FB12001F
:103F9000DB173032D3EBA40380B201F8012BF1D14F
:103FA0000B7030BD2D230B700131E2E77089FF1FCC
:103FB00067666666F0B40C4D0C4F0E460FCD8CB0A4
:103FC00001AC0FC40FCD0FC495E807003B8884E80F
:103FD00007000CAA02EB8303304653F82C1C042282
:103FE0000CB0F0BC08F07ABBA4CD00006299FF1FB2
:103FF00030B40A4B0A4D0C4693E8070084B02B8876
:1040000004AD05E9070005EB8303204653F80C1CBB
:10401000042204B030BC08F061BB00BFD0CD00006A
:10402000EC99FF1FF0B40A4D0A4F0E460FCD86B033
:1040300001AC0FC42A683B88226006AA02EB830306
:10404000304653F8141C0C2206B0F0BC08F046BBF6
:10405000DCCD00004C9AFF1F054B1B881BB9054B9C
:10406000186808607047044B18680860704700BF04
:104070007E99FF1F70D400006CD40000164B1B8883
:104080000BB31BB230B583EAE374A4EBE374002BEB
:10409000A0B21CDB012300E0134603EB83025200B5
:1040A0009442F9DA0D4D90FBF3F285FB03E403FB38
:1040B0001200DB173032D3EBA40380B201F8012BDE
:1040C000F1D10B7030BD064B1868086070472D2386
:1040D0000B700131DEE700BFF699FF1F6766666669
:1040E0003CD40000164B1B880BB31BB230B583EADF
:1040F000E374A4EBE374002BA0B21CDB012300E00B
:10410000134603EB830252009442F9DA0D4D90FB03
:10411000F3F285FB03E403FB1200DB173032D3EB31
:10412000A40380B201F8012BF1D10B7030BD064B16
:104130001868086070472D230B700131DEE700BF5F
:10414000289AFF1F676666663CD40000164B1B88E2
:104150000BB31BB230B583EAE374A4EBE374002B1A
:10416000A0B21CDB012300E0134603EB83025200E4
:104170009442F9DA0D4D90FBF3F285FB03E403FB67
:104180001200DB173032D3EBA40380B201F8012B0D
:10419000F1D10B7030BD064B1868086070472D23B5
:1041A0000B700131DEE700BF4099FF1F676666664E
:1041B00074D40000174B1B881BB31BB270B583EA85
:1041C000E375A5EBE375002BACB21EDB012300E029
:1041D000034603EB830040008542F9DA0E4E94FB60
:1041E000F3F086FB03E503FB1044DB173030D3EB21
:1041F000A503A4B201F8010BF1D108480B701060BF
:1042000070BD074B1868086070472D230B70013193
:10421000DCE700BF209AFF1F6766666678D400005F
:104220003CD40000164B1B880BB31BB230B583EA9D
:10423000E374A4EBE374002BA0B21CDB012300E0C9
:10424000134603EB830252009442F9DA0D4D90FBC2
:10425000F3F285FB03E403FB1200DB173032D3EBF0
:10426000A40380B201F8012BF1D10B7030BD064BD5
:104270001868086070472D230B700131DEE700BF1E
:104280005099FF1F676666663CD40000184B1A8879
:1042900052B3184A128830B50A80B3F90030002BA7
:1042A00083EAE374A4EBE374BCBF2D238B70A0B24C
:1042B000ACBF02310331012300E0134603EB83025C
:1042C00052009442F9DA0C4D90FBF3F285FB03E4C3
:1042D00003FB1200DB173032D3EBA40380B201F8EA
:1042E000012BF1D10B7030BD044B1868086070478A
:1042F0002E9AFF1F7CD40000676666663CD40000DF
:10430000174B1B881BB31BB270B583EAE375A5EB93
:10431000E375002BACB21EDB012300E0034603EB88
:10432000830040008542F9DA0E4E94FBF3F086FBE1
:1043300003E503FB1044DB173030D3EBA503A4B235
:1043400001F8010BF1D108480B70106070BD074BEC
:104350001868086070472D230B700131DCE700BF3F
:10436000849AFF1F6766666678D400003CD400001C
:10437000054B1B881BB9054B186808607047044B38
:1043800018680860704700BFB299FF1F84D400000E
:1043900080D40000054B1B881BB1054B18680860D2
:1043A0007047044B18680860704700BF829AFF1F6F
:1043B0008CD4000088D40000F0B480EAE075A5EB4E
:1043C000E0750028ACB21FDB1DBF2B230B704E1C09
:1043D0000E46012300E0134603EB83025200954290
:1043E000F9DA0B4F94FBF3F287FB030503FB12444E
:1043F000DB173032D3EBA503A4B206F8012BF1D1C1
:1044000033700846F0BC70472D230B704E1CE0E75C
:1044100067666666054B18880C2803D00C3800B216
:10442000FFF7CABF024A1068086070477C9AFF1FF6
:1044300090D40000024B1888183800B2FFF7BCBFB8
:10444000549AFF1FC3681888183800B2FFF7B4BF2A
:10445000034B1888A0EB8000400000B2FFF7ACBF10
:104460008C99FF1F024B1888033800B2FFF7A4BFD6
:10447000E499FF1F024B18880C3800B2FFF79CBF6D
:104480008099FF1F30B5134C85B001252B463C2287
:1044900002212046009502F0C7FC204602F09EFE55
:1044A00000224021802320460191009311460A4BAF
:1044B000029503F041FB204602F09CFF07480849A3
:1044C000084A0023036083800B608B801360938015
:1044D00005B030BDA09AFF1F48CE0000009BFF1F13
:1044E0002C9BFF1F1C9BFF1F10B500EBC00000F1B1
:1044F0000F02D2B293B284B09C1E981C3D2303914C
:104500008DE819003921024803F07AFA04B010BD91
:10451000A09AFF1F70B5CEB20C46054604F0E4F831
:10452000864203D03146284604F0F8F80135284683
:1045300004F0DAF8240A844205D021462846BDE872
:10454000704004F0EBB870BD38B5FDF717FB0D4BAC
:104550001B7833B90C4B10201988FFF7DBFF0120C3
:1045600038BD0A4D0A4C2B782288B3FA83F382F0C7
:1045700008025B09114642202B702280FFF7CAFF18
:10458000002038BD4899FF1FB899FF1F689AFF1F88
:10459000AE99FF1F024B10201988FFF7BBBF00BF69
:1045A000B899FF1F024B4E201988FFF7B3BF00BF19
:1045B0007E99FF1F024B44201988FFF7ABBF00BF55
:1045C000549AFF1F024B2C201988FFF7A3BF00BF8E
:1045D000169AFF1F024B1E201988FFF79BBF00BFD2
:1045E000F699FF1F70B55C4D2B780646002B35D130
:1045F0001C4673780BB9204670BDFDF7BFFA574AC9
:10460000574B5848127831781B78007802EB4303F7
:104610004A1E03EB80030E2AEDD801A050F822F0C9
:10462000AD460000CF460000F7450000AD46000053
:10463000F7450000F7450000F74500007746000009
:10464000F7450000F7450000F7450000F74500007A
:10465000F7450000F745000073460000AE214248D0
:1046600002F06CFB404802F0B9FD00232B700124DE
:10467000BFE704F0B9FF3D4B3D491B78002B3DD00F
:104680003C4B3D4A09881B8812680B44B2EB630F10
:1046900059DA3A4B1B78002B4BD0AF21324802F04D
:1046A0004DFB374A012313702B70A4E783B93548BB
:1046B000038804294FF6FF7103F1FF320CBF012379
:1046C0000B46134403F07F03013303800FE073B103
:1046D000013B2D4A32F813304BB12A4E2B482C495E
:1046E0002C4A33800123002606700B701370244A75
:1046F0000221012311702B70204670BD1D4B1E4AF4
:1047000009881B8812680B44B2EB630FC5DB224E8D
:10471000224D33882A88B3FA83F382F002025B09C0
:104720003380114642202A80FFF7F4FEFFF714FB86
:1047300061E7AF210C4802F001FB114A0621012379
:1047400011702B7057E7164E144D33882A88B3FA30
:1047500083F382F00402E2E7E48AFF1F7E9AFF1FE0
:10476000B499FF1F809AFF1FA09AFF1F4899FF1F4F
:10477000529AFF1FEE99FF1F6C9AFF1FA599FF1F0A
:10478000989AFF1F8299FF1F5499FF1F699AFF1F74
:10479000E699FF1F089BFF1F4E9AFF1FAE99FF1F50
:1047A000DC99FF1FC3680E201988FFF7B3BE00BF56
:1047B000024B28201988FFF7ADBE00BFE499FF1F08
:1047C000064A07491388098823F0020343EA410394
:1047D0009BB2194642201380FFF79CBEAE99FF1F83
:1047E0004E9AFF1F064A07491388098823F00403DD
:1047F00043EA81039BB2194642201380FFF78ABE29
:10480000AE99FF1FDC99FF1F064A074913880988E4
:1048100023F0100343EA01139BB219464220138090
:10482000FFF778BEAE99FF1F049AFF1F064A07499B
:104830001388098823F0200343EA41139BB21946E9
:1048400042201380FFF766BEAE99FF1F429AFF1FFA
:10485000024B5A201988FFF75DBE00BF7099FF1FF9
:10486000024B16201988FFF755BE00BF4099FF1F65
:10487000024B2E201988FFF74DBE00BF209AFF1F64
:10488000024B30201988FFF745BE00BF5099FF1F2B
:10489000024B18201988FFF73DBE00BFEC99FF1F9F
:1048A000024B1A201988FFF735BE00BF2E9AFF1F52
:1048B000024B1C201988FFF72DBE00BF4C9AFF1F2A
:1048C000024B20201988FFF725BE00BF849AFF1FE6
:1048D000024B32201988FFF71DBE00BF7C9AFF1FD4
:1048E000024B52201988FFF715BE00BFA889FF1F91
:1048F000024B50201988FFF70DBE00BF6489FF1FCF
:10490000024B54201988FFF705BE00BF6A89FF1FBC
:10491000024B5C201988FFF7FDBD00BF6689FF1FB1
:10492000024B5E201988FFF7F5BD00BF7089FF1F9D
:10493000024B60201988FFF7EDBD00BFB299FF1F41
:10494000024B56201988FFF7E5BD00BF829AFF1F72
:1049500038B5054603F0C8FE4FF0000460F30704C5
:10496000681C03F0C1FE60F30F24A0B238BD00BF85
:1049700038B5094D46242046FFF7EAFF35F8021BFB
:1049800000B28842204601D0FFF7C4FD0234E4B2F1
:104990004E2CF0D138BD00BF449AFF1F08B512203D
:1049A000FFF7D6FF054B1988884206D01220FFF783
:1049B000B1FDBDE8084001F041B908BD6299FF1F93
:1049C00008B55820FFF7C4FF054B1988884206D068
:1049D0005820FFF79FFDBDE8084001F02FB908BD42
:1049E000289AFF1F08B51420FFF7B2FF054B19885E
:1049F000884206D01420FFF78DFDBDE8084001F085
:104A00001DB908BD1C9AFF1F014B01221A70704787
:104A1000329BFF1FF0B585B003F01EFE4D4C4E4B90
:104A200002934E4A01920423009320464C4B4D4F73
:104A30004D4E4E4D4022802101F0FEFF20464C4C51
:104A40004C4A4D4907F066FAA7614C484C4FE76164
:104A50004C4F87614C494D4FC7614D4F8F614D4A57
:104A60004D4FCF614D4F97614D4B4E4FD7614E4FDC
:104A70009F614E4FDF614E4FB7614E4FF7614E4F12
:104A8000AF614E4C4E4FEF614E4FA7614E484F4FB6
:104A9000E7614F4F87614F494F4FC7614F4F504AB2
:104AA0008F61504FCF61504F504B9761504FD7613E
:104AB000504F514E9F61514FDF61514F514DB76182
:104AC000514FF761514F524CAF61524FEF61524F0E
:104AD0005248A761524FE761524F53498761534F84
:104AE000C761534F8F61534A534FCF61534F976103
:104AF000534B544FD761544F9F61544E544FDF6115
:104B0000544F554DB761554FF761554F554CAF61F7
:104B1000554F56485649EF61564F574DA761E561CD
:104B2000564F574D574CDFF880E1574A574B876136
:104B3000C5618C61564E574F574D584CC1F81CE01B
:104B4000574858499761D5619C61D861B16005B0FB
:104B5000F0BD00BFA09AFF1FA0860100801A0600CA
:104B6000388EFF1F75440000D48BFF1FD88DFF1FA8
:104B7000F88BFF1F1C89FF1F916A0000C08AFF1F6E
:104B8000A547000065440000FC8AFF1FB1470000F4
:104B9000593B0000908DFF1FC1470000813B000082
:104BA0001C8CFF1FE5470000A93B000009480000DE
:104BB000D13B00002D48000051440000108DFF1F24
:104BC000913D0000B53F0000448BFF1F9D49000050
:104BD000E54000008C8BFF1FC14900009D3D000097
:104BE000E889FF1F51480000F93B0000B48DFF1F0A
:104BF000E54900004D410000688BFF1F614800003F
:104C0000B54100003C8AFF1F7148000025420000AA
:104C1000208BFF1F81480000F13F00009C8AFF1F8E
:104C2000914800008D420000648CFF1FA1480000E5
:104C300025400000B08BFF1FB14800000143000079
:104C40004C8DFF1FC148000015440000608AFF1F03
:104C5000D1480000FD3D00000C8AFF1FE148000024
:104C6000553E0000C489FF1FF1480000C88CFF1F9B
:104C7000EC8CFF1FAD3E000001490000053F000025
:104C8000114900005D3F0000FC8DFF1F408CFF1F9D
:104C9000308AFF1F71430000314900009543000036
:104CA0004149000019500000214900002DE9F04F52
:104CB0002F4DDFF8CCB0DFF8C4A0DFF8C8900FCDDF
:104CC00091B003AC0FC40FCD0FC40FCD0FC42B6830
:104CD00023600025A8462F462E4600E09846BAF8E5
:104CE000003024495BF8232028461123FBF796FF68
:104CF00000EBC00400EB840089FB00340444C017BF
:104D0000C0EB6434C4F13C00C6F13C0207F1410140
:104D1000012600B208F1410300901BB2019612B2C5
:104D200009B2154802F0B2FD08EB060305F21115B1
:104D30003C2B2646ADB24746D0D134226B210E48DB
:104D400003F036F900210C4803F036F90B4B1B88B1
:104D500010AA02EB830353F8344C204607F050FCB2
:104D600002460548214611B0BDE8F04F03F024BAD1
:104D7000F0CD0000C0CA0000A09AFF1F169AFF1FC6
:104D8000E0CB0000090002802DE9F043804685B0A9
:104D9000002956D10121304803F00EF92F4998F827
:104DA000062098F8083011F80290994522DA4FEA67
:104DB00089064D460C24D8F80C3027489B595F686B
:104DC00022B2002103F0F4F8384607F019FC394606
:104DD0000246214803F0F0F91F4803F003FA98F85F
:104DE000083001350934AB42A4B206F1040601DDF6
:104DF000422CE0D1B9F1000F13D109F10609994510
:104E00000CDA3C2301213B2203910293009301928F
:104E100039233F223A21104802F0F2FD05B0BDE8E7
:104E2000F0830F2301213B2203910293009301920F
:104E300039230C223A21084802F0E2FD98F80830A4
:104E4000DBE700213423009301913F230C22024829
:104E500002F0EAFC9EE700BFA09AFF1F2C9BFF1FF9
:104E600010B5104C0121204603F0ACF8204601217A
:104E700003F0A2F820463422552103F099F8204689
:104E80000222094903F098F920460522074903F058
:104E900093F9204603F0A6F92046BDE8104002F041
:104EA000A9BA00BFA09AFF1F94D4000098D40000B4
:104EB00070B50D46064607F0A3FB00EB40008400EA
:104EC000002D36D0284607F09BFB00EB4000400049
:104ED00023185B1003F16001091A282209B2174850
:104EE000C3F1600403F064F80121144803F064F88E
:104EF000284607F085FB29460246104803F05CF976
:104F00000E4803F06FF902210C4803F055F821B266
:104F100021220A4803F04CF8304607F071FB314675
:104F20000246064803F048F90448BDE8704003F023
:104F300059B96410C4F16004E5E700BFA09AFF1FEF
:104F4000214B70B5B3F9003083EAE374A4EBE3744A
:104F5000002B82B0A1B22FDB68466D46012300E032
:104F6000134603EB830252009442F9DA174E91FB89
:104F7000F3F286FB03E403FB1211DB173032D3EBB1
:104F8000A40389B205F8012BF1D119462B70FFF764
:104F90008FFF0F4B1B786BB101210E4803F00CF80B
:104FA000332274210B4803F003F801220A4909480F
:104FB00003F002F902B070BD2D238DF800300DF121
:104FC00001056846CAE700BFB899FF1F67666666B5
:104FD000689AFF1FA09AFF1F88D6000010B50D4BDE
:104FE0001B5C51F82340237884B013B1012004B036
:104FF00010BD04AA01A942F8103D2046A3699847B4
:10500000A38A9B07F2D401A80099FFF751FF012062
:1050100004B010BD009BFF1FF8B51F4D287840B9A4
:105020001E4B1B68994203D31D4A012313702B703A
:10503000F8BD0C4600261B48184F02F0CFF804F6C6
:10504000B833324617483B6031212E7002F0B0FF72
:105050000121144802F0B6FF3146124802F0ACFFBD
:10506000052211490F4803F0A7F80E4803F0BAF8DB
:105070000C2210210B4802F09BFF0B220B49094820
:1050800003F09AF805220A49064803F095F8054806
:1050900003F0A8F80120F8BDE48AFF1F189BFF1F4A
:1050A000989AFF1FA09AFF1FA0D40000A8D4000068
:1050B00098D4000010B5424C424882B002F08EF8FD
:1050C0002378C3B906213F4802F076FF2378012BED
:1050D00037D90A22022B11463A486BD002F068FFFA
:1050E00039490322374803F067F8364802B0BDE873
:1050F000104003F077B8354B1A7801210523002AB8
:1051000035D10191009311462E4802F00FFC304B2F
:105110001A78002A36D0052301220192009300223A
:105120000A21284802F080FB2A4B1A78002A35D140
:1051300001210523019100931421224802F0F6FB7E
:10514000C0E7254C2388092B32D9632B8CBF0A2159
:105150001F210A221B4802F02BFF2188194803F067
:1051600091F8184802B0BDE8104003F03BB80022A7
:10517000019100931146134802F056FB144B1A7824
:10518000002AC8D105230121019100930A210D486D
:1051900002F0CCFB0F4B1A78002AC9D0012205235C
:1051A0000192009300221421064802F03DFB89E79A
:1051B0003021CEE702F0FCFE0322084992E700BF4F
:1051C000089BFF1FA09AFF1FB8D400007E9AFF1F04
:1051D000B499FF1F809AFF1F8299FF1FB4D400006B
:1051E0002DE9F041754C2278002A05460F4614BF80
:1051F0004FF001084FF000084ED1714E3368CB1AC2
:10520000B3F5FA6F04D86B78A3B94046BDE8F081D6
:105210006C4B6D486D49DFF8D0E11A7001230370C3
:105220000988237026208EF80020FFF773F96B7829
:10523000002BEAD03760FCF7A1FC654A654B664954
:10524000127828781B78097802EB4303421E03EB9F
:1052500081030E2AD9D801A151F822F04D53000044
:10526000195300000B5200004D5300000B52000078
:105270000B5200000B520000015300000B520000C3
:10528000B35200000B5200000B5200000B52000002
:105290000B520000AF520000AF215048484E01F0C1
:1052A0004DFDFFF707FF002337602370ABE704F0E5
:1052B0009BF94A4801F092FF0221484802F07CFE27
:1052C0000F222321454802F073FE0522444943483A
:1052D00002F072FF414802F085FF1E2223213F4861
:1052E00002F066FE05223F493C4802F065FF3B485C
:1052F00002F078FF394802F07DF800F0ABFC84E75B
:10530000394D2B78012B50D9304B26201988FFF7C7
:1053100001F900232B7078E7002B3FF476AF013BB7
:10532000324A32F81330002B3FF46FAF274C30482D
:1053300025492D4A23804FF001080023037081F88E
:10534000008082F80080FFF7B5FE5EE793B1013B75
:10535000264A32F8131019B31C4B254D1A4C224A19
:1053600019800026012326202E7023701370FFF76A
:10537000D1F815E0154C1E4922880B7004284FF611
:10538000FF7002F1FF310CBF012202460A440E4EAB
:10539000154D02F07F0201320121228031702B7005
:1053A000FFF788FE4FF001082FE70649064A012360
:1053B0000020087013702370A6E700BFE48AFF1F67
:1053C000289BFF1F989AFF1FE699FF1F8299FF1FD6
:1053D0007E9AFF1FB499FF1F809AFF1FA09AFF1F9C
:1053E000BCD40000C4D40000089BFF1F5499FF1FC9
:1053F000699AFF1F2DE9F04F05468BB00F46AD4867
:105400000121164602F0DEFDAA8812F0010440F0E8
:10541000B180DFF8CC8298F80030002B7ED1AB79D8
:10542000A54AD15CA1B9DFF8BCA279781AF803903B
:1054300041B339780139072900F2B880DFE811F06B
:10544000F2005401B6006C01B600B600B600EA00E6
:105450007C78002C00F0CB800139EC68387854F867
:105460002170FC68411EB4F80080072900F2A88072
:10547000DFE811F074015901A6006C01A600A60036
:10548000A600A000DFF854A2DAF80020B21AB2F5A4
:10549000967F76D9894A107801281ABF01201070AA
:1054A0001170874A18BF0146D05CC0EB0900C0B23A
:1054B000FFF71AF80124CAF80060AB889B0771D582
:1054C0007B78002B6ED0FCF759FB7E4B7E4A7F48E1
:1054D0001B78127839780078022515FB02330A29E7
:1054E00003EB800300F04E810C295BD1002B59D0D7
:1054F00003F11900764E774A013B0021400000F08D
:10550000FE0026F813100123157088F80030FFF70D
:1055100001F8714B032220461A702FE0654801F014
:105520005DFE0121634802F047FD624822462146A4
:1055300002F03EFDAB88580725D42C68204607F0C2
:105540005FF8214602465B4802F036FE594802F0F9
:1055500049FE092201238DE80C0000217F235548D4
:1055600002F094F900212846FFF70EFC002388F88A
:10557000003054E7AB683146384698470BB0BDE879
:10558000F08F0846FAE72B6804A8984704A807F0AC
:1055900037F804A90246474802F00EFE454802F0DB
:1055A00021FED6E720460BB0BDE8F08F00240AF8B4
:1055B000039082E70021D1543846FB699847FC6884
:1055C000A4F80080002725223C238DE88400412197
:1055D0001822384802F028F9E968A879FFF7FEFC9C
:1055E000364A3E4B17701E600BB0BDE8F08F3B494A
:1055F0000A68B21AB2F5967FD4D9304F0E603E7861
:10560000012E00F0B380E968184601233B70FFF7D4
:10561000E5FCB3E72F4AE9791170012288F80020F0
:105620000024C4E72A7A013A4A45BFDD09F10106A0
:10563000F6B2B145BAD0224A039212F803B0CBEBCE
:105640000900C0B20021FEF74FFF2B7A052B5C4604
:105650001BD9CBEB06010429039A40F3AB80A6F1DA
:10566000040BBBF1000FC0F2AD80063B9B45A8BF09
:105670009B465FFA8BF4AB791148D25C5A4504D053
:10568000C45401212846FFF77FFB301BC0B2012123
:105690000A4CFEF729FF00213423019100930548AD
:1056A000217040230B223F2102F0BEF8B1460124B5
:1056B000AB797CE7A09AFF1F1C9BFF1F149BFF1F69
:1056C0002C9BFF1F7E9AFF1FB499FF1F809AFF1F1C
:1056D0005499FF1F989AFF1F089BFF1F109BFF1FE5
:1056E000E48AFF1F009BFF1F0FFA89F1E8685F4CF7
:1056F00050F821602168049134785D49049808606D
:10570000002C70D0012C7FF451AF5A4A317A88F8BE
:105710000040117000244AE7B9F1000F50D009F1A0
:10572000FF36F6B285E7B98A01F0040189B2002993
:105730003FF441AF3B6A03929847039A00283FF435
:105740003EAFAB79FC680021D15439E77B8A4345F1
:105750003BD908F101081FFA88F831E73B8A434535
:105760003AD208F1FF381FFA88F829E725238DE897
:10577000180041483C703C231822412102F054F8A3
:105780003046FBE6002B3FF40DAF3C4A3C4E1188FF
:10579000384A5F1E1933580000F0FE00012388F8D4
:1057A000003026F817101570FEF7B4FE354B204672
:1057B0001D70E3E600293FF758AF06F1FF3B50E7C5
:1057C0004C46F4E60024A34655E7BB8ADA077FF58A
:1057D000F7AEB7F81080F3E6BB8AD9077FF5F0AED5
:1057E000B7F81280ECE62849C85CC0EB090009F163
:1057F000010EC0B201214FF0340B02F803E0FEF7B6
:1058000073FEB6681C48019440230B223F210124FB
:10581000CDF800B002F008F840230B223F211648D3
:10582000CDF800B0019402F081F82146124802F050
:10583000C3FB304606F0E4FEA0EB800000F15F0100
:1058400009B20F220C4802F0B3FB304606F0D8FE36
:1058500031460246084802F0AFFC074802F0C2FC9D
:10586000E968A879FFF7BAFBAB79A0E6609BFF1F58
:10587000109BFF1F989AFF1FA09AFF1F8299FF1F7E
:105880005499FF1F089BFF1F2C9BFF1F2DE9F0471A
:10589000DFF808926D4B99F800601B68DFF800A2F2
:1058A00082B0003601934FF0030018BF0126019F1C
:1058B0009AF8008003F050FB0546042003F04CFBEF
:1058C0000446052003F048FB800040EA440406201B
:1058D00003F042FB2C4364B25D4944EAC0000A78FD
:1058E00080F00F03DBB29A425A4A3CD01760002284
:1058F00059480B7003788DF800808DF8012053B360
:10590000564A12684EF66021BA1A8A4219D8022BFA
:1059100059D0012B5FD0062B48D0032B63D0042B2A
:1059200069D0052B77D0072B7DD0082B00F0838022
:10593000092B68D016B14A4801F05CFD02B0BDE801
:10594000F087484A484C00230121237003701360FC
:10595000938089F800103A4669464448FFF74AFDAB
:105960003043C6B2E6E71268BA1A1E2A6BD99AF813
:105970000020934222D0394C3D488AF80030012B58
:10598000276082EA030207609846B1D0042BAFD1AA
:1059900037480068381AB0F5C87FA9D9354C206857
:1059A000381A3228A4D927601A46A1E73A46694630
:1059B0003148FFF71FFD3043C6B2BBE7012B4FF064
:1059C0000002E3D1E4E73A4669462C48FFF712FDAE
:1059D0003043C6B2AEE73A4669462948FFF70AFDAA
:1059E0003043C6B2A6E73A4669462648FFF702FDAD
:1059F0003043C6B29EE73A4669462348FFF7FAFCB1
:105A00003043C6B296E73A4669462048FFF7F2FCB3
:105A10003043C6B28EE73A4669461D48FFF7EAFCB6
:105A20003043C6B286E73A4669461A48FFF7E2FCB9
:105A30003043C6B27EE73A4669461748FFF7DAFCBC
:105A40003043C6B276E7002252E700BF609BFF1FDB
:105A5000229BFF1F949AFF1F989AFF1F0C9BFF1F0A
:105A6000A09AFF1F1C9BFF1F069BFF1F1CD400005A
:105A7000249BFF1F9C9AFF1F64D30000CCD2000020
:105A800054D3000078D2000084D3000074D3000007
:105A900028D40000B8D30000308AFF1FE48AFF1F1B
:105AA000079BFF1F28B11028044BA8BF10201860C7
:105AB0007047024B01201860704700BF349BFF1FE6
:105AC00038B50F4D2B78013B01381B02C4B203F4EB
:105AD0007063200443F4404343F00C0300F4FE00E1
:105AE000184304F0A1FB2868013860F03F00C0B201
:105AF00003F0C8FB2046BDE8384003F0C3BB00BF3D
:105B0000349BFF1F70B5124D2B78013B1B0203F431
:105B10007063064643F430430806320400F0FE404A
:105B200043F00B03034302F4FE0018430C4604F059
:105B30007BFB2868013860F04F00C0B203F0A2FB85
:105B4000304603F09FFB2046BDE8704003F09ABB4F
:105B5000349BFF1F70B5124D2B78013B1B0203F4E1
:105B60007063064643F410430806320400F0FE401A
:105B700043F00903034302F4FE0018430C4604F00B
:105B800053FB2868013860F06F00C0B203F07AFB65
:105B9000304603F077FB2046BDE8704003F072BB4F
:105BA000349BFF1F38B5104D2B78013B1B0203F4CB
:105BB0007063044643F41043000443F0090300F407
:105BC000FE00184304F030FB2868013860F06F00D5
:105BD000C0B203F057FB204603F054FB0020BDE8A1
:105BE000384003F04FBB00BF349BFF1F38B50E4D4C
:105BF0002B78013B1B0203F47063044643F45043CB
:105C0000000443F00D0300F4FE00184304F00CFB05
:105C10002868013860F02F00C0B203F033FB204643
:105C2000BDE8384003F02EBB349BFF1F08B50020B1
:105C300004F05EFB0028FAD108BD00BF08B564215E
:105C40000720FFF75FFF7F210B20BDE80840FFF72B
:105C500059BF00BF10B500217B20FFF753FF002480
:105C6000E0B2FFF79FFF0134022003F0ABF9802C74
:105C7000F6D110BD10B504464FF4406003F0B2FAFF
:105C800003F00AFB2CB1102C044BA8BF10241C609D
:105C900010BD024B01241C6010BD00BF349BFF1FD0
:105CA00010B5044641F0E00003F0ECFA04F07F0088
:105CB00003F0E8FAC4F3C610BDE8104003F0E2BAFE
:105CC00038B5134D2B78044641F6FF72A0F500500D
:105CD000824203F1FF33A8BF02461B0202F50052C5
:105CE00003F47063100443F4604343F00E0300F4C4
:105CF000FE005204184302F0FE42104304F094FAEE
:105D0000296801392046C9B2BDE83840FFF7C8BF4D
:105D1000349BFF1F38B504460D46F02003F0B2FA5D
:105D200035B1254414F8010B03F0ACFAAC42F9D1BB
:105D3000F720BDE8384003F0A5BA00BF00B50B4B13
:105D400083B00246998818680090032AADF80410C1
:105D500002D903B05DF804FB684606218DF80520E2
:105D6000FFF7D8FF03B05DF804FB00BF50D7000079
:105D70000020704790F8392090F83800101A7047CA
:105D800090F8383090F839209A4205D95A1C0344CB
:105D900080F83820187E70474FF0FF30704700BF02
:105DA00090F8383090F839209A4286BF1B18187E38
:105DB0004FF0FF30704700BF704700BF38B5054651
:105DC000B0F85E0090B195F85D301446C3F1210241
:105DD00094420CD805F13B001844224602F0CEFC58
:105DE00095F85D30234485F85D30204638BD0120AC
:105DF00014462871EEE700BFB0F85E306BB190F842
:105E00005D30202B07D8C218013380F85D300120A7
:105E100082F83B107047012303710020704700BFD8
:105E20000023426980F8383080F8393080F85C30DF
:105E300080F85D3080F85E3080F85F3006CA30B49C
:105E40000D68046943662A4383660A60A370426949
:105E500090F861301649146813441D7A5B7B01EB9E
:105E6000C5051B026D6803F4E06343F064032B6017
:105E700090F8623013449D7CDB7D01EBC5011B0271
:105E8000496803F4E06343F064030B6021685368DE
:105E9000194205D0036927225A70036904229A71B6
:105EA000036920225A71036980229A7030BC7047BE
:105EB00084E2000043690CCB12681A420CD0094BF3
:105EC00099420AD9084B9942036994BF1A220D22BC
:105ED0005A70036904229A717047036927225A7025
:105EE000F7E700BF7F1A06003F420F0010B50269B6
:105EF000D378DBB2D90604463DD510215806D170BF
:105F000038D503F0040303F0FF02002B51D03D49C4
:105F1000626E00230B7084F85D30002A5BD09047DE
:105F200094F85D30002B56D02369D0229A702369F3
:105F300094F83B201A712369012284F85C20022224
:105F4000DA7010BD304B84F860009C424AD02F4B71
:105F50009C4252D094F8391013791F29DBB207D82C
:105F60002848007820B16018013184F83910037690
:105F70000223D37010BD5906C3D4917801F01001EB
:105F800001F0FF000029DDD013F001031ED194F8C9
:105F90005C1094F85D00884281BF4B1C091984F89D
:105FA0005C3091F83B3013712369D0229A702269DA
:105FB000DEE7236984F83920C0229A702369114AE8
:105FC0001979012111700222DA7010BDC02393707B
:105FD00022691379CCE70122002384F85D2084F83C
:105FE0003B30A1E7626994F8613009491344032208
:105FF000187A02F049FD2269ACE7626994F86130D1
:106000000449F3E7389BFF1F388EFF1FA48EFF1F44
:1060100075600000816000000369DB7803F02003F5
:1060200073B190F860300133DBB2012B80F860303F
:106030001AD9426990F861301344187A02F0A0BD71
:1060400070B5426903F0FF0590F8613013440446CF
:10605000187A02F095FDA36E5BB184F8385094F87D
:106060003900BDE87040184790F85F30002BE0D051
:10607000704770BD0148FFF7CFBF00BF388EFF1FCC
:106080000148FFF7C9BF00BFA48EFF1F2DE9F047ED
:10609000374FDFF8E0903B68026982B00646009314
:1060A000DDF800800021A025D3789B065BD53B68F6
:1060B0000193019BC8EB03030F2BF5D949B1102BBA
:1060C000F2D000209070336980229A7002B0BDE84F
:1060D000F087726996F8613013440521187A02F04E
:1060E00049FF726996F861301344012193F812A0B8
:1060F000504602F03FFF09240021504602F026FFDF
:106100002B46013BFDD10121504602F01FFF2B46DB
:10611000013BFDD1013CEFD1706996F8611001445B
:106120004FF4A0720C7A4B7B09EBC4011B02496847
:1061300003F4E06343F064030B6096F862300344B9
:10614000997CDB7D09EBC1011B02496803F4E06324
:1061500043F064030B60013AFDD13269D3789B06AA
:106160004FF00101A3D4012002B0BDE8F08700BFC9
:10617000609BFF1F84E20000F0B503691222DA7011
:106180000269937803F0200385B004460D46002B86
:106190005ED0B42393703C4922690B680093009E43
:1061A00005E00B680193019B9B1B042B42D8D3781D
:1061B00003F0200303F0FF00002BF2D094F85D30D1
:1061C000002B31D04FF0000E4FF0020C04EB0E0309
:1061D00093F83B3013710B680393039F206907E02A
:1061E0009B060DD50B680293029BDB1B052B28D861
:1061F000C378DBB203F0020202F0FF06002AEFD000
:1062000080F803C02669F378DBB2DF0632462DD46E
:106210009F062BD5DB0731D40EF1010E94F85D30CB
:106220005FFA8EFE7345D1D800201DBB002384F891
:106230005E3004E09070236980229A70042005B0DB
:10624000F0BD86702369802204209A7005B0F0BDED
:1062500003F0FF06FFF71AFF10B9042005B0F0BDE8
:10626000236984F85F60B0229A7094E78023B3704A
:106270000420DAE726698023B370D7E7BEF1000F68
:106280000CBF02200320F6E7609BFF1F2DE9F041C1
:1062900006690025122780F8385080F83950F770C9
:1062A000D0F810C09CF802E00EF0200E88B0044632
:1062B000884615461E46BEF1000F49D0B4238CF81F
:1062C0000230784B21691A680092DDF800E006E0A0
:1062D0001A6801920198CEEB0000042830D8C878E3
:1062E00000F0200000F0FF070028F1D04FEA48023C
:1062F00042F00102D2B20A711A680292DDF808E097
:10630000206906E01A6803920399CEEB0101052982
:106310002AD8C17801F0020101F0FF070029F1D06D
:106320004FF0020C80F803C02269D17811F01107F8
:1063300022D12DBB002E0CBFA0238023937003E03D
:106340008F70236980229A70384608B0BDE8F081CA
:106350000EF0FF07FFF79AFE0028F5D0236984F8B6
:106360005F70B0229A70ACE787702369802238464C
:106370009A7008B0BDE8F081802393700027E3E7AE
:10638000012D75D0A021917021690A79BE4667461A
:106390004FF0A80C1A680492049805E01A68059258
:1063A000059A121A052A4AD8CA7802F0020202F0A7
:1063B000FF08002AF2D0CF702169CA78D2B212F059
:1063C000100F08465AD1920658D5013DEDB2012D65
:1063D00049D0BEF11F0F3BD90A79012DDAD11A68D5
:1063E0000692069D05E01A680792079A521B052A35
:1063F00046D8C27802F0020202F0FF01002AF2D071
:106400000223C3702269D378DBB2D9063AD49B0643
:1064100034D5B023BEF11F0F93703FD8226904EB2F
:106420000E0312791A760EF1010E5FFA8EFE16B186
:10643000236980229A7084F839E0774684E781F8EE
:106440000280236980229A70774684F839E07BE7DE
:1064500004EB0E0291F8048082F818800EF1010E10
:106460005FFA8EFEB9E781F802C021690846B0E7FD
:10647000A82191702069BE460279B0E7774663E7AC
:106480008170DEE71021A023D170013BFDD122698C
:10649000937803F0F7037746937055E723691B79E8
:1064A000C5E700BF609BFF1F0148FFF71FBD00BF8E
:1064B000388EFF1F0148FFF719BD00BFA48EFF1FD4
:1064C000704700BF38B5144C037801225B000546C5
:1064D000204684F83B3084F85E2084F85D20FFF786
:1064E0008BFC20460021FFF747FE0B4C2978012347
:1064F00020461A46FFF7CAFE0128F6D194F8383034
:1065000094F839209A4205D9E218013384F83830DA
:10651000107E38BDFF2038BD388EFF1F38B51B4CAC
:10652000037801225B000546204684F83B3084F85E
:106530005E2084F85D20FFF75FFC20460021FFF716
:106540001BFE124C2978204601230222FFF79EFEF3
:106550000228F6D194F8382094F839108A420FD2E4
:10656000531CDBB2A018994284F83830007E0AD957
:10657000234402321B7E84F8382040EA032038BDD1
:106580004FF6FF7038BD40F47F4038BD388EFF1F96
:106590000C2901D9002070470231490001F0FE01A9
:1065A000FFF7BCBF70B50C4C0378164601255B00A5
:1065B000204684F83B3084F85E5084F85D50FFF745
:1065C0001BFC31462046FFF717FC29462046BDE854
:1065D0007040FFF7D1BD00BF388EFF1FF8B50546EC
:1065E0000F461646412421463A462846FFF7DAFF71
:1065F000611C0234C9B232462846E4B2FFF7D2FF2A
:10660000592CF0D1F8BD00BF38B504460D463548C9
:10661000FFF706FC6322802120462570FFF7C2FFAA
:10662000012002F0CFFC204600225E21FFF7BAFFD6
:1066300020465D21FFF746FF242801D0002038BD09
:10664000204606220C21FFF7C9FF204601222B21FC
:10665000FFF7A8FF204601222C21FFF7A3FF2046C9
:106660000E222D21FFF79EFF204600222E21FFF74C
:1066700099FF204601222F21FFF794FF2046052293
:106680003021FFF78FFF204601223121FFF78AFFDB
:10669000204600223221FFF785FF204600223321C9
:1066A000FFF780FF204600223421FFF77BFF2046C2
:1066B00000223521FFF776FF204600225B21FFF7FD
:1066C00071FF204610225C21FFF76CFF204620223C
:1066D0005D21FFF767FF20468F225E21FFF762FFF3
:1066E000012038BD388EFF1F10B4047F4160022C9A
:1066F000C26002D010BC01F073BC836810BC1847A4
:1067000090E80C00F0B41C6859682568164F174EC5
:1067100029432160164D17491760D6601561116035
:10672000417A154A5C180A3194F8244053F82150F4
:1067300002EBC40149680D60017A5C1803EB81012A
:10674000247ECD6902EBC40149680D60817A581836
:1067500003EB810390F83000596B02EBC002F0BCF0
:1067600053681960704700BF01401F0001100038D6
:106770000110007800001F8084E2000038B5044654
:10678000104621700A491D4605F0B8F901464FF040
:106790007E5005F067FA074905F0B0F9E5606060E2
:1067A0002561656102F0ECFBE061204638BD00BF69
:1067B000DB0FC9400024744938B5044610462170E7
:1067C00009491D4605F09AF901464FF07E5005F043
:1067D00049FA064905F092F9E56060602561656156
:1067E00002F0CEFBE06138BDDB0FC94000247449E4
:1067F00038B503780446032B20D8DFE803F01A18D5
:106800001002C168406905F06FF80D4905466068DF
:1068100005F028FA0146284605F024FA38BD084953
:10682000406805F01FFAE16805F068F938BDC068F6
:1068300038BDC168406905F057F838BD002038BD43
:106840000024744970B504460E4602F099FB0546D3
:10685000E069281A05F0FEF8E3682361E5616661E6
:10686000A0610146606805F0FDF90146A06010488E
:1068700005F0F8F904F0CEFC04F06EF904F0E0FF46
:10688000054601464FF07E5005F02EF8616905F08F
:1068900035F921690646284605F030F901463046AB
:1068A00005F024F8E0602046BDE87040FFF7A0BF87
:1068B000000080BF704700BFF0B50C1EBDF814602B
:1068C00034DBB0F906701919B942C4BF3B1B1BB2C7
:1068D000002BA6461CDD002A1146B8BFD11D02F0D0
:1068E0000705CC10826A012007FB04E1A840012EB5
:1068F0000A44C0B21ED00CD3022E09D1013B12FAB9
:1069000083F3013A12F8011F41409A421170F9D104
:10691000F0BDC043013B12FA83F3C0B2013A12F852
:10692000011F014093421170F9D1F0BD23441BB205
:106930000024C6E7013B12FA83F3013A12F8011F63
:1069400001439A421170F9D1F0BD00BFF8B50D1E98
:106950000EDB14461F46064601F03AFBA84207DD4F
:10696000002C05DB304601F037FBA04201DCF8BD0E
:10697000F8BD304601F02AFB022853D003284BD043
:10698000012806D16540F3886C406540013B5D1BE2
:106990002DB2012F03D02AD3022F14D0F8BD002C22
:1069A0002246B6F90630B06AB8BFE21D42F3CF0204
:1069B00002FB035504F00704435D012101FA04F4CE
:1069C0001C434455F8BD002C2246B6F90630B06A87
:1069D000B8BFE21D42F3CF0202FB035504F00704E7
:1069E000435D012101FA04F45C404455F8BD002CDC
:1069F0002246B6F90630B06AB8BFE21D42F3CF02B4
:106A000002FB035504F00704435D012101FA04F47D
:106A100023EA04044455F8BD3389013B591B25463C
:106A20000CB2B6E7F18832890139013A4D1B141BCB
:106A30002DB224B2ADE700BF2DE9F041079E9DF9CC
:106A40001880089D04461F4600F0C0FF0D4B0E48FD
:106A50000E4984F83380FF22002F08BF1F4684F8B8
:106A60002F20002384F8302084F8312084F832204D
:106A70002060A665E565676261652362A3622046C2
:106A8000BDE8F081388EFF1FDCD70000011001380F
:106A900010B50446806A034B236008B105F07CFA08
:106AA000204610BDDCD70000F8B5436ADBB190F892
:106AB0002C200125AA4083F83B2083F85E5083F800
:106AC0005D500446406A03680E461B6800219847E3
:106AD000606A036831461B6898472946606ABDE8CA
:106AE000F840FFF749BBC26BC56C1368046A23EA20
:106AF000050313604CB122684FF00043D362516329
:106B0000D36A002BFCDA936BF8BD836B466B0825C8
:106B1000802410E03768426C3A4332601F68826C10
:106B20003A431A601A68876C013D22EA07024FEA6D
:106B300054041A6007D02142ECD13268476C22EA33
:106B400007023260EAE7F8BD70B50446406A0D46B8
:106B500000282BD0A16DFFF7ADF9002D20460CBF0A
:106B6000A621A721FFF7A0FF606A20B1E16DBDE873
:106B70007040FFF79FB9216C226D0868236A0243B9
:106B80000A6093B1DA7A82B1D00703D5224A9969B3
:106B90001160DA7A910703D5204AD9691160DA7A4F
:106BA000520702D51E4A1B6A136070BD236A002B70
:106BB0002BD0D97A626DE1B172B6D97ACE0706D5FB
:106BC0001848D9680668314099610160D97A880708
:106BD00006D51548196906683140D9610160D97A2E
:106BE0004E0705D5114859690668314019620160A0
:106BF00062B61B68D968914207D00D4818600D49EC
:106C0000DA6042F0804018611960226C216D1368CF
:106C100023EA01031360A0E700E100E004E100E0E3
:106C200008E100E080E100E084E100E088E100E0CC
:106C300001403F0000003F80436A2DE9F0410546D6
:106C40000E469046002B3ED090F82C100124A14017
:106C500083F83B1083F85E4083F85D40406A036828
:106C600000211B6808F1FF379847FFB2B8F1000F09
:106C700023D03744A046013E686A16F8011F036816
:106C80001B6898470134B742E4B216D0202CF3D1E8
:106C90000121686AFFF770FA95F82C206B6A5200A0
:106CA00083F83B2083F85E8083F85D80686A036820
:106CB00000211B6898470124DEE7686A0121BDE8CE
:106CC000F041FFF759BAC26BC16C136823EA0103A4
:106CD00006EB080413604FF00048A6420ED02B6A62
:106CE00016F801EB63B11A68C2F82C80C2F834E0E0
:106CF000D36A002BFCDAA642936BF0D1BDE8F08199
:106D0000AB6BD5F834C008208021DCF800206F6C14
:106D10001EEA010F14BF3A43BA43CCF800201A68A8
:106D2000AF6C3A431A601A68AF6C013822EA070266
:106D30004FEA51011A60E8D1CFE700BF70B50446B1
:106D4000406A0D46002828D0A16DFFF7B3F8204611
:106D50002946FFF7A9FE606A20B1E16DBDE87040E9
:106D6000FFF7A8B8216C226D0868236A02430A6005
:106D700093B1DA7A82B1D00703D5234A99691160B9
:106D8000DA7A910703D5214AD9691160DA7A520774
:106D900002D51F4A1B6A136070BD236A002B2BD0DB
:106DA000D97A626DE1B172B6D97ACE0706D51948A3
:106DB000D9680668314099610160D97A880706D59B
:106DC0001548196906683140D9610160D97A4E07C2
:106DD00005D512485969066831401962016062B6EA
:106DE0001B68D968914207D00D4818600D49DA60D8
:106DF00042F0804018611960226C216D136823EA0B
:106E000001031360A3E700BF00E100E004E100E03C
:106E100008E100E080E100E084E100E088E100E0DA
:106E200001403F0000003F802DE9F041044686B05C
:106E3000806A9DF830801E460F461546B4F908302A
:106E4000002800F04281DA1D48BF03F10E02B4F9B8
:106E50000630D21003FB02F2002105F05DFBB4F90D
:106E60000820202A00F39280B4F90610A34B0120D9
:106E7000203A733902EBD27201EBD1714FF0200E40
:106E8000029073208DE8014042F34F0241F34F011D
:106E9000204600F051FE606A84F82D70002800F052
:106EA0004D81002D40F08A80B4F90830202B14BFAA
:106EB0003D253C2584F82C50B8F1000F40F085802A
:106EC00006B394F93300002818DBC0B2012102F0A8
:106ED00051F8012194F8330002F038F8012002F053
:106EE00071F8002194F8330002F030F80A2002F023
:106EF00069F8012194F8330002F028F8606A00284C
:106F000000F08280A16DFEF7D5FF04227C49204667
:106F1000FFF792FE217A0139C9B22046FFF7C4FD7E
:106F2000784904222046FFF787FE94F92D30012B83
:106F300014BF142110212046FFF7B6FD0422724928
:106F40002046FFF779FEB4F90630802B00F09280DE
:106F5000602B00F0A680D9212046FFF7A5FD94F90B
:106F60002D30012B14BFF12122212046FFF79CFD7B
:106F7000204606226549FFF75FFE606A50B3E16D67
:106F8000FEF798FF012006B0BDE8F081B4F90610C5
:106F90005F4B0120403A52394FF0400E029002EB15
:106FA000D272522001EBD1718DE8014042F34F02C1
:106FB00041F34F01204600F0BFFD6CE76DB284F84D
:106FC0002C50B8F1000F3FF47BAFFEF729FF002EE5
:106FD00094D076E7216C226D0868236A02430A6028
:106FE00073B1DA7A62B1D00703D54A4A9969116060
:106FF000DA7A91077CD4520702D5474A1B6A13609C
:10700000012006B0BDE8F081236A002B2BD0D97A8D
:10701000626DE1B172B6D97ACF0706D53F48D9681B
:107020000568294099610160D97A8E0706D53C48E8
:10703000196905682940D9610160D97A4D0705D5DC
:1070400038485969056829401962016062B61B68B1
:10705000D968914207D0344818603449DA6042F068
:10706000804018611960226C216D136823EA0103C6
:1070700013604AE7B4F90830202B00F08680402BDB
:107080007FF469AF2A4920460322FFF7D5FD94F922
:107090002D30012B14BFCF219F212046FFF704FD87
:1070A00059E7B4F90830102B7FF455AF2149204639
:1070B0000322FFF7C1FD94F92D30012B14BFAF213E
:1070C00010212046FFF7F0FC45E7DA1D48BF03F129
:1070D0000E02B4F90630D21003FB02F210460592FC
:1070E00004F052FFA06200283FF44DAF059AB3E6CA
:1070F000114AD9691160DA7A7DE700BF34D80000FF
:1071000014DA000018DA00001CDA000020DA0000AF
:1071100028DA000000E100E008E100E080E100E0A2
:1071200084E100E088E100E001403F0000003F8092
:1071300030D80000E8DC000004E100E0012194F810
:107140003100244F01F016FF94F83200012101F0C4
:1071500011FF94F9312094F9323057F83220E2636C
:1071600057F83330206A23640125E56425651A68E1
:107170002A431A6078B1B8F1000F3FF428AFFFF747
:10718000BFFA002E3FF4BAAE9BE604221249204615
:10719000FFF752FDDFE6294694F82F0001F0EAFEE2
:1071A000294694F8300001F0E5FE94F92F2094F977
:1071B000303057F83220626357F833306564A56485
:1071C0001A68A36322F001021A60002E3FF496AE03
:1071D00077E600BF84E200002CD80000B0F9082058
:1071E000D31D48BF02F10E03B0F90620806ADB1000
:1071F00002FB03F2002105F08FB900BFF0B50029B2
:10720000BDF814502EDBB0F90660B1422ADA002A2C
:1072100059DBB0F9087014461C44BC42C4BFBB1A09
:107220001BB2002B1EDDD2B2D408D0F828E016FB2A
:10723000041112F00702DBB20EEB010421D0C2F1FF
:107240000807FAB2374F9342BF5C0CD2C3EB020C73
:10725000FF2646FA0CF6012D07EA06073FD005D3B4
:10726000022D36D0F0BD012D39D030D21EF801608C
:1072700026EA07070EF801709342F3D3B0F906101F
:107280000C449A1AD2B2072A10D9022D36D0002DFA
:1072900014BFFF26002613462670083BB0F90610DF
:1072A000DBB2072B0C44F7D802F00702002AD9D032
:1072B0001D4B012D9B5C1DD017D3022DD2D12278FE
:1072C00053402370F0BD13441BB20022A1E7022DEE
:1072D00025D11EF8016077400EF80170CCE71EF84A
:1072E000016037430EF80170C6E7227822EA0303F3
:1072F0002370F0BD227813432370F0BD114623782C
:10730000DB4323700839B0F90630C9B207291C44A1
:10731000F5D812F00702A5D0034B9B5CCFE73444AD
:10732000AFE700BFCCD70000BCD7000070B4C47D6D
:10733000BDF80C50022C18D0032C1FD0012C0BD000
:10734000002A03DBB0F90840944201DC70BC7047AE
:10735000039570BCFFF7B0BAC4880395013CA41A2A
:107360000A4621B270BCFFF749BF0689C488013EB6
:10737000641AB21AE41A12B221B2E1E70489039541
:10738000E41A641A114622B270BCFFF737BF00BF7F
:1073900070B4C57DBDF80C60022D1AD0032D12D03B
:1073A000012D03D0039670BCFFF728BFC488E41AF0
:1073B000A41A0A4621B2002A03DBB0F9084094421D
:1073C00013DC70BC70470489013C641A114622B278
:1073D000F1E7C48805890396013CAD1AED1A621ADB
:1073E00011B22AB270BCFFF709BF039670BCFFF759
:1073F00063BA00BF2DE9F8430446406A002863D011
:10740000A16DFEF757FD052274492046FFF714FCD5
:10741000A1790139C9B22046FFF746FBB4F908202B
:10742000E588A66AD31D48BF02F10E03DB10626A2D
:1074300015FB03F51FFA85F8002A7BD094F82C3051
:107440000125AB4082F83B3082F85E5082F85D50F7
:10745000606A036840211B6808F1FF379847BFB294
:10746000B8F1000F23D03744A846013E606A16F8F1
:10747000011F03681B6898470135B742EDB216D06B
:10748000202DF3D10121606AFEF776FE94F82C20BE
:10749000636A520083F83B2083F85E8083F85D8046
:1074A000606A036840211B6898470125DEE70121D7
:1074B000606AFEF761FE606A002800F08D80E16D71
:1074C000BDE8F843FEF7F6BC236A002B2BD0D97A2F
:1074D000626DE1B172B6D97ACE0706D54048D96857
:1074E0000568294099610160D97A8D0706D53D4824
:1074F000196905682940D9610160D97A480705D51D
:1075000039485969056829401962016062B61B68EB
:10751000D968914207D0354818603549DA6042F0A1
:10752000804018611960226C216D136823EA010301
:10753000136068E7E26BE36C1168276A0B4306EBA4
:10754000080913604FF0004E4E450DD016F801CBE0
:107550002FB33A68C2F82CE0C2F834C0D36A002BCB
:10756000FCDA4E45936BF1D1226C236D11680B430D
:10757000136097B1FB7A83B1D90703D51D4BBA6964
:107580001A60FB7A9A0703D51B4BFA691A60FB7ADB
:107590005B0702D5194B3A6A1A60BDE8F883A36B02
:1075A000D4F8348008208021D8F80020656C1CEACB
:1075B000010F14BF2A43AA43C8F800201A68A56C1B
:1075C0002A431A601A68A56C013822EA05024FEABC
:1075D00051011A60E8D1B7E7276AC5E7C4D70000B0
:1075E00080E100E084E100E088E100E001403F004C
:1075F00000003F8000E100E004E100E008E100E07D
:107600002DE9F04F85B09946BDF93870BDF83CA022
:10761000BB1AC1EB090B002BB8BF5B42BBF1000FDB
:10762000B8BFCBF1000B5B450D4616460093804674
:1076300048DC4D453A4633464CDC194613460A466B
:10764000C5EB09019B1A89B2002B0CB2B8BF5B4293
:1076500004EBD474BE42ACBF4FF0FF3201224D4563
:10766000039102924FEA640429DC9BB201930DE07E
:10767000D8F80070BF69B847019BE41AA3B21CB2E6
:107680000135002C2DB211DBA94518DB009B5B45B1
:107690002A46534631464046EADCD8F80020534695
:1076A0009769294632464046B847E5E7029A1644AC
:1076B000039AA94502EB030436B224B2E6DA05B018
:1076C000BDE8F08F4A462B46B94635464D4517462C
:1076D0001E46B2DD304629463E464D46074689469F
:1076E000AEE700BF10B404682469A44610BC60472C
:1076F00030B40468BDF808500295A46BA44630BCB1
:10770000604700BF30B40468BDF808500295E46BD0
:10771000A44630BC604700BF70B40468BDF90C607B
:10772000BDF8105003960495246CA44670BC6047C5
:10773000704700BF10B582B0B0F90C20019101680C
:10774000009200220C6CB0F90A301146A04702B03A
:1077500010BD00BF704700BF01F003010129C175D2
:1077600006D0032904D0C2880389428183817047EF
:107770000289C38842818381704700BF2DE9F041AF
:107780000568134E6F6986B0B7420446BDF8308075
:1077900010D1013B13441BB20093CDF804800B467B
:1077A000AD6A2046A8472368DB6AB3420AD106B017
:1077B000BDE8F081059304920391B84703A92568B9
:1077C0000EC9E6E7204606B0BDE8F041184700BF05
:1077D000317700002DE9F0410568124E6F6986B0DF
:1077E000B7420446BDF830800FD1013BCDF804808C
:1077F0000B4400921BB2AD6A2046A8472368DB6A9F
:10780000B3420AD106B0BDE8F0810593049203911A
:10781000B84703A925680EC9E7E7204606B0BDE8CA
:10782000F0411847317700002DE9F04F0568DFF887
:1078300058B06F6985B05F450646BDF93890BDF810
:107840003CA00C46904615D11F19BC420CDACDF86D
:1078500000A0214601342D6A4B464246304624B2F0
:10786000A847BC423568F2DBEB6A5B4507D105B03F
:10787000BDE8F08F0393B8473568039BE4E73046D3
:1078800005B0BDE8F04F1847317700002DE9F0430F
:1078900087B099420546BDF93840BDF83C6025D017
:1078A000A24212D00768DFF88080D7F81490C14553
:1078B00032D18DE850002846BC6AA0472B68DB6AAD
:1078C000434524D107B0BDE8F083994202DD084664
:1078D0001946034628680E96C46B01335B1A1BB227
:1078E0002846A44607B0BDE8F0436047A24202DD47
:1078F000134622461C4628680E96631C846B9B1A0E
:107900001BB22846A44607B0BDE8F04360472846AE
:1079100007B0BDE8F0431847059304920391C847A8
:1079200003A92F680EC9C4E7317700002DE9F04F95
:10793000D0F800E0DFF89090DEF814B083B0CB45CB
:107940000446BDF93080BDF834A00D4617461E46EA
:1079500031D1CDF800A0DEF824B0294633463A46AE
:107960002046D8472368CDF800A008F1FF323A44FA
:10797000D3F824B0294612B233462046D8472368AC
:10798000CDF800A02946D3F820B03A464346204619
:10799000D8472068CDF800A0711E29444346056AE7
:1079A00009B23A462046A8472368DB6A4B4506D110
:1079B00003B0BDE8F08FD847D4F800E0C9E720460F
:1079C00003B0BDE8F04F184731770000F0B4002451
:1079D00001264FF6FF75094F07600471C475C48115
:1079E00004824476C4618675067685824582C180AC
:1079F000028141818281F0BC704700BFF4DC00004D
:107A00002DE9F04F85B00668BDF84450BDF93880C7
:107A1000CDF8008004460195D6F848B00392BDF930
:107A20003C60BDF9407089469A46D8472368019565
:107A3000009742465146D3F8488020463346C04717
:107A40002068039B0E930F95856C4B463A46314652
:107A50002046AC4605B0BDE8F04F60472DE9F04F39
:107A600087B01746BDF9404000912546E91D0593B2
:107A700044BF2B4603F10E010268BDF8486053690C
:107A80000294C91003912B49BDF9444001968B42E1
:107A9000824645D1002C3CDD029B3C445E1EB6B2C2
:107AA0004FF0000923B2049301364D46029B002B90
:107AB00028DD059B002403EB090806E0EDB22B0648
:107AC00004F1010411D4A6421CD0A1B211F0070F99
:107AD00023B24FEA4505F1D1002BB8BF0733DB10C5
:107AE000013418F803502B06EDD5009BD2F818B0DE
:107AF00019443A4609B2019B5046D847A642DAF8E3
:107B00000020E2D1039B01379944049B3FB2BB4262
:107B1000CCD1D36A074A934206D107B0BDE8F08FB3
:107B20009847DAF80020B5E7504607B0BDE8F04FB7
:107B3000184700BF3177000070B4BDF90C60BDF983
:107B40001050BDF8144003960495059470BCFFF7DF
:107B500085BF00BF2DE9F04F93B090460591C169F4
:107B60001090BDF870000790BDF874909DF878A053
:107B70000493002900F0CD800A7A0AC98946049945
:107B80008A1AD2B203EBC203BAF1010FDA780B9270
:107B900093F905201E8893F802B00F9293F90640DE
:107BA00079D913B2099323B20C93109B1A68A94B8D
:107BB0001193194653698B4240F0A6800B9B002B12
:107BC00055D01FFA88F300210D93C8462344DDF8F1
:107BD000409006910E930F460C46BBF1000F3FD02C
:107BE000BDF818100C9B03971FFA8AF0CB1813FBF3
:107BF00000F304900E9801440D98034409B21BB29F
:107C00000A910893002505E00135EBB264009B451D
:107C1000E4B222D9039B2B44590703D1731C18F8F3
:107C200006409EB22306EFD5099BBDF81000E91867
:107C300011FB00F10598BAF1010F0FFA8AF3014424
:107C40001CD0079801900093D26909B217464846A4
:107C5000089AB847D9F80020D6E7039F5F44FFB2DF
:107C6000069B0B9901330693DBB29942B5D8D36AD0
:107C7000119A934243D113B0BDE8F08F0F9B1918AE
:107C800093690A9A29441F4609B2079B4846B84798
:107C9000D9F80020B8E700230C93099385E70A9AE6
:107CA0000D9B0132013B52B213F0FF030A920D9378
:107CB0006FD1DDF81890079BDDF83C80DDF820A03F
:107CC0004B4517D0BAF1010F00F0C8800B9A109DF8
:107CD000CDF804900BEB8B014FEACB030A440093E1
:107CE0001146DEF81C405346424609B22846A047DA
:107CF000D5F800E0DEF82C30119A9342BBD01098F2
:107D000013B0BDE8F04F1847109D284698472A68E1
:107D100054E7109A0598B2F90A308342ABDDB2F904
:107D20000C304345A7DD062313FB0A03002BA2DD1D
:107D300008EBCA03002B9EDD537E2BB9049BAF2BAF
:107D400002D90133DBB20493109BD3F800E0414B1E
:107D500011931A46DEF81430934240F08E801FFAD9
:107D600088F30E9308339BB2BDF8142005930523C6
:107D70000D9300230A93CDF83C800FFA8AF3DDF8C7
:107D80004080CDF818900B921FFA8AFBCDF820A006
:107D900099460A9ABDF810000B9C0E9D05231946C2
:107DA00011FB00232C481146C75C039702FB0B42D2
:107DB00014FA81F312B21BB209920C932C462E4690
:107DC0001CE0089B0999012B2AB24B4640462DD056
:107DD000079F0197CDF80090DEF81CA0D047D8F897
:107DE00000E0039B5B0801340393059BA4B25D4450
:107DF0005E44A342ADB2B6B23FF451AF039BD80785
:107E0000DFD4079B069A9342EBD0089B012B16D038
:107E1000069B0193CDF80090DEF81CA009994B4613
:107E200032B24046D047D8F800E0DAE7DEF818A0D2
:107E3000079B0C9922B2D047D8F800E0D1E7DEF8D2
:107E400018A00C991346404622B2D047D8F800E05B
:107E5000C7E700BF3177000044DD00000B99109D9B
:107E6000CDF800900531DEF8204009B242460823E3
:107E70002846A047D5F800E03CE7109C20469847EC
:107E8000D4F800E06BE700BFF0B5C36985B00446E5
:107E90002BB30A2968D00D294AD01A7A914247D3C8
:107EA000587A884244D35D688A1A05EBC205AA78DD
:107EB000002A50D0E87800284DD0207E00283AD003
:107EC00095F905E0B4F90E00A67DB4F90A70724484
:107ED00006FB0202BA4262DCB4F9102030E00A2943
:107EE00056D00D2924D0027E002A4BD0B0F90E00C6
:107EF000A57DB4F90A60062212FB0502B2423EDDFE
:107F0000228AE38102EBC50212B218462282A78AB6
:107F1000668A02950B468DE8C00001462046FFF7B1
:107F200019FEA37DE28903EB430302EB4303E381E4
:107F3000012005B0F0BDA67DB4F90E00B4F9102003
:107F4000B4F814E0678A02960B468DE8804001463B
:107F50002046FFF7FFFD2979E389A27D012001FB7F
:107F60000233E38105B0F0BD0022C2819A7A817D9F
:107F7000038A01FB02330382012005B0F0BDB4F98E
:107F80001020C4E7857DB4F91020B0F90E00BEE7DB
:107F9000028A817DC38102EBC1030382C8E700200E
:107FA000E0819B7A228A03FB062212B22282C7E773
:107FB000C1810282704700BF002908BF012181757D
:107FC000704700BF81824182704700BFC07D70470B
:107FD000B0F90A00704700BFB0F90C00704700BF4D
:107FE00010B4EFF3108272B6437F33B9017F0129D9
:107FF00007D003290FD00123437702B962B610BC22
:108000007047124C2168A1B1114943610B6883612B
:1080100008605861EFE70F4C216881B10E49436158
:108020000B688361086058610C4B4FF080511960F8
:10803000E1E7074B4161816120601860DBE7064B97
:108040004161816120601860EEE700BF4C9BFF1F1B
:10805000489BFF1F3C9BFF1F409BFF1F04ED00E060
:1080600070B5EFF3108272B60C4C206880B10C4EE4
:1080700000254369236073B19D6102B962B64577FB
:1080800083689847EFF3108272B620680028F0D119
:1080900002B962B670BD3360EFE700BF3C9BFF1FC3
:1080A000409BFF1FFFF7DCBF184A30B41468002C58
:1080B00027D0036821688B420ED2CB1A002184603E
:1080C000C1602360E06010600223037530BC70471C
:1080D00011688B42144608D3A2685B1A0360002A19
:1080E000F6D18260C460A060EEE7D268C2608460AE
:1080F000E060C568CB1A0222A8602360027530BC1C
:1081000070478460C4601060DEE700BF449BFF1FBF
:10811000F8B5224E34682CB32368002B3AD1204F97
:108120001D4604E03468ECB12368002B32D1A3680B
:1081300003B1DD6020693360036825751B68BB42AD
:1081400021D1037F4560022BC46020D0FFF748FF98
:108150006368002BE6D023602046FFF7A5FF346854
:10816000002CE1D1EFF3108372B60E4A00211068A3
:10817000116003B962B628B18468FFF795FF204605
:108180000028F9D1F8BD224600219847E0E783682E
:108190009847DDE7013B2360E4E700BF449BFF1FF6
:1081A000E9660000549BFF1F024A13680133136005
:1081B000FFF7AEBF609BFF1FF8B50E4671B17AB1F5
:1081C0000746144600253B6816F8011B1B68384615
:1081D0009847013C0544F6D12846F8BD0846F8BD4D
:1081E0001046F8BD00B5064A036812885B6883B084
:1081F00001A9ADF804200222984703B05DF804FB02
:1082000044E20000F0B507468BB0002A33D0012AC3
:1082100008BF0A2251B3212400E0F4B2B1FBF2F509
:1082200002FB1511C8B2092900F1300198BFC8B28C
:108230000AA988BF3730214488BFC0B201F8240C96
:10824000661E2946002DE8D133B1013CE4B20AABE9
:1082500023442D2203F8242C3B6801AA11195B68E2
:108260003846C4F1220298470BB0F0BD30228DF899
:1082700025202124E8E70368C9B21B6898470BB0A2
:10828000F0BD00BF0029BABF49422D2300230A22B6
:10829000FFF7B8BF374A384913681B06FCD40B6890
:1082A00013F08003F8D172B634490A78002A5FD0FF
:1082B000334A3448F0B4344C176806682568D468EB
:1082C0000C303E44143200681268304F35442C4460
:1082D00020440244C2F34E022D4E2E482E4D2F4C08
:1082E00042F400423A60376806682D682C4A2468D8
:1082F0000C303E44006812682A4F35442C44204418
:108300000244C2F34E02284E2848294D294C42F41B
:1083100000423A60376806682D68274A24680C30A6
:108320003E4400681268254F35442C4420440244E2
:10833000C2F34E02224E2348234D244C42F4004205
:108340003A60376806682D68214A24680C303E443C
:108350000068126835442C4420440244C2F34E02A3
:108360001C4842F4004202600B7062B6F0BC7047D9
:1083700062B6704724B0034024B00B40599BFF1FE6
:1083800038B003403CB0034040B003402CB0034041
:1083900058B003405CB0034060B0034064B0034099
:1083A0006CB0034030B0034038B00B403CB00B40E1
:1083B00040B00B4044B00B404CB00B402CB00B40D5
:1083C00058B00B405CB00B4060B00B4064B00B4049
:1083D0006CB00B4030B00B4030B42948294A2A4BCE
:1083E0002A4D6024E121047011701B78284C082B61
:1083F00030D00A2B2748284937D00C2B0CBF352208
:108400003D2212232A60236002600B60234B244923
:108410001B78244ABBB101230B601360224B234914
:108420001B78234A012B26D9042B0FD9082B1ED9E0
:10843000102B94BF862387230B6013601D4B0122F2
:108440001A7030BC70470B601360E7E784230B6041
:108450001360F3E700F58E200F4908300122132343
:108460002A60236002600B60D0E73922F7E785239A
:108470000B601360E2E780230B601360DEE700BF50
:108480000040074001400740108FFF1F08B0034025
:108490000CB0034008B00B400CB00B405C9BFF1FBE
:1084A00020B0034020B00B40118FFF1F24B00340C9
:1084B00024B00B40599BFF1F0C2830B417D9102350
:1084C000984228BF18461C46104A114D1178181AB8
:1084D0008C42287018D00F4913700B7823B10E49C5
:1084E0000E4A00230B60136030BCFFF775BF0A28EB
:1084F00002D90C231C46E7E7082802D90A231C46A8
:10850000E2E708231C46DFE730BC7047108FFF1FEF
:10851000589BFF1F599BFF1F24B0034024B00B4002
:1085200028282FD8334B2DE9F0411E5CFF2E2BD08D
:10853000314B1B78002B2AD132062CD472B62F4D2A
:108540002F4C2F46012326602B7062B672B623682B
:108550001B060CD43B781BB9F4E72B78002BF1D029
:1085600062B602F035F972B623681806F5D5254BC8
:108570001B6800222A7062B6234A107843FA00F082
:10858000BDE8F081002070470020BDE8F081FFF7D2
:1085900081FE3206D2D572B61C4DDFF87C801C4CB1
:1085A00006F04007FFB206F03F06D8F80030DFB112
:1085B00023F01003C8F8003001232660134A2B7003
:1085C00062B672B6236819060CD413781BB9ECE7AF
:1085D0002B78002BE9D062B602F0FAF872B6236865
:1085E0001B06F5D50B4BC3E743F01003C8F800306A
:1085F000E2E700BF48E20000599BFF1F5B9BFF1FA3
:1086000000B0034010B00340589BFF1F5A9BFF1F50
:1086100000B00B4010B00B400CB00B400A4A0B49A5
:10862000136843F4805313600B7843B9084BC0229E
:108630001A70084B80F30C0000B218807047044B8E
:1086400080221A70F5E700BF2C8004405C9BFF1F5E
:1086500021C00C4000C00C40F0B51B4B1B4E5968AC
:1086600018689A68DB6885B06C460FC43378990740
:108670001DD5174A174C1378174913F0700318BF0C
:108680001370164A164B80271770002633200322DA
:1086900026706D4608701A7072B6043C45F00105EC
:1086A0002046A84762B6237813F0700309D10D4B1A
:1086B000064901E0013B02D00A78D207FAD505B09D
:1086C000F0BD237005B0F0BD74E20000010002406F
:1086D00000000240040002400B000240070002407C
:1086E0000A000240410D0300B0F5006F0AD210B538
:1086F000094B1B78DB07044606D504F1A05000782F
:10870000C0B210BD00207047FFF7A6FF04F1A050D3
:108710000078C0B210BD00BF01000240B0F5006F8C
:1087200017D238B50F4B1B78DA070D46044611D522
:1087300004F1A0500378AB420AD00B4A137813F02F
:10874000700318BF1370074A05701378DB07FCD558
:1087500038BD7047FFF780FF04F1A0500378AB42AB
:10876000EBD1F5E7010002400000024008B5F7F741
:10877000B7FEF9F721FB02F02BF8FAE7844641EA4D
:10878000000313F003036DD1403A41D351F8043B89
:1087900040F8043B51F8043B40F8043B51F8043BDB
:1087A00040F8043B51F8043B40F8043B51F8043BCB
:1087B00040F8043B51F8043B40F8043B51F8043BBB
:1087C00040F8043B51F8043B40F8043B51F8043BAB
:1087D00040F8043B51F8043B40F8043B51F8043B9B
:1087E00040F8043B51F8043B40F8043B51F8043B8B
:1087F00040F8043B51F8043B40F8043B51F8043B7B
:1088000040F8043B51F8043B40F8043B403ABDD2E9
:10881000303211D351F8043B40F8043B51F8043B8B
:1088200040F8043B51F8043B40F8043B51F8043B4A
:1088300040F8043B103AEDD20C3205D351F8043B1A
:1088400040F8043B043AF9D2043208D0D2071CBFE6
:1088500011F8013B00F8013B01D30B88038060460F
:10886000704700BF082A13D38B078DD010F0030385
:108870008AD0C3F10403D21ADB071CBF11F8013BF5
:1088800000F8013B80D331F8023B20F8023B7BE744
:10889000043AD9D3013A11F8013B00F8013BF9D26F
:1088A0000B7803704B7843708B7883706046704709
:1088B00008B5104C08E0236859050DD423681A0543
:1088C0000FD42368DB0411D423685803F3D500F0D8
:1088D0008DFE23685905F1D501F0DEFF23681A05E6
:1088E000EFD502F06FF82368DB04EDD500F0F0FC63
:1088F000EAE700BF3480044008B5FFF7D9FF00BFA6
:10890000014B10221A80704700200540704700BFBD
:10891000094908B50B6830B16A461844A2F580527F
:10892000904202D20860184608BD03F0FFFA0C23FB
:1089300003604FF0FF3008BD148FFF1FFEE700BF3C
:10894000EFF3138070B9EFF310836BB9EFF3058287
:108950005AB94FF48070EFF311832BB1984228BFBE
:10896000184670474FF0FF3070470F2A01D818465D
:10897000F1E7014BD05CEEE7F0E300E0F0B44D1E10
:108980002E46002400E00134B0FBF2F302FB13009A
:10899000092800F130078ABF3730F8B2C0B206F8B4
:1089A000010F1846002BEED10A1953704CB1107804
:1089B00015F8016F28700133E01A834202F801694B
:1089C000F5DB0846F0BC7047704700BF10B40F4B92
:1089D00053F8302092F880422CB1012369B182F81B
:1089E000803010BC704703EBC0035B681A6841B964
:1089F00022F002021A6010BC704782F8003110BCED
:108A0000704742F003021A6010BC704784E2000015
:108A10001C4A02EBC00301295B6811D004291BD05A
:108A200052F83000002280F8802229B1022920D09B
:108A3000032922D01A6070474FF480721A60704781
:108A400052F830004FF4A27280F880121A601A684F
:108A500022F020021A60704752F830104FF4A272D0
:108A6000012081F880021A601A6842F020021A6020
:108A7000704740F203121A6070474FF481721A6017
:108A8000704700BF84E20000212848D8F8B5042AC6
:108A900044D8DFE802F0484B4E0345004FF410265F
:108AA0002B4B03EBC0030D465C68216811F4E061B9
:108AB00048D0284B284A2949C3F89C2104F1404258
:108AC0002748C3F8A411A2F59221264FC3F8A001AC
:108AD0007C292548C3F8A871C3F8AC012CD9A2F5AC
:108AE00094237C2B2AD9A2F596237C2B28D9A2F596
:108AF00098237C2B29D9A2F59A227C2A27D81B48B7
:108B000072B6236823F4702343F08072C4F38401A7
:108B10001643236040F82150266062B6F8BD7047C6
:108B20004FF43026BCE74FF40026B9E74FF4402657
:108B3000B6E74FF42026B3E70D48E1E70D48DFE73D
:108B40000D48DDE7FFF764FFB3E70C48D8E7F8BD51
:108B500084E200000082FF1FF188FF1F9988FF1F39
:108B6000C588FF1F6D88FF1F4188FF1FF08FFF1F03
:108B7000188FFF1F508FFF1FA08FFF1FD08FFF1F69
:108B80001A4B03EBC00010B4426802F14043A3F556
:108B900092217C2923D9A3F594217C290DD9A3F511
:108BA00096217C291FD9A3F598217C2919D9A3F5F1
:108BB0009A237C2B11D80E4C00E00E4C72B6136831
:108BC0000D4823F08773C2F3840123F4803343F00C
:108BD0008073136044F8210062B610BC7047074CE4
:108BE000ECE7074CEAE7074CE8E700BF84E2000047
:108BF000F08FFF1F508FFF1FC9890000188FFF1FC4
:108C0000D08FFF1FA08FFF1F30B4054B054D064CC2
:108C1000002210211A602A602060196030BC704761
:108C200014D0034004D0034000D00340282838B5B6
:108C30002ED0002904464FDD5F4B1B78012505FA35
:108C400003F28A4202D8212837D938BD0338C2B28C
:108C5000012A3AD9202C4AD0192C48D0574A1268F8
:108C600002FB011222FA03F31D2800F29B80DFE8C9
:108C700000F0928B847D9999766F99999999999939
:108C800099999968615A53994C99999999999945E3
:108C9000494B1B780B2B08D90C2B1CBF0C3B1941E3
:108CA0000846BDE83840FFF7B9BCC3F10C03994052
:108CB0000846BDE83840FFF7B1BC2946FFF786FEFD
:108CC0002946BDE83840FFF7A3BE3D4A126802FBC3
:108CD000011222FA03F3C7E72128B6D80021FFF7D3
:108CE00075FE20460121BDE83840FFF791BE354AA8
:108CF000126802FB011222FA03F3B5E73249334A44
:108D00000B604FF45173136038BD3149314A0B6029
:108D10004FF45173136038BD2F49304A0B6040F255
:108D20004443136038BD2E492E4A0B6040F2444341
:108D3000136038BD2C492D4A0B6040F24443136048
:108D400038BD2B492B4A0B6040F24443136038BDB9
:108D500029492A4A0B6040F24443136038BD284930
:108D6000284A0B6040F24443136038BD2649274A25
:108D70000B6040F24443136038BD2549254A0B601F
:108D800040F24443136038BD2349244A0B604FF43A
:108D90005173136038BD2249224A0B604FF451735E
:108DA000136038BD212C3FF650AF7F29D4BF00217E
:108DB0000121204693E700BFF88FFF1F0880034082
:108DC0000890034008800B4010800B4048A00440EE
:108DD00018800B404CA004401880034008B00440A9
:108DE0001080034004B004404080034018C0044099
:108DF0003880034014C004402880034010B0044071
:108E0000208003400CB004403080034010C0044078
:108E1000488003401CC00440189003403490044034
:108E2000109003403090044038B1102828BF102023
:108E3000044AC3B2107813707047024A01231078B5
:108E400013707047F88FFF1F2DE9F8430E468046D8
:108E50003249334D304602F0EFFF47F61223002827
:108E60001ABF1D464FF002094FF00109002425FAF0
:108E700004F002F0EBFD4FF05E51074602F03EFEBB
:108E80000146304602F0ECFF30B90134072CEED138
:108E9000E80902F0DBFD07463146384602F0E2FE03
:108EA0004FF07C5102F020FD03F014F84FF6FF72F2
:108EB0009042A8F1030328BF1046012B29D9B8F12D
:108EC000170F17D8174B23FA08F303F0010383F0A9
:108ED000010223B9B8F1190F0FD0BDE8F883124B86
:108EE000124D13491A6044EAC9042A6008601C60E4
:108EF000BDE8F883B8F1200FECD10E4B0E4D0F49B1
:108F0000002244EAC9041A602A6008601C60BDE8B7
:108F1000F8830B4B0B4D0C49F2E700BF001BB74029
:108F2000006CDC026006F000008003400480034017
:108F30000880034000800B4004800B4008800B40F9
:108F4000009003400490034008900340212801D87A
:108F5000FFF73CBD704700BF212806D8044B53F8EB
:108F6000303093F80002C0B270470020704700BF55
:108F700084E20000212801D8FFF74ABD704700BFF6
:108F800072B60C490C4B0D4A1B680868126862B631
:108F9000520102D5322B88BF01300949C3F5BB33DA
:108FA0004FF47A72FF33A1FB031302FB00F000EBD6
:108FB00093107047609BFF1F18E000E004ED00E095
:108FC000ABAAAAAA2DE9F843054672B6204F214B59
:108FD000214A1B683C68126862B6520102D5322BE6
:108FE00088BF013495B3C3F5BB331C4EDFF86490E2
:108FF000DFF86480FF334FF47A72A6FB031302FBA1
:1090000004F404EB931472B6D9F800103A68D8F857
:1090100000E062B6C1F5BB33FF33A6FB03031EF0CD
:10902000806FC4EB93134FF47A7002D0322988BF5B
:10903000013200FB0233B3F57A7F04D3013D05D042
:1090400004F57A74DFE701F0C3FBDCE7BDE8F883E1
:10905000609BFF1F18E000E004ED00E0ABAAAAAAA5
:10906000F8B52D4B2D49DFF8D0E0DFF8D0C02C4EFD
:109070002C4D2D4C2D4A2E4F4FF4000018604FF010
:10908000807018604FF0007018604FF080601860BA
:109090004FF0006018600020086028234BF6FF7135
:1090A000CCF80010CEF80030336013602B602360E2
:1090B0003B60B3629362092245F8242CC4F8D80FB0
:1090C00005F57F65C7F8D41F07F5FF2707F5FA6791
:1090D000C6F8F83F2B6006F5FF26C4F8D42F05F537
:1090E000FD2504F5FF24386006F2F476114831605E
:1090F00005F5FF6504F5FD642B6023600260FFF752
:109100006BF91920FFF75EFF00F0B6FF40F2131075
:10911000BDE8F840FFF756BF08E100E004800340D7
:1091200014800340248003402C8003401C800340B3
:109130003480034000800B400C80034008800340D3
:109140002DE9F84F214B1B6807460BB101221A701D
:10915000DFF888901E4D99F80040DFF884801D4E9E
:109160000134272C8ABF4FF0000A5FFA84FA544674
:10917000AB462B78A34216D1FFF7E2FB40281FDC59
:1091800033791B06F5D59BF800300133272B86BFBA
:1091900000221346DAB218F80330DBB2F3712A70FA
:1091A0002B78A342E8D00C490A4BFFB208F80470B0
:1091B0000120AC22087089F800A0DA70BDE8F88FB1
:1091C000FF28D6DD01F004FBD3E700BFD89BFF1FCB
:1091D000D59BFF1F00C00640D49BFF1FDC9BFF1FD9
:1091E0006C9BFF1F1C4BDFF894C01A681B49F0B53D
:1091F00042F480521A4D1A60DFF884E0194F1A4E7B
:109200001A4C00238CF800304FF451722B701F2839
:1092100040F213358EF800303B70337025600A60E1
:1092200012D819460124124A124D11701248547076
:1092300000212C27402693724FF400349170117452
:10924000D7702E700460F0BDC0F34431C0F34714F2
:1092500000F01F03E7E700BF348004400CC0044067
:10926000699BFF1FD59BFF1FD49BFF1F08C00440B5
:1092700000C0064031E400E004E100E0689BFF1F0D
:10928000DC9BFF1F034B1B68DB0401D5FFF758BFB6
:10929000704700BF3480044010B5044C237823B1DC
:1092A00001F096FA2378002BFAD110BDD49BFF1F52
:1092B000054A064B10781B78C0B2DBB2984238BF23
:1092C0004030C01A704700BF689BFF1F699BFF1F9B
:1092D00030B42B4B1A7994061FD52A48DA790378D3
:1092E000294901333F2B0978C8BF00238B42D2B2F2
:1092F00003D0264CD9B2E2540170254A116861B1FD
:10930000244A1278D2B2934236BFC2F140029B1A6D
:109310009B18272BC4BF01230B70194AD378DBB2EB
:10932000180611D45A060DD5154B1B795B0609D5C5
:10933000194B1A491B6800220A7003B11A70104BAE
:109340002C22DA7030BC704711790906EAD514492D
:1093500010480C780178C9B28C420DD04A1C272ADB
:1093600084BF00210A460F4D054C98BFD1B2AA5CBC
:10937000D2B2E2710170D5E76C21D170D2E700BFA3
:1093800000C00640689BFF1F699BFF1F949BFF1F47
:10939000649BFF1FD59BFF1FD89BFF1FD49BFF1F04
:1093A000DC9BFF1F6C9BFF1F21282FD8184B195CDB
:1093B000FF292BD0174B184ADFF870C003EBC00011
:1093C000F0B54368DFF868E0144F154D154E0024E2
:1093D0001C60DEF80030012043F020038840CEF806
:1093E000003014604FF4A07338602E60C2F800C0E3
:1093F000013BFDD113689B05FCD42023013BFDD12B
:10940000094B09B233F8110080B2F0BD002070475B
:1094100094E3000084E2000000500440085004403F
:1094200004500440000002030051044080014A003F
:1094300038800440431E032B14D872B60A4951F8F1
:10944000230068B170B4094C058834F813204668CD
:1094500041F82360521B24F8132062B670BC704799
:1094600062B6704700207047389CFF1F7C9EFF1F2C
:10947000013803280BD872B6074B53F8203043B19C
:1094800000205B680130002BFBD162B670470020E2
:1094900070471846F9E700BF8C9CFF1F30B472B6C6
:1094A0002B4A13781D0706D52A4B196A002936D096
:1094B000996A002941D053781C0706D5254B196CB1
:1094C00000293ED0996C002939D09378190705D529
:1094D000204B196E002936D0996E89B1D3781B07BD
:1094E00007D51C4BD3F880207AB3D3F888201121FC
:1094F0003AB162B6184B00221A7030BC00F04ABE76
:109500000D21154C154D227843F8315003EBC10362
:109510000830013A5860227062B630BC70470422AD
:109520000D4C0F4D217843F8325003EBC203083045
:109530004A1E5860227062B6EFE70521E1E7092173
:10954000DFE70822ECE70C22EAE71022E8E700BF99
:10955000B8E300000080FF1FB59CFF1FC80040005B
:1095600088004000431E032B1DD81B4A400140F0D9
:10957000100030B4104472B6184CE25C032A1BD8B9
:10958000DFE802F00212151703220D88E25410F0F2
:10959000080F14BFC823882343EA0543083103603A
:1095A000416062B630BC704708300222EDE7052208
:1095B000EBE708300422E8E7094A52F8230038B103
:1095C000084A52F82300416042F8231062B6E9E7E6
:1095D00042F82310034AF7E70080FF1FC49CFF1FD7
:1095E0008C9CFF1F9C9CFF1F00BE70472DE9F04F15
:1095F000DFF818B3DFF818A387B044E0AD4F4FEAA7
:10960000930807EBC809013ED9F8042003F00803CA
:10961000F6B2A2F1080003F0FF04002B40F0018134
:1096200057F838301B0C99B222F8081C002B00F0B8
:10963000EF80A14B22F8064C42F8044C53F8262048
:10964000002A00F0CF819D4D55F8263058609C4C83
:1096500045F8260034F81630194424F8161000F0A6
:1096600079FD002800F0C281964A974B19F0080F47
:1096700000F1080018BF1346C9F8040047F8383055
:1096800008238BF800309BF80040E4B265071CD536
:109690008E4B1B78B3B18E490A7802F0FF0322B1DA
:1096A000013BDBB20B7003B900BE8A490A7802F0B5
:1096B000FF032AB1013BDBB20B70002B00F0688185
:1096C00000F000FE04238BF8003004F0080303F0E0
:1096D000FF02002B00F0C9809AF80030DBB21E09AF
:1096E0008CD19A08DFF8CC9159F8321009EBC200FE
:1096F000C1F38301013940680C2900F28580DFE85D
:1097000001F07A7A8383838383834683838307008C
:109710000168714D4068714F714E6860296088B270
:1097200040F281610024674B49F832304FF0010E5E
:1097300088423C60C9F81040C9F8184086F800E03B
:109740005C4A00F2E780B0F5D06F80F01B82B0F584
:10975000817F00F0D98100F26981802800F02A829F
:10976000822840F0D781A98801F07F01042900F206
:10977000D1815C485C4A89000844147054700178B7
:109780008C0740F1608382F800E0022173E1534FBF
:109790003A682AB3554B524E5548198834780578A3
:1097A00040298E4645F0020828BF4FF0400E002C9D
:1097B00084F001043470CEEB01010CBF8824C8246E
:1097C00009EBC80689B285F0010544EA0E447260CF
:1097D000198049F8384072440570002965D03A6014
:1097E0003D4B1A88B2F5A06F0ED100219A785970BE
:1097F000404B1A7008E038493F4C0D68A54200F014
:109800009880304949F832103C4A0123137037E7F9
:109810002C4A2D4B19F0080F18BF134647F8383063
:109820002EE700F0B7FC364A364952F82630002BB6
:1098300000F0E38058688C5D42F8260003F10802CE
:10984000C9F80420032C05D8DFE804F02C022926EF
:1098500002228A551A8819F0080F0CBF8823C823E2
:1098600043EA024347F838300AE7E00700F1938003
:10987000210600F1D180A20706D5234A2349137897
:109880000220DBB213700870E30602D51F4B1022D2
:109890001A7007B0BDE8F08F04228A55DAE7052276
:1098A0008A55D7E703228A55D4E7BEF1400F18BF87
:1098B000002294E70080FF1F389CFF1FE49BFF1FDE
:1098C0007C9EFF1FC800400088004000C09CFF1F16
:1098D000499CFF1F349DFF1FAC9CFF1FE09BFF1F97
:1098E000489CFF1FC0200740B89CFF1FF49BFF1F30
:1098F000B49CFF1F982007402109000394200740D3
:109900008C9CFF1FC49CFF1F8820074080200740BD
:1099100090200740B0F5106F00F07C8140F2A380EA
:1099200040F62112904240F07B82A54A0123137039
:109930006AE74C68A3498C427FF463AF0178A92998
:109940007FF45FAF417845297FF45BAF8178C2290E
:109950007FF457AFC1786B297FF453AF9A489B4E81
:109960000178347881F00105002C41F00201057086
:109970000CBF8820C82084F0010449F8310009EBAD
:10998000C10193483470002505244D60047038E708
:1099900000F0FEFE94E68F4B89488B491A614FF028
:1099A000020E80F800E08C4F0A708C4919609960B3
:1099B0008B4E8C4D8C4C9A610D213970FF2131708A
:1099C000DFF84CE229702270884D894A8EF8001029
:1099D0009F27012406F8047C5D600470DA6007B0FC
:1099E000BDE8F08F43F82600824D30E6824A47F802
:1099F000380013780133137042E68B5D032B00F2BD
:109A0000BA8001A252F823F08196000081960000EE
:109A1000619A00005B9A00006F49724B80220D2012
:109A200008701A70A2077FF52FAF26E740F20232C6
:109A3000904240F0ED81AA8802F07F02042A69D8A2
:109A40006D88002D66D16449CDF804E09200114480
:109A50000A7842F002020A70C1E101238B550FE639
:109A600000238B550CE6B0F5086F53D16349644A67
:109A7000097811707146ED888D4280F0E882524875
:109A80000478402DAE4644F0020C28BF4FF0400E43
:109A900002EB0E0309EBCC01029301234A604FEA6B
:109AA0000E48CEEB050101930025C82242EA0803C7
:109AB00084F0010249F83C3035700270DFF814C1BF
:109AC000424BDFF8048149BBBEF1400F7FF42DAF5C
:109AD00042F0020C09EBCC03029ADFF8F8E05A607E
:109AE0008DBB0D0445F088059DF804304EF83C50C0
:109AF0000A4433700470134640297FF416AF0021E6
:109B0000404A3B60118010E7AA8802F07F02042AD5
:109B100040F28B81304A0F23137006E74029D7D9D2
:109B200042F002020CEBC200029E4660BDB19DF8FD
:109B3000045035481D703346403988F800404033A2
:109B40004CF83200DCE79DF8043033700D04029BC2
:109B5000047045F0C8050B444EF83C50CCE79DF826
:109B600004501D70029B1D4888F800404039403366
:109B70004CF83200C4E719F0080F0CBF022303238E
:109B80008B557DE521494A68002AC3D06C88B5F819
:109B900004E003E00C314A68002ABBD00B88A342E2
:109BA000F8D14B887345F5D1240A032C0CBF1178EA
:109BB000098960E7124A0221147054705BE700BF04
:109BC0009420074001000400B49CFF1F489CFF1F25
:109BD000499CFF1F0080FF1FC020074088004000F5
:109BE000882007408020074098200740F89BFF1FEF
:109BF0004C9CFF1FE49BFF1FB59CFF1FC09CFF1FD9
:109C0000B89CFF1FF49BFF1FC8004000BCE300008E
:109C10008C200740B248116AAC7804700C0600F141
:109C20009881D9F82820AF49100600F1DB81D9F8D6
:109C30003020AC49120600F1D081D9F83820A9496A
:109C4000130600F1C581D9F84020A649150600F198
:109C5000BA81D9F84820A349140600F1AF81D9F898
:109C60005020A049100600F1A481D9F858209D4940
:109C7000120600F19981D9F860209A49130600F183
:109C80008E81D9F868209749150600F18381D9F8AB
:109C900070209449140600F17881D9F87820914910
:109CA000100600F16D81D9F880208E49120600F16E
:109CB0006181D9F888208B49130600F15581D9F8C4
:109CC00090208849150600F14981D9F898208549E6
:109CD000140600F1FF808448844A85490190854834
:109CE000854D864C049700230596029580460F46C5
:109CF00016461D460394306828B1446800F04AFABD
:109D00002046002CF9D100233360029B38681A46A4
:109D1000002342F8253028B1446800F03BFA204681
:109D2000002CF9D100223A60019A98F800301146CF
:109D3000002241F8042B039A0191023B4FF00001ED
:109D400022F81510032B07D8DFE803F05D025D024F
:109D50004FF0010388F800300135042D06F10406A8
:109D600007F1040708F10108C5D1654C654D22785B
:109D7000654B049F059E0021100729701A7000F1A1
:109D80009280624962780A700021C9F83010C9F8DF
:109D900038101107DFF84C816ED4A2785C49DFF8E7
:109DA00044810A7000211207C9F85010C9F85810F0
:109DB0004BD4E27857494B4C0A7013074FF000011F
:109DC000C9F87010C9F8781000F1AE8033780193AB
:109DD000002283F00105C9F89020C9F898200021DD
:109DE000029188468E460A464B48047844F0020C9D
:109DF00009EBCC030393019B002B039B5A600CBF20
:109E00008822C82252E64FF0000388F80030A3E70A
:109E1000B0F5A06F7FF47EAE012300250193DEE74D
:109E200040F621229042F7D074E66D88002D7FF431
:109E300071AE3A49CDF804E0920011440A7822F05C
:109E400002020A70CBE7022115E600F083F9002830
:109E500000F0EB800830324AC8F86400C8F860208F
:109E600000F078F9002800F0DA8008302D4AC9F8AF
:109E70006C00C9F868209CE700F06CF9002800F03D
:109E8000E0800830264AC8F84400C8F8402000F0B6
:109E900061F9002800F0CF800830224AC9F84C0050
:109EA000C9F8482079E700F055F9002800F0A580AE
:109EB00008301B4AC9F82400C9F8202000F04AF9EC
:109EC000002800F094800830164AC9F82C00C9F820
:109ED000282056E7D1F89C00083800F05BF9FAE634
:109EE000C09CFF1F0080FF1F9C9CFF1F389CFF1F12
:109EF0008C9CFF1FC49CFF1FE49BFF1F7C9EFF1FC9
:109F0000B8E30000B59CFF1FC4200740C8200740ED
:109F1000CC200740D0200740B49CFF1FC020074042
:109F200088004000C800400000F014F9002870D0FC
:109F300008304F4AC4F88400C4F8802000F00AF9C1
:109F4000002860D008304B4AC9F88C00C9F8882036
:109F50003CE7506A083800F01DF962E6D1F8940039
:109F6000083800F017F9B0E6D1F88C00083800F096
:109F700011F9A4E6D1F88400083800F00BF998E64E
:109F8000C86F083800F006F98DE6486F083800F011
:109F900001F982E6C86E083800F0FCF877E6486EF2
:109FA000083800F0F7F86CE6C86D083800F0F2F8F1
:109FB00061E6486D083800F0EDF856E6C86C0838E0
:109FC00000F0E8F84BE6486C083800F0E3F840E6AB
:109FD000C86B083800F0DEF835E6486B083800F04A
:109FE000D9F82AE6C86A083800F0D4F81FE62A78BB
:109FF000C9F8280001322A70C3E62A78C9F820007F
:10A0000001322A705AE72A78C9F8880001322A708A
:10A01000DCE62A78C4F8800001322A708EE72A78BC
:10A02000C9F8680001322A70C3E62A78C8F86000CF
:10A0300001322A7014E72A78C9F8480001322A70E0
:10A04000ABE62A78C8F8400001322A701FE74029A1
:10A050008E4628BF4FF0400E02EB0E030293012301
:10A06000CEEB01014FEA0E4800250193BCE600BF8C
:10A0700088004000C8004000F8B500F029FD294BD9
:10A0800029482A4C2A4F2B4DDFF8BCC0DFF8BCE032
:10A09000294E00221A605A609A60DA601A615A6189
:10A0A0009A61DA611A625A629A62DA621A635A63D0
:10A0B0009A63DA631A645A649A64DA641A655A65B0
:10A0C0009A65DA651A665A669A66DA661A675A6790
:10A0D0009A67DA67C3F880200168C3F8842041F4E6
:10A0E00080210160C3F307212170C3F307401349A6
:10A0F00038701B0E2B70FF238CF80030104D8EF83B
:10A10000003010480B700123337084F864207026EF
:10A110004FF40074102207F82C3C2E70046081F874
:10A12000F820F8BD0080FF1F348004409C200740C9
:10A13000B0200740B420074094200740102007407B
:10A1400049E400E008E100E0802007408820074063
:10A15000704700BF72B60D480268B2FA82F30F2B47
:10A1600010DC4FF00041D94022EA0102026062B6E1
:10A17000074803EBC303DB00C2180021C15010469F
:10A180005160704762B60020704700BFFC8FFF1F10
:10A19000BC83FF1F0D4B0E4AC31AA2FB03231B09EE
:10A1A0000F2B0CD80B4A127852B972B60A484FF0EE
:10A1B0000041026821FA03F31A43026062B6704755
:10A1C000064A1278002AF0D0FFF768B9BC83FF1F57
:10A1D000398EE338B59CFF1FFC8FFF1FC09CFF1F0B
:10A1E00038B50E4B0E4C1B68218805468BB1B1F576
:10A1F000917F05D20B4A4B1C55549BB2238038BD2E
:10A200000022084898470021064A5554012323801C
:10A2100038BDB1F5917FEDD338BD00BFEC9CFF1F79
:10A22000869EFF1F8C9EFF1F2DE9F843214E224F73
:10A230003168012380463B70B1B1204D4B8801EB62
:10A240008302013300240F2BC2F808802C7004D83D
:10A250004B8000233B70BDE8F88340230B80032034
:10A26000FFF780F93460F4E7DFF8549099F8003094
:10A27000002BF0D0114D45F6215408E0013C12D0DE
:10A280002B7883B900F0A4FA99F800307BB1032051
:10A29000FFF7EEF80528F1D8FFF75CFF01463060C4
:10A2A0000028EBD0CAE701232B70BDE8F883BDE896
:10A2B000F88300BF089DFF1FDC9CFF1F0C9DFF1F44
:10A2C000C09CFF1F38B5084B1C7824B9074D29687E
:10A2D00009B14B8803B938BD9B000B800320FFF701
:10A2E00041F92C6038BD00BFDC9CFF1F089DFF1F9B
:10A2F0002DE9F041AD4E33680746002B00F0928007
:10A300001D885A88910803EB81010432AA428C68A7
:10A3100042D25A8004F00F064FEA1428A449A6F14D
:10A32000080208F00F00C4F30313062A00F1010528
:10A330000B701AD9B31E012B5FFA88F04ED9052E87
:10A3400048D0042E00F0A481731F022B7FD90F2E5A
:10A350000ED1F72842D8F02802D0964B1B883BB18B
:10A36000FFF73EFF0020BDE8F08127B1BD4202D0DB
:10A370000020BDE8F081082EC4F3033300F087808D
:10A38000092E11D00A2E40F094800A2BF0D18A4B6E
:10A390008A4A1B68A02181E01846FFF7FBFE0420D3
:10A3A000FFF748F83060B5E7092BE1D1270E00F040
:10A3B0007B81834B814A1B689021C4F3074611704F
:10A3C000EDB2FCB2002B00F09D80224631462846BB
:10A3D000984797E0F02843D9F72841D0F1380E2864
:10A3E000C6D801A353F820F09FA5000083A5000064
:10A3F00071A5000071A3000071A3000063A5000017
:10A4000071A3000043A6000071A300000DA6000088
:10A4100027A600004BA5000071A3000033A5000093
:10A4200017A50000674B1B78002BA1D00420FFF775
:10A4300001F80346306000289AD00588002D7FF48B
:10A4400060AFFFF7A7FE35602846BDE8F081FFF753
:10A45000C7FEC4F30740FFF7C3FE072E02D1200E4C
:10A46000FFF7BEFE534B584A198858481468584D98
:10A47000524A017000270E0AF0201F802E701070C3
:10A480000CB301225348A0470120BDE8F081082BFE
:10A490007FF46EAF504B494A1B688021C4F30746D6
:10A4A0001170EDB2240E6BB3284622463146984710
:10A4B00028E00B2E11D10B2B7FF45AAF474B3F4AAC
:10A4C0001B68B021EAE7464B1B68002B00F0FB80BD
:10A4D000404898470120BDE8F0810C2E40F00081F3
:10A4E0000C2B7FF445AF3F4B344A1B68C0211170E1
:10A4F000EDB2C4F30746002B00F0C8802846314671
:10A50000240E98473849314A314B0D7016701C7033
:10A510000120BDE8F081354B1B68002B00F0D68090
:10A520009847C4F30746254BEDB2240E83F800800C
:10A53000E8E72F4B1B68002BF2D12E4B1B68A3B111
:10A54000FE209847C4F30746EDE72B4B1B68002B12
:10A55000E6D1284B1B6843B1FC209847C4F307465B
:10A56000E1E7264B1B68002BDAD1C4F30746DAE794
:10A57000234B1B68C4F30746002BD4D030469847C2
:10A58000D1E7204B1A68002AEFD0260C630C06F0A6
:10A590007F0003F47E531843F6B29047C3E71A4B8B
:10A5A0001B68C4F30746002BE8D1BCE7149DFF1FCE
:10A5B0008A9EFF1F869EFF1FF09CFF1F849EFF1F29
:10A5C000249DFF1FC09CFF1FEC9CFF1F889EFF1F48
:10A5D000899EFF1F8C9EFF1F1C9DFF1F209DFF1F3C
:10A5E000049DFF1FE09CFF1F8B9EFF1FCC9CFF1F45
:10A5F000D09CFF1FD49CFF1F109DFF1F009DFF1FBD
:10A60000189DFF1FE89CFF1FFC9CFF1F3F4B1B6812
:10A61000002B85D13E4B1B68002BA6D0FA20984713
:10A62000C4F307467FE73B4B1B68002B7FF478AFF2
:10A63000374B1B68002B98D0FB209847C4F3074684
:10A6400071E7354B1B68002B7FF46AAF304B1B68FA
:10A65000002B8AD0F8209847C4F3074663E70E2BF7
:10A660007FF486AE2D4A2E4B1268E0211970002A25
:10A6700047D0260C610C06F07F0301F47E5119438C
:10A68000EDB2A1F5005128469047F6B2240E39E705
:10A69000FFF7A6FDC4F30740FFF7A2FD200EFFF76A
:10A6A0009FFD0020BDE8F0811E4B1D4A1B688021E4
:10A6B0001170EDB2C4F3074683B1314628463A46DD
:10A6C00098473C461EE70120BDE8F081104B1B680F
:10A6D000002B3FF44AAFFF20984746E71C4611E79E
:10A6E0000D2EBCD10D2B7FF443AE0F4B0C4A1B68D3
:10A6F000D0211170EDB2C4F30746002B7FF4FEAEFB
:10A70000C4E7C4F30746EDB2240EFBE6F89CFF1F36
:10A71000D49CFF1FD89CFF1FC89CFF1FE49CFF1FF9
:10A72000849EFF1F1C9DFF1FF49CFF1F38B5164D14
:10A730002868E0B101884488A14213DD03191B7A1F
:10A7400083B104F10803C2180C1B002302E012F8C5
:10A75000011F21B10133A342F9D1204638BD1C4667
:10A76000204638BDFFF716FD0020286038BD074B96
:10A770001B780BB9002038BD0220FEF75BFE286075
:10A780000028D7D1F6E700BF309DFF1FC09CFF1FF8
:10A790000D4B1B78BBB910B50C4C216803F0FF02C0
:10A7A0004B883F2B07DC07330B4401F1470003F8CC
:10A7B000012F8342FBD140230B800120FEF7D2FE04
:10A7C0000023236010BD7047289DFF1F2C9DFF1F95
:10A7D00038B5224C237803B138BD01232370FFF72D
:10A7E000A5FF70BB00F048F840BB00F0DBF810BBE1
:10A7F000FEF75EFDE0B900232370EFF30583002B25
:10A80000EAD1EFF3108172B6154B1868E0B1154C20
:10A810002278CAB945691D6001232370C5B1AA61B8
:10A8200001B962B600254577836898472570D3E75C
:10A8300000F020F8DFE700F01BF8D9E700F016F889
:10A84000D3E7FFF785FCCDE70029C5D162B638BD57
:10A85000054B1D600029E5D1E3E700BF359DFF1FD3
:10A860004C9BFF1F509BFF1F489BFF1F704700BF63
:10A87000704700BF704700BF054A064B10781B7831
:10A88000C0B2DBB2984238BF4030C01A704700BF38
:10A890003C9DFF1F3D9DFF1FF0B4384B1A7912F00D
:10A8A000300F2CD072B6997D01F0FF0200293DD007
:10A8B00062B6334F334938780D78334E1C46C0B2F8
:10A8C000EDB2431C402BE17928BF0023AB4202F1DB
:10A8D000FF32C9B21CBFF154184612F0FF02F0D18A
:10A8E0002A4B1B68C2B23A704BB1A84236BFC5F1C1
:10A8F0004005401B40192728C4BF01221A701F4978
:10A90000CA78D2B2150616D452060DD51B4B1B7948
:10A910005B0609D51E4B1F491B6800220A7003B154
:10A920001A70164B3C22DA70F0BC70474022D9797D
:10A930005A7462B6E3E70B791C06E5D5164B174E41
:10A940001C783378E4B2DBB29C420ED0144D01E0A7
:10A95000A3420AD00133402B28BF00230879E85CCA
:10A96000C0B2C871087D0728F2D9DBB20349337041
:10A970000B79180644BF7C23CB70C5E700A00640C6
:10A980003C9DFF1F3D9DFF1F809DFF1F389DFF1FAA
:10A99000C49DFF1FC09DFF1FC89DFF1FC19DFF1FBE
:10A9A000409DFF1F054A064B10781B78C0B2DBB2F2
:10A9B000984238BF4030C01A704700BF3C9EFF1F0E
:10A9C000D19DFF1FF0B4384B1A7912F0300F2CD004
:10A9D00072B6997D01F0FF0200293DD062B6334F77
:10A9E000334938780D78334E1C46C0B2EDB2431C63
:10A9F000402BE17928BF0023AB4202F1FF32C9B2FC
:10AA00001CBFF154184612F0FF02F0D12A4B1B680C
:10AA1000C2B23A704BB1A84236BFC5F14005401BE7
:10AA200040192728C4BF01221A701F49CA78D2B220
:10AA3000150616D452060DD51B4B1B795B0609D59E
:10AA40001E4B1F491B6800220A7003B11A70164B77
:10AA50003C22DA70F0BC70474022D9795A7462B651
:10AA6000E3E70B791C06E5D5164B174E1C783378B7
:10AA7000E4B2DBB29C420ED0144D01E0A3420AD0F6
:10AA80000133282B28BF00230879E85CC0B2C871C5
:10AA9000087D0728F2D9DBB2034933700B79180619
:10AAA00044BF7C23CB70C5E700B006403C9EFF1F2F
:10AAB000D19DFF1FFC9DFF1FCC9DFF1F409EFF1FD0
:10AAC000D09DFF1F449EFF1F3D9EFF1FD49DFF1F73
:10AAD00070B584B072B6194B194D1A4870224126D0
:10AAE0000F2480211A702E701A4604701970137882
:10AAF0001B06FCD5144B186862B6144B144C9842D4
:10AB000098BF00EB800001A998BF40000A22FDF722
:10AB100035FF01A92046002311F8012B01333AB17A
:10AB20000A2B20F8022FF7D11623237004B070BD32
:10AB30005B00DBB2237004B070BD00BF00000240B8
:10AB40000700024006000240080002407F9698007D
:10AB5000C890FF1FFFFFFFFF2DE9F043DFF8EC80F7
:10AB60008BB006460F4600F073F898F900300133B9
:10AB700004460D4637D03046394600F0DFF900284C
:10AB800031D02BA3D3E900233046394600F026FE0E
:10AB9000814668BB28A3D3E900233046394600F03C
:10ABA000FFFD00B398F90030254ACDF82090042429
:10ABB00000200021022BCDE90467CDE90267009453
:10ABC0000192CDE906012CD0684600F0BDF940B3F2
:10ABD000089B1BB101F0AAF9089B0360DDE906019F
:10ABE0000BB0BDE8F083204629460BB0BDE8F083EA
:10ABF000134A98F90030019203210022CDE904673D
:10AC0000CDE90267009108922BB90E4B4FF06042DC
:10AC1000CDE90623D8E70C490020022BCDE9060137
:10AC2000D2D101F083F922230360D1E7AFF3008092
:10AC3000EF39FAFE422E864051302DD5104987C09B
:10AC400028E40000FFFFEF470000F07FDE90FF1FC9
:10AC50002DE9F04FB04F21F00042BA4283B00C46CC
:10AC60004FEAD17605460DD9AC4FBA4225D9C1F38A
:10AC70001303034340F0EF800EB10020014603B000
:10AC8000BDE8F08FA64B9A4200F2CC80A54B9A42C9
:10AC900000F2DE808AA3D3E9002300F05DF90022F0
:10ACA000A14B00F09BFD002800F0058128462146BD
:10ACB00000229D4B00F050F9E1E783A3D3E9002384
:10ACC00000F08CFD002840F0CB802846214680A370
:10ACD000D3E9002300F064FD0028CED1934B284631
:10ACE00003EBC60821467CA3D3E9002300F0E6FA73
:10ACF000D8E9002300F030F900F07AFD804600F03A
:10AD000077FA77A3D3E9002306460F4600F0D6FA78
:10AD100002460B462846214600F01CF972A3D3E9EF
:10AD20000023CDE900013046394600F0C7FA8246DB
:10AD30008B4652465B46DDE9000100F00BF9054603
:10AD40000C462A4623462846214600F0B7FA68A357
:10AD5000D3E9002306460F4600F0B0FA66A3D3E914
:10AD6000002300F0F7F832463B4600F0A7FA64A350
:10AD7000D3E9002300F0F0F832463B4600F09EFA9B
:10AD800061A3D3E9002300F0E5F832463B4600F02A
:10AD900095FA5FA3D3E9002300F0DEF832463B4684
:10ADA00000F08CFA02460B462846214600F0D2F805
:10ADB00006460F462846214632463B46B8F1000F6C
:10ADC00056D000F07BFA324604460D463B46002042
:10ADD0004FF0804100F0BEF802460B46204629465F
:10ADE00000F096FB02460B465046594600F0B2F87A
:10ADF000DDE9002300F0AEF80B4602464A49002088
:10AE000000F0A8F86FF47F7398454FDA08F57A7868
:10AE100001EB085100224FF0B87300F04FFA03B075
:10AE2000BDE8F08F424B9A423FF658AF414BF400D9
:10AE30002344D3E9002300F08DF83F4BC6F101080D
:10AE40001C44CDE90001D4E900ABC6EB080870E76B
:10AE50004FF0000875E702460B4600F07DF80EE75C
:10AE600017A3D3E900231046194600F027FA06E796
:10AE700000F024FA0022804689464FF08043304695
:10AE8000394600F067F802460B464046494600F056
:10AE90003FFB2A46234600F05DF802460B460020A1
:10AEA000214900F057F803B0BDE8F08F01EB0851DD
:10AEB00003B0BDE8F08F804643E700BFAFF30080EA
:10AEC0009C7500883CE4377EEF39FAFE422E8640BE
:10AED00051302DD5104987C0FE822B654715F73FAD
:10AEE0000000E0FE422EE63F763C7935EF39EA3D40
:10AEF000D0A4BE726937663EF16BD2C541BDBB3E80
:10AF00002CDE25AF6A56113F93BDBE166CC1663F5D
:10AF10003E5555555555C53F412E8640FFFFEF7FA5
:10AF2000422ED63FFFFF2F3E0000F03F30E40000EE
:10AF3000B1A2F03F50E4000040E4000041F00041C5
:10AF400001F58010C00F70470020704781F000416C
:10AF500002E000BF83F0004330B54FEA41044FEAFE
:10AF6000430594EA050F08BF90EA020F1FBF54EA99
:10AF7000000C55EA020C7FEA645C7FEA655C00F035
:10AF8000E2804FEA5454D4EB5555B8BF6D420CDD06
:10AF90002C4480EA020281EA030382EA000083EA89
:10AFA000010180EA020281EA0303362D88BF30BD29
:10AFB00011F0004F4FEA01314FF4801C4CEA11317F
:10AFC00002D0404261EB410113F0004F4FEA0333DE
:10AFD0004CEA133302D0524263EB430394EA050F69
:10AFE00000F0A780A4F10104D5F1200E0DDB02FAD8
:10AFF0000EFC22FA05F2801841F1000103FA0EF26C
:10B00000801843FA05F359410EE0A5F120050EF131
:10B01000200E012A03FA0EFC28BF4CF0020C43FA62
:10B0200005F3C01851EBE37101F0004507D54FF06F
:10B03000000EDCF1000C7EEB00006EEB0101B1F5BF
:10B04000801F1BD3B1F5001F0CD349085FEA300005
:10B050004FEA3C0C04F101044FEA445212F5800F10
:10B0600080F09A80BCF1004F08BF5FEA500C50F1AD
:10B07000000041EB045141EA050130BD5FEA4C0C90
:10B08000404141EB010111F4801FA4F10104E9D119
:10B0900091F0000F04BF01460020B1FA81F308BF10
:10B0A0002033A3F10B03B3F120020CDA0C3208DDDC
:10B0B00002F1140CC2F10C0201FA0CF021FA02F1B7
:10B0C0000CE002F11402D8BFC2F1200C01FA02F127
:10B0D00020FA0CFCDCBF41EA0C019040E41AA2BF4C
:10B0E00001EB0451294330BD6FEA04041F3C1CDA14
:10B0F0000C340EDC04F11404C4F1200220FA04F034
:10B1000001FA02F340EA030021FA04F345EA0301DD
:10B1100030BDC4F10C04C4F1200220FA02F001FA9F
:10B1200004F340EA0300294630BD21FA04F0294621
:10B1300030BD94F0000F83F4801306BF81F48011BA
:10B140000134013D4EE77FEA645C18BF7FEA655C2D
:10B1500029D094EA050F08BF90EA020F05D054EAFF
:10B16000000C04BF1946104630BD91EA030F1EBF04
:10B170000021002030BD5FEA545C05D14000494108
:10B1800028BF41F0004130BD14F580043CBF01F5FB
:10B19000801130BD01F0004545F0FE4141F47001E1
:10B1A0004FF0000030BD7FEA645C1ABF19461046BC
:10B1B0007FEA655C1CBF0B46024650EA013406BFBD
:10B1C00052EA033591EA030F41F4002130BD00BF7C
:10B1D00090F0000F04BF0021704730B54FF4806439
:10B1E00004F132044FF000054FF0000150E700BFBA
:10B1F00090F0000F04BF0021704730B54FF4806419
:10B2000004F1320410F0004548BF40424FF0000105
:10B210003EE700BF42004FEAE2014FEA31014FEA48
:10B2200002701FBF12F07F4393F07F4F81F0605197
:10B23000704792F0000F14BF93F07F4F704730B506
:10B240004FF4607401F0004521F0004120E700BF99
:10B2500050EA010208BF704730B54FF000050AE020
:10B2600050EA010208BF704730B511F0004502D521
:10B27000404261EB41014FF4806404F132045FEA23
:10B28000915C3FF4DCAE4FF003025FEADC0C18BFC8
:10B2900003325FEADC0C18BF033202EBDC02C2F1BE
:10B2A000200300FA03FC20FA02F001FA03FE40EA50
:10B2B0000E0021FA02F11444C1E600BF70B54FF050
:10B2C000FF0C4CF4E06C1CEA11541DBF1CEA135532
:10B2D00094EA0C0F95EA0C0F00F0DEF82C4481EA9A
:10B2E000030621EA4C5123EA4C5350EA013518BFBA
:10B2F00052EA033541F4801143F4801338D0A0FBA7
:10B3000002CE4FF00005E1FB02E506F00042E0FB53
:10B3100003E54FF00006E1FB03569CF0000F18BF59
:10B320004EF0010EA4F1FF04B6F5007F64F5407401
:10B3300004D25FEA4E0E6D4146EB060642EAC62194
:10B3400041EA55514FEAC52040EA5E504FEACE2E01
:10B35000B4F1FD0C88BFBCF5E06F1ED8BEF1004F04
:10B3600008BF5FEA500E50F1000041EB045170BD80
:10B3700006F0004646EA010140EA020081EA0301C4
:10B38000B4EB5C04C2BFD4EB0C0541EA045170BDC0
:10B3900041F480114FF0000E013C00F3AB8014F13A
:10B3A000360FDEBF002001F0004170BDC4F1000483
:10B3B000203C35DA0C341BDC04F11404C4F1200504
:10B3C00000FA05F320FA04F001FA05F240EA02005F
:10B3D00001F0004221F0004110EBD37021FA04F695
:10B3E00042EB06015EEA430E08BF20EAD37070BD4F
:10B3F000C4F10C04C4F1200500FA04F320FA05F0AE
:10B4000001FA04F240EA020001F0004110EBD370AF
:10B4100041F100015EEA430E08BF20EAD37070BD1F
:10B42000C4F1200500FA05F24EEA020E20FA04F3F8
:10B4300001FA05F243EA020321FA04F001F00041A7
:10B4400021FA04F220EA020000EBD3705EEA430E18
:10B4500008BF20EAD37070BD94F0000F0FD101F047
:10B460000046400041EB010111F4801F08BF013C80
:10B47000F7D041EA060195F0000F18BF704703F0BE
:10B480000046520043EB030313F4801F08BF013D45
:10B49000F7D043EA0603704794EA0C0F0CEA135501
:10B4A00018BF95EA0C0F0CD050EA410618BF52EABB
:10B4B0004306D1D181EA030101F000414FF00000C1
:10B4C00070BD50EA410606BF1046194652EA4306CF
:10B4D00019D094EA0C0F02D150EA013613D195EA43
:10B4E0000C0F05D152EA03361CBF104619460AD18B
:10B4F00081EA030101F0004141F0FE4141F4700195
:10B500004FF0000070BD41F0FE4141F4780170BD84
:10B5100070B54FF0FF0C4CF4E06C1CEA11541DBFE9
:10B520001CEA135594EA0C0F95EA0C0F00F0A7F8EB
:10B53000A4EB050481EA030E52EA03354FEA013118
:10B5400000F088804FEA03334FF0805545EA13132B
:10B5500043EA12634FEA022245EA111545EA1065F3
:10B560004FEA00260EF000419D4208BF964244F18A
:10B57000FD0404F5407402D25B084FEA3202B61AA9
:10B5800065EB03055B084FEA32024FF480104FF47D
:10B59000002CB6EB020E75EB030E22BFB61A7546F1
:10B5A00040EA0C005B084FEA3202B6EB020E75EB84
:10B5B000030E22BFB61A754640EA5C005B084FEAEC
:10B5C0003202B6EB020E75EB030E22BFB61A7546B9
:10B5D00040EA9C005B084FEA3202B6EB020E75EBC4
:10B5E000030E22BFB61A754640EADC0055EA060E85
:10B5F00018D04FEA051545EA16754FEA06164FEAC8
:10B60000C30343EA52734FEAC2025FEA1C1CC0D173
:10B6100011F4801F0BD141EA00014FF000004FF000
:10B62000004CB6E711F4801F04BF01430020B4F1C1
:10B63000FD0C88BFBCF5E06F3FF6AFAEB5EB030C79
:10B6400004BFB6EB020C5FEA500C50F1000041EB76
:10B65000045170BD0EF0004E4EEA113114EB5C0443
:10B66000C2BFD4EB0C0541EA045170BD41F4801116
:10B670004FF0000E013C90E645EA060E8DE60CEA1E
:10B68000135594EA0C0F08BF95EA0C0F3FF43BAF3B
:10B6900094EA0C0F0AD150EA01347FF434AF95EAF2
:10B6A0000C0F7FF425AF104619462CE795EA0C0FD6
:10B6B00006D152EA03353FF4FDAE1046194622E7A3
:10B6C00050EA410618BF52EA43067FF4C5AE50EA7D
:10B6D00041047FF40DAF52EA43057FF4EBAE12E76D
:10B6E0004FF0FF3C06E000BF4FF0010C02E000BF4E
:10B6F0004FF0010C4DF804CD4FEA410C7FEA6C5C31
:10B700004FEA430C18BF7FEA6C5C1BD001B050EAD3
:10B71000410C0CBF52EA430C91EA030F02BF90EABE
:10B72000020F0020704710F1000F91EA030F58BF7D
:10B73000994208BF90422CBFD8176FEAE37040F0DF
:10B74000010070474FEA410C7FEA6C5C02D150EA7D
:10B75000013C07D14FEA430C7FEA6C5CD6D152EA38
:10B76000033CD3D05DF8040B704700BF84461046FD
:10B7700062468C461946634600E000BF01B5FFF7FC
:10B78000B7FF002848BF10F1000F01BD4DF808EDCC
:10B79000FFF7F4FF0CBF012000205DF808FB00BF9D
:10B7A0004DF808EDFFF7EAFF34BF012000205DF8F7
:10B7B00008FB00BF4DF808EDFFF7E0FF94BF012044
:10B7C00000205DF808FB00BF4DF808EDFFF7CEFF45
:10B7D00094BF012000205DF808FB00BF4DF808ED84
:10B7E000FFF7C4FF34BF012000205DF808FB00BF55
:10B7F0004FEA410212F5001215D211D56FF4787399
:10B80000B3EB625212D94FEAC12343F0004343EA3B
:10B81000505311F0004F23FA02F018BF4042704716
:10B820004FF00000704750EA013005D111F00040A0
:10B8300008BF6FF0004070474FF00000704700BF36
:10B840004FEA4102B2F1E04324BFB3F5001CDCF142
:10B85000FE5C0DD901F0004C4FEAC0024CEA50707A
:10B86000B2F1004F40EB830008BF20F001007047A9
:10B8700011F0804F21D113F13872BCBF01F00040AC
:10B88000704741F480114FEA5252C2F11802C2F1DE
:10B89000200C10FA0CF320FA02F018BF40F001005F
:10B8A0004FEAC1234FEAD32303FA0CFC40EA0C0011
:10B8B00023FA02F34FEA4303CCE77FEA625307D14E
:10B8C00050EA01331EBF4FF0FE4040F44000704785
:10B8D00001F0004040F0FE4040F40000704700BF1F
:10B8E00080F0004002E000BF81F0004142001FBF35
:10B8F0005FEA410392EA030F7FEA226C7FEA236C3E
:10B900006AD04FEA1262D2EB1363C1BFD218414032
:10B9100048404140B8BF5B42192B88BF704710F0C8
:10B92000004F40F4000020F07F4018BF404211F06B
:10B93000004F41F4000121F07F4118BF494292EAD3
:10B94000030F3FD0A2F1010241FA03FC10EB0C00FF
:10B95000C3F1200301FA03F100F0004302D549428C
:10B9600060EB4000B0F5000F13D3B0F1807F06D339
:10B9700040084FEA310102F10102FE2A51D2B1F131
:10B98000004F40EBC25008BF20F0010040EA030026
:10B990007047490040EB000010F4000FA2F10102D3
:10B9A000EDD1B0FA80FCACF1080CB2EB0C0200FA5D
:10B9B0000CF0AABF00EBC25052421843BCBFD040AB
:10B9C0001843704792F0000F81F4000106BF80F425
:10B9D00000000132013BB5E74FEA41037FEA226CE8
:10B9E00018BF7FEA236C21D092EA030F04D092F0B3
:10B9F000000F08BF0846704790EA010F1CBF0020E7
:10BA0000704712F07F4F04D1400028BF40F0004043
:10BA1000704712F100723CBF00F50000704700F063
:10BA2000004343F0FE4040F4000070477FEA22628A
:10BA300016BF08467FEA23630146420206BF5FEA5B
:10BA4000412390EA010F40F4800070474FF000035B
:10BA500004E000BF10F0004348BF40425FEA000C22
:10BA600008BF704743F0964301464FF000001CE0CA
:10BA700050EA010208BF70474FF000030AE000BF20
:10BA800050EA010208BF704711F0004302D540425E
:10BA900061EB41015FEA010C02BF844601460020D0
:10BAA00043F0B64308BFA3F18053A3F50003BCFAEB
:10BAB0008CF2083AA3EBC25310DB01FA02FC634498
:10BAC00000FA02FCC2F12002BCF1004F20FA02F29F
:10BAD00043EB020008BF20F00100704702F1200292
:10BAE00001FA02FCC2F1200250EA4C0021FA02F2F3
:10BAF00043EB020008BF20EADC7070474FF0FF0CF8
:10BB00001CEAD0521EBF1CEAD15392EA0C0F93EAF2
:10BB10000C0F6FD01A4480EA010C400218BF5FEA94
:10BB200041211ED04FF0006343EA501043EA511107
:10BB3000A0FB01310CF00040B1F5000F3EBF490001
:10BB400041EAD3715B0040EA010062F17F02FD2A05
:10BB50001DD8B3F1004F40EBC25008BF20F00100E8
:10BB6000704790F0000F0CF0004C08BF49024CEAFF
:10BB7000502040EA51207F3AC2BFD2F1FF0340EA91
:10BB8000C250704740F400004FF00003013A5DDC02
:10BB900012F1190FDCBF00F000407047C2F1000243
:10BBA000410021FA02F1C2F1200200FA02FC5FEA30
:10BBB000310040F1000053EA4C0308BF20EADC707A
:10BBC000704792F0000F00F0004C02BF400010F4EC
:10BBD000000F013AF9D040EA0C0093F0000F01F099
:10BBE000004C02BF490011F4000F013BF9D041EABB
:10BBF0000C018FE70CEAD15392EA0C0F18BF93EABD
:10BC00000C0F0AD030F0004C18BF31F0004CD8D1E6
:10BC100080EA010000F00040704790F0000F17BF6D
:10BC200090F0004F084691F0000F91F0004F14D0B3
:10BC300092EA0C0F01D142020FD193EA0C0F03D10B
:10BC40004B0218BF084608D180EA010000F000400E
:10BC500040F0FE4040F40000704740F0FE4040F4E9
:10BC6000400070474FF0FF0C1CEAD0521EBF1CEA88
:10BC7000D15392EA0C0F93EA0C0F69D0A2EB0302A6
:10BC800080EA010C49024FEA402037D04FF0805340
:10BC900043EA111143EA10130CF000408B4238BF05
:10BCA0005B0042F17D024FF4000C8B4224BF5B1A13
:10BCB00040EA0C00B3EB510F24BFA3EB510340EA61
:10BCC0005C00B3EB910F24BFA3EB910340EA9C000F
:10BCD000B3EBD10F24BFA3EBD10340EADC001B017F
:10BCE00018BF5FEA1C1CE0D1FD2A3FF650AF8B4223
:10BCF00040EBC25008BF20F0010070470CF0004C30
:10BD00004CEA50207F32C2BFD2F1FF0340EAC2505A
:10BD1000704740F400004FF00003013A37E792F01B
:10BD2000000F00F0004C02BF400010F4000F013A79
:10BD3000F9D040EA0C0093F0000F01F0004C02BF74
:10BD4000490011F4000F013BF9D041EA0C0195E7DD
:10BD50000CEAD15392EA0C0F08D142027FF47DAF76
:10BD600093EA0C0F7FF470AF084676E793EA0C0F66
:10BD700004D14B023FF44CAF08466EE730F0004C64
:10BD800018BF31F0004CCAD130F000427FF45CAFF4
:10BD900031F000437FF43CAF5FE700BF4FF0FF3C62
:10BDA00006E000BF4FF0010C02E000BF4FF0010CB5
:10BDB0004DF804CD4FEA40024FEA41037FEA226C7E
:10BDC00018BF7FEA236C11D001B052EA530C18BFA0
:10BDD00090EA010F58BFB2EB030088BFC81738BF05
:10BDE0006FEAE17018BF40F0010070477FEA226CF3
:10BDF00002D15FEA402C05D17FEA236CE4D15FEAEF
:10BE0000412CE1D05DF8040B704700BF8446084622
:10BE10006146FFE70FB5FFF7C9FF002848BF10F1E3
:10BE2000000F0FBD4DF808EDFFF7F4FF0CBF012028
:10BE300000205DF808FB00BF4DF808EDFFF7EAFFB2
:10BE400034BF012000205DF808FB00BF4DF808ED6D
:10BE5000FFF7E0FF94BF012000205DF808FB00BF62
:10BE60004DF808EDFFF7D2FF94BF012000205DF8E8
:10BE700008FB00BF4DF808EDFFF7C8FF34BF0120F5
:10BE800000205DF808FB00BF4FEA4002B2F1FE4F10
:10BE90000FD34FF09E03B3EB12620DD94FEA00238C
:10BEA00043F0004310F0004F23FA02F018BF404265
:10BEB00070474FF00000704712F1610F01D142024C
:10BEC00005D110F0004008BF6FF0004070474FF000
:10BED0000000704742000ED2B2F1FE4F0BD34FF07C
:10BEE0009E03B3EB126209D44FEA002343F00043F0
:10BEF00023FA02F070474FF00000704712F1610F13
:10BF000001D1420202D14FF0FF3070474FF00000E4
:10BF1000704700BF0B460146184600F001B800BF4D
:10BF200013460A460146022000F00CBC014B18687B
:10BF3000704700BF0895FF1F70B50F4E0F4D761B61
:10BF4000B61018BF002405D0013455F8043B9847BB
:10BF5000A642F9D10A4E0B4D761B02F083FAB610B9
:10BF600018BF002406D0013455F8043B9847A64278
:10BF7000F9D170BD70BD00BF70E4000070E4000036
:10BF800080E4000070E40000024B0146186800F0F5
:10BF90000BB800BF0895FF1F024B0146186800F060
:10BFA00095BC00BF0895FF1F2DE9F04F01F10B056F
:10BFB000162D83B0064640F29F8035F0070500F14C
:10BFC000BF80A94200F2BC8000F0F4FAB5F5FC7F16
:10BFD000C0F09C826B0A00F0BA80042B00F28381CF
:10BFE000A80900F1390E4FEA4E033830C44F07EB71
:10BFF0008303A3F108015C68A14207D1ACE0002AE9
:10C0000080F2AC80E468A14200F0A680636823F06F
:10C0100003035A1B0F2AF2DDB9493C6901F1080EEE
:10C02000744500F0B381636823F003035A1B0F2AA1
:10C0300000F39981002AC1F814E0C1F810E080F201
:10C040009E80B3F5007F80F06781DB0803F1010C6F
:10C0500001229B1002FA03F34A6851F83C80C4F8AD
:10C06000088001EBCC091A43A9F10803E3604A6098
:10C0700041F83C40C8F80C40831001249C40944295
:10C0800000F28A80144206D120F0030064001442BA
:10C0900000F10400FAD007EBC009CC468046DCF87A
:10C0A0000C108C4507D173E1002A80F28181C968A8
:10C0B0008C4500F06D814B6823F003035A1B0F2A57
:10C0C000F2DD0C46D1F80CC054F8088F4B1945F03E
:10C0D00001054D6042F00101C8F80CC03046CCF8B3
:10C0E00008807B613B61C3F80CE0C3F808E059604D
:10C0F0009A5000F061FA1FE0102921D800F05AFA96
:10C100001025062302207E4F07EB8303A3F10802CC
:10C110005C68944200F045816368E168A56823F09B
:10C120000303234430465A68E96042F001028D60FF
:10C130005A6000F041FA0834204603B0BDE8F08FA1
:10C1400000240C232046336003B0BDE8F08F802329
:10C150004FF0400E3F2049E770465DE72344E16819
:10C160005A68A56842F00102E96030468D605A6065
:10C1700000F022FA0834204603B0BDE8F08F2344D3
:10C1800030465A6842F001025A6000F015FA08344D
:10C19000204603B0BDE8F08FBC68636823F0030855
:10C1A000A84504D3C5EB08030F2B00F38C80554B37
:10C1B000DFF860911A68D9F8003001332A4404EBA3
:10C1C000080A00F0608102F580520F3222F47F628B
:10C1D00022F00F0211463046019200F0EFF9B0F163
:10C1E000FF3F8346019A00F05881824500F2FC80AF
:10C1F000454B1968DA451144196000F05381D9F8AC
:10C200000000DFF810E101301BBFCAEB0B0A5144FC
:10C21000CEF800B019601BF0070100F01781C1F1E2
:10C220000800C1F58051834408315A44C2F30B021F
:10C23000C2EB010949463046019300F0BFF9431CA7
:10C24000019B00F03F81CBEB00024A4442F0010227
:10C250001968C7F808B04944BC42CBF804201960FB
:10C26000DFF8A49016D0B8F10F0F40F2FD8062689D
:10C27000A8F10C0323F00703E01802F001024FF0CD
:10C28000050E1A430F2B6260C0F804E0C0F808E006
:10C2900000F21C811D4BBC681A68914288BF19606E
:10C2A0001B4B1A689142626888BF196022F0030232
:10C2B0009542A2EB050301D80F2B04DC304600F0B9
:10C2C0007BF9002438E7621943F0010345F00105CA
:10C2D00065603046BA60536000F06EF9083420465D
:10C2E00003B0BDE8F08F142B71D9542B00F2A48059
:10C2F000280B00F16F0E4FEA4E036E3076E600BF5A
:10C300000C95FF1F509EFF1F549EFF1F4C9EFF1F4A
:10C31000489EFF1F1899FF1F5A0A042A5ED9142A43
:10C3200000F2B38002F15C0149005B3207EB810C43
:10C3300057F82110DFF8DC81ACF1080C8C4500F0D7
:10C3400088804A6822F00302934202D289688C45B1
:10C35000F7D1D1F80CC07A68C4F80CC0A160CCF851
:10C360000840CC6088E6631942F0010745F00105FA
:10C37000656030464B610B61C3F80CE0C3F808E020
:10C380005F609A50083400F017F9D5E64A6873E602
:10C3900008F1010818F0030F0CF1080C7FF47FAED0
:10C3A00030E0DC68A34208BF02303FF435AEB3E6AC
:10C3B0000B440C465A68C96854F8085F42F0010201
:10C3C0005A603046E9608D6000F0F6F8B4E603F19B
:10C3D0005C0E03F15B004FEA4E0307E69A0902F197
:10C3E000390149003832A1E7BC424A4B3FF400AF63
:10C3F0009C68626822F003025AE759F808399945A7
:10C4000040F0828010F0030F00F1FF30F5D17B681F
:10C4100023EA04037B6064009C423FF6BDAE002C1F
:10C420003FF4BAAE1C4240467FF435AE64001C4275
:10C4300000F10400FAD02EE6B3F5AA7F18D8E80B75
:10C4400000F1780E4FEA4E037730CFE54FF480517C
:10C45000EBE60121D8F80430921001FA02F21A43F7
:10C46000C8F80420614677E70123CBF8043025E7BC
:10C4700040F25452934220D8A80C00F17D0E4FEAAE
:10C480004E037C30B2E51032A4E6542A26D81A0BAB
:10C4900002F16F0149006E3248E7BC68626822F021
:10C4A000030205E7CAF30B0000287FF4A8AE42445C
:10C4B000BB6842F001025A60ECE6FE234FF07F0EAB
:10C4C0007E2093E501224FF00009C1E604F1080146
:10C4D000304600F0FBF9D9F80010DBE6B2F5AA7F90
:10C4E00005D8DA0B02F17801490077321EE740F2F5
:10C4F00054518A4205D89A0C02F17D0149007C32E0
:10C5000014E7FE217E2211E77B6884E7E808431CDC
:10C510005B00F8E50C95FF1F70B4840746D0541EED
:10C52000002A41D0CDB2034602E0621EE4B31446B5
:10C5300003F8015B9A07F8D1032C2ED9CDB245EA56
:10C5400005250F2C45EA054519D903F110022646A9
:10C55000103E0F2E42F8105C42F80C5C42F8085C6A
:10C5600042F8045C02F11002F2D8A4F1100222F0A9
:10C570000F0204F00F041032032C13440DD91E4691
:10C580002246043A032A46F8045BFAD8221F22F016
:10C5900003020432134404F003042CB1C9B21C4456
:10C5A00003F8011BA342FBD170BC7047144603463D
:10C5B000C2E700BF704700BF704700BF38B5074CE7
:10C5C0000023054608462360FCF7A2F9431C00D06F
:10C5D00038BD2368002BFBD02B6038BDB09FFF1FF8
:10C5E000FFFFFFFFFFFFFFFFFFFFFFFFFFFFFFFF5B
:10C5F000FFFFFFFFFFFFFFFFFFFFFFFFFFFFFFFF4B
:10C6000090F800F06DE9024520F007016FF0000C92
:10C6100010F0070491F820F040F049804FF000043A
:10C620006FF00700D1E9002391F840F000F1080015
:10C6300082FA4CF2A4FA8CF283FA4CF3A2FA8CF34D
:10C640004BBBD1E9022382FA4CF200F10800A4FAB4
:10C650008CF283FA4CF3A2FA8CF3E3B9D1E9042308
:10C6600082FA4CF200F10800A4FA8CF283FA4CF33F
:10C67000A2FA8CF37BB9D1E9062301F1200182FAF9
:10C680004CF200F10800A4FA8CF283FA4CF3A2FAFF
:10C690008CF3002BC6D0002A04BF04301A4612BA0D
:10C6A000B2FA82F2FDE8024500EBD2007047D1E910
:10C6B000002304F00305C4F100004FEAC50514F09F
:10C6C000040F91F840F00CFA05F562EA05021CBF70
:10C6D00063EA050362464FF00004A9E740EA01035C
:10C6E0009B0770B42BD1032A29D90C460346214657
:10C6F00054F8046BA6F1013525EA060515F0803FD4
:10C7000006D1043A032A43F8046B2146EFD8A2B1BC
:10C710000C781C70013A013301313CB16AB111F857
:10C72000014B03F8014B013A002CF7D12AB11A440E
:10C73000002103F8011B9A42FBD170BC70470346ED
:10C74000E5E700BF2DE9F047254C2568D5F84841BD
:10C750000646884692469946C4B360681F2817DC8F
:10C76000431C76B104EB80050122C5F888A0D4F8FB
:10C77000881182401143022EC4F88811C5F808912F
:10C780001ED00230636044F820800020BDE8F087AE
:10C79000144B03B34FF4C870FFF7F6FB0446D0B157
:10C7A000D5F84831002780E88800C5F84841384668
:10C7B0000123C4F88871C4F88C71002EE1D0D1E750
:10C7C000D4F88C110A43C4F88C21DAE705F5A67475
:10C7D000C5F84841C1E74FF0FF30BDE8F08700BF22
:10C7E00060E4000089BF0000024B13B1024800F072
:10C7F00005B870470000000009C80000002301468A
:10C800001A461846FFF79EBF38B5074D074C2C1B3C
:10C81000A41005D0013C55F8043D9847002CF9D1EF
:10C82000BDE8384001F02CBE000000000000000010
:10C83000F8B5234F0C460646FFF7BCFEBB685D68A3
:10C8400025F00305291B01F6EF7121F47F6121F02A
:10C850000F01A1F58054B4F5805F07DB002130465D
:10C86000FFF7ACFEBB682B44984204D03046FFF77C
:10C87000A3FE0020F8BD61423046FFF79FFE013065
:10C880000DD0104BBA6819682D1B45F001053046D4
:10C89000091B55601960FFF78FFE0120F8BD0021CC
:10C8A0003046FFF78BFEBA68831A0F2BDEDD064C8D
:10C8B0000449246843F00103001B53600860D5E776
:10C8C0000C95FF1F549EFF1F1899FF1F002945D08C
:10C8D0002DE9F0410D468046FFF76CFE55F8047CCB
:10C8E0006A4927F00103A5F10804E2188E68506830
:10C8F000B24220F0030062D0FE0750600BD455F81E
:10C90000087CE41B01F1080EA56875453B446FD017
:10C91000E768EF60BD6015186D68ED0742D543F01C
:10C9200001026260E350B3F5007F18D2DB085A1CA5
:10C930004D6851F83270A76001209B1000FA03F394
:10C9400001EBC2001D430838E0604D6041F8324001
:10C95000FC604046BDE8F041FFF72EBE70475A0A22
:10C96000042A53D89A0902F139077F0002F13805E9
:10C9700001EB870051F827204449083890424DD0F8
:10C98000516821F003018B4202D292689042F7D1A4
:10C99000D068E060A2608460D4604046BDE8F041A9
:10C9A000FFF70ABE95683A4FBD4203443FD0D068B6
:10C9B000E86043F0010285606260E350B3E7FF077F
:10C9C000034407D455F8082CA41A1344A068E2685D
:10C9D000C26090602F4A126843F001009342606089
:10C9E0008C60B6D32C4B40461968FFF721FFB0E7A7
:10C9F00011184968C90744D49168D268CA600344D1
:10CA000043F0010091606060E350A2E7142A17D858
:10CA100002F15C077F0002F15B05A9E7AA104B68F1
:10CA2000012505FA02F213434B600246B1E743F0D9
:10CA300001024C610C61E560A5606260E35088E72B
:10CA4000542A06D81A0B02F16F077F0002F16E0517
:10CA50008EE7B2F5AA7F06D8DA0B02F178077F00DD
:10CA600002F1770584E740F25450824206D89A0CCE
:10CA700002F17D077F0002F17C0579E7FE277E2524
:10CA800076E743F001026260E35062E70C95FF1F16
:10CA90001495FF1F1499FF1F509EFF1F000058029E
:10CAA00046056608540BD80E5C127017FC21F82A54
:10CAB00070305834DC37663A8C3C803EFF3FFFFFD5
:10CAC0000000FF03FF07FF0BFF0FFF13FF17FF1B04
:10CAD000FF1FFF23FF27FF2BFF2FFF33FF37FF3BF6
:10CAE000FF3FFFFF0000580246056608540BD80EB2
:10CAF0005C12E015FA19141E6022AC265C2B0C3077
:10CB0000BC34023AFF3FFFFF0000900120031405F0
:10CB1000D0075A0AAC0DCC10B4146A18E81C3421A2
:10CB200080252A2B70301437FF3FFFFF0000C8001C
:10CB3000F4018403140508072E091C0CD80EF81103
:10CB4000AE159619401F1C25F22B5834FF3FFFFFEE
:10CB500000006400C8009001BC021A04DC059E07B6
:10CB6000F609800CA00F2413A2174C1D5424442F47
:10CB7000FF3FFFFF0000580246056608540BA00F58
:10CB8000D4172823F82A442F643284354038663A73
:10CB90008C3C803EFF3FFFFF00007805220B041015
:10CBA000B4143219B01DFC214826FE29822D3831DB
:10CBB00026344637663A223DFF3FFFFF0000540B04
:10CBC000EC13FA1908201C253629EC2C0C302C33D8
:10CBD000E8357238663AF63B863D163FFF3FFFFF69
:10CBE00060CC0000BCCB00009CCC000098CB0000C7
:10CBF000C0CA0000E4CA000008CB00002CCB000033
:10CC000050CB00009CCA000074CB0000C0CC0000D8
:10CC100014CC00000000D007800CD80E0010C01209
:10CC2000EC130C17FA19141E6022AC265C2B0C3086
:10CC3000BC34023AFF3FFFFF00000000CDCC4C3D6A
:10CC4000CDCCCC3D9A99193ECDCC4C3E0000803ED7
:10CC50009A99993E3333B33ECDCCCC3E6666E63EE0
:10CC60000000CC10581BFC21AC26C62A7C2E383183
:10CC7000F4334C36A438983A5A3C543D803E7A3FBF
:10CC8000FF3FFFFF2C011301FA00E100C800AF00D5
:10CC900096007D0064004B00320019000000D007B0
:10CCA000100E88133219AA1E282374275C2B442FD8
:10CCB000643284354038663A8C3C803EFF3FFFFF4B
:10CCC000000078053408540B800C3C0F5C12E01512
:10CCD000FA19141E6022AC265C2B0C30BC34023ACC
:10CCE000FF3FFFFF54CD0000B699FF1F0000FF0F6C
:10CCF000869AFF1F0000FF0F0533000020CD0000C3
:10CD0000149AFF1F32005E010000000000000000C6
:10CD1000A532000054485200534E53004D41580074
:10CD2000544F5543482053454E534500455854529F
:10CD30004120434F4E54524F4C4C4552000000008E
:10CD400050495443482042454E440000424954450E
:10CD50000000000042524541544800FF2CCD000025
:10CD6000529AFF1FF401A00FEE99FF1FF401A00FCC
:10CD7000B13200004CCD0000409AFF1FBC025C1293
:10CD80002A9AFF1FBC025C12E932000040CD00006D
:10CD9000509AFF1FF401A00F0C9AFF1FF401A00F7F
:10CDA000CD3200003CD40000CCD40000E0D4000020
:10CDB000E4D40000E8D40000ECD40000F0D400007B
:10CDC000F4D40000F8D40000D4D40000FCD4000057
:10CDD0003CD4000038D40000DCD400003CD4000077
:10CDE000CCD40000D0D40000D4D40000D8D40000AB
:10CDF00000D5000004D5000008D500000CD50000C7
:10CE000010D5000014D5000018D500001CD5000076
:10CE100020D5000024D5000028D500002CD5000026
:10CE200030D500000000000098D6000080D6000039
:10CE3000469AFF1F0000300000000000454400003B
:10CE40007149000000000000000000000000000028
:10CE500000000000000000000000000000000000D2
:10CE600000000000000000000000000000000000C2
:10CE700000000000000000000000000000000000B2
:10CE800000000000000000000000000000000000A2
:10CE90000000000000000000000000000000000092
:10CEA0000000000000000000000000000000000082
:10CEB0000000000000000000000000000000000072
:10CEC0000000000000000000000000000000000062
:10CED0000000000000000000000000000000000052
:10CEE0000000000000000000000000000000000042
:10CEF0000000000000000000000000000000000032
:10CF00000000000000000000000000000000000021
:10CF10000000000000000000000000000000000011
:10CF20000000000000000000000000000000000001
:10CF300000000000000000000000000000000000F1
:10CF400000000000000000000000000000000000E1
:10CF500000000000000000000000000000000000D1
:10CF60000000000000000000000000000001FFFFC2
:10CF7000FFE3600007736000000000000001FFFF96
:10CF8000FFE360000EE3600000000000000180008D
:10CF9000000360001DC36000000000000001BFFF2F
:10CFA000FFE360003B836000000000000001BFFF62
:10CFB000FFE3600077036000000000000001B000A4
:10CFC00000036000EE036000000000000001B000FC
:10CFD00000036001DC036000000000000001B000FD
:10CFE00000036003B8036000000000200001B000EF
:10CFF0000003600770036000000000600001BFFFD5
:10D00000FFE3600EE0036000000000600001BFFF6E
:10D01000FFE3601DC00360000003006000018000AA
:10D020000003603B80036000000300E00001BFFFDD
:10D03000FFE3607700036000000300C00001BFFF52
:10D04000FFE360EE00036000000380C00001B00059
:10D05000000361DC00036000000780C00001B00035
:10D06000000363B8000360000007C0C00001B00007
:10D0700000036770000360000006C0C00001B0003C
:10D0800000036EE000036000000660C10101B00013
:10D0900000037DC000036000000630C30301BFFF32
:10D0A000FFE37B8000036000000C30C30701BFFF7B
:10D0B000FFE3770000036000000C1CC30601800042
:10D0C00000030E0000036000000C0CC20E01FFFF05
:10D0D000FFE3FC0000036000000C0EC61E01FFFF12
:10D0E000FFE3F80000036000000C07C61E0000000C
:10D0F0000000000000000000000C03C676000000E5
:10D100000000000000000000000C01C7E600000065
:10D110000000000000000000000C00C7C600000076
:10D120000000000000000000000C000306000000EA
:10D130000000000000000000000C000000000000E3
:10D140000000000000000000000C000000000000D3
:10D1500000000000000000000000000000000000CF
:10D1600000000000000000000000000000000000BF
:10D1700000000000000000000000000000000000AF
:10D18000000000000000000000000000000000009F
:10D19000000000000000000000000000000000008F
:10D1A000000000000000000000000000000000007F
:10D1B000000000000000000000000000000000006F
:10D1C000000000000000000000000000000000005F
:10D1D000000000000000000000000000000000004F
:10D1E000000000000000000000000000000000003F
:10D1F000000000000000000000000000000000002F
:10D20000000000000000000000000000000000001E
:10D21000000000000000000000000000000000000E
:10D2200000000000000000000000000000000000FE
:10D2300000000000000000000000000000000000EE
:10D24000000000000000000000000000B0D6000058
:10D2500080D60000549AFF1F00003000000000003C
:10D2600035440000B545000000000000010000004A
:10D27000E4D60000030000000000000001000000F0
:10D28000E13C000001000000C4D6000009000000DD
:10D290000100000034D5000007000000000000007D
:10D2A0008CD6000080D60000489AFF1F0000300096
:10D2B000000000004544000071490000000000002B
:10D2C00001000000CCD600000500000000000000B6
:10D2D00001000000E151000001000000BCD6000088
:10D2E000080000000000000008D6000008D600007A
:10D2F000169AFF1F00000C0003000000AD4C000058
:10D30000C5450000000000000000000074D60000C9
:10D3100080D600004A9AFF1F000030000000000085
:10D3200045440000714900000000000000000000BA
:10D33000ECD60000F4D60000B899FF1F01001000E1
:10D3400006000000414F00009545000049450000DF
:10D350002C010000213C0000060000000800000035
:10D36000A88CFF1F4CD6000002000300060000003E
:10D37000348DFF1FC4D60000000005010500000029
:10D38000E88AFF1FE0D5000000000101080000004E
:10D39000708DFF1F00000000A4D6000080D60000A2
:10D3A000449AFF1F000030000000000045440000C8
:10D3B000714900000000000034D5000000000405A1
:10D3C00008000000888CFF1F000000005CD60000F1
:10D3D00068D600007E99FF1F0000010001000000D8
:10D3E00059400000A54500000000000000000000BA
:10D3F00090D500005CD50000F699FF1F00000900E1
:10D40000000000007D400000D54500000000000045
:10D4100001000000D8D60000040000000000000059
:10D4200001000000E545000098D500000000020161
:10D4300006000000848AFF1F4F4E00004F46460042
:10D44000424154004C4F5720000000005553420009
:10D450004D454E552020202020202020205858586F
:10D4600020592E595600000058000000524F540019
:10D470004D454C0044594E006D730000312F0000A3
:10D48000424954004C5652004E524D0052455600EF
:10D4900050424400762E0000312E332E3900000019
:10D4A0004E754556490000006669726D7761726578
:10D4B00020762E0053455400434C5200444F4E27D3
:10D4C0005400000050414E49430000004D570000F9
:10D4D00046500000434600005350000053570000E0
:10D4E00042520000564C0000455800004D572B009A
:10D4F00042522B00564C2B0045582B00554E4F00E6
:10D500002D3400002D3300002D3200002D3100009D
:10D510004C494E002B3100002B3200002B33000011
:10D520002B34000053310000533200005A31000008
:10D530005A3200005649425241544F004449524524
:10D540004354494F4E000000434F4E54524F4C003D
:10D55000535155454C434820420000004C45564528
:10D560004C00000053454E534520425445000000F6
:10D57000535155454C4348204C00000053454E53F1
:10D5800045204C565200000052455455524E000062
:10D5900044455054480000005345545550204354CE
:10D5A000524C530050494E4B59204B4559000000F6
:10D5B0004445474C495443480000000045585452E4
:10D5C0004120435452000000504954434842454EC4
:10D5D00044000000504F52542F474C4400000000BC
:10D5E00053455455502042524541544800000000D4
:10D5F00056454C20424941530000000056454C20FE
:10D6000044454C4159000000435552564500000026
:10D6100056454C4F43495459000000004252454181
:10D62000544820415400000043433220524953459E
:10D6300000000000425254482043433200000000E2
:10D64000425254482043433100000000524F54419D
:10D65000544F522053455455500000005052494FEA
:10D6600052495459000000004D4F4E4F205052492E
:10D670004F000000524F5441544520340000000038
:10D6800053454D49544F4E4553000000524F5441AD
:10D690005445203300000000524F5441544520327D
:10D6A00000000000524F544154452031000000005A
:10D6B000504152414C4C454C0000000041424F55F6
:10D6C00054000000455854524153000053455455EE
:10D6D000502043544C0000005345545550204252B2
:10D6E0000000000041444A55535400004D4944494C
:10D6F000204348004D4944492043484E4C00000017
:10D70000574C20504F57455200000000535045439E
:10D71000204B4559000000004741544520484F4CDC
:10D72000440000004C45474143592042520000004C
:10D730004C45474143592050420000004F4354415B
:10D74000564500005452414E53504F534500FFFF81
:10D75000002111020200FFFF34800440400000005D
:10D760001211FFFFFF02020000001310FFFFFF0273
:10D770000200000018000000348004408000000017
:10D780001EFFFFFFFF02000000001DFFFFFFFF0262
:10D790000000000019000000000000000000000070
:10D7A000F95D0000BD5D0000715D0000B95D000025
:10D7B000755D0000815D0000A15D000000010307B0
:10D7C0000F1F3F7F2200FF2100FFFFFF0080C0E00E
:10D7D000F0F8FCFE0000000000000000897E000060
:10D7E000B9810000715D0000B56800004D6900005E
:10D7F00031770000E576000019770000F17600002F
:10D8000005770000017600003177000059770000AD
:10D81000496B0000917300002D730000297800000F
:10D82000357700008D7800002D790000DA02818FB5
:10D83000DA1281FF0000600000000000000000001C
:10D840000000000000E000000000000000000000F8
:10D8500000000001E00000000000000000000000E7
:10D86000000001F0000000000000000000000000C7
:10D870000003F000000000000000000000000000B5
:10D8800007F000000000000000000000000000079A
:10D89000F8000000000000000000000000000FF889
:10D8A00000000003C0007E000001E0007F0FF800D0
:10D8B000000003C000FE000001E000FFEFF80000E0
:10D8C0000003C000FE000001E000FFFFF8000000C0
:10D8D00003C000F00000000F007FFE7FC0000003C7
:10D8E000C000F00000000F003FFE7FF83FF1FBCFCB
:10D8F000FCFEF3BC3DEFE01FFE7FFF7FFBFFDFFE82
:10D90000FEFFBC3DEFE01FC6FFFF7FFBFFDFFEFE1B
:10D91000FFBC3DEFE00FE3C7FE787BC3DE1EF0FFE8
:10D92000BC3DEF0007FF87FC787BC3DE1EF0F83CB0
:10D930003DEF0001FFFFF0007BC3C01EF0F03C3D57
:10D94000EF0001F37FE03FFBC3CFFEF0F03C3DEF83
:10D950000003E33F807FFBC3DFFEF0F03C3DEF00C0
:10D9600007E73C00787BC3DE1EF0F03C3DEF00078C
:10D97000FFBE00787BC3DE1EF0F03C3DEF0007FFEA
:10D98000FE00787BC3DE1EF0F03C3DEF000FFFFE93
:10D99000007FFBFFDFFEF0F03FFDEFE00FFFFF0039
:10D9A0007FFBFFDFFEF0F03FFDEFE00FF9FF003EF1
:10D9B00079F9CF9EF0F01F3DE7E01FF1FF00000076
:10D9C0000000000000000000001F80FF007FFFFF3C
:10D9D000FFFFFFFFFFFFFFE01C007F007FFFFFFF57
:10D9E000FEB46D888D18E000001F007FFFFFFFFE72
:10D9F00095AD7DB577E000000F007FFFFFFFFEA52E
:10DA0000AD9D8D19E0000006007FFFFFFFFEB5AD64
:10DA1000EDB57EE0AED580A8D300408D2000A1C832
:10DA2000DB40A4A62EAFFFFF000000000001800035
:10DA30000000000000000000038000000000000063
:10DA400000000007C000000000000000000007C048
:10DA50000000000000000000000FC00000000000F7
:10DA6000000000001FE00000000000000000001F98
:10DA7000E00000000000000000003FE000000000A7
:10DA800000000000003FF000000000000000000067
:10DA90007FF0000000000000001FF87FF000000091
:10DAA000000000003FFE7FF0000000000000003F8B
:10DAB000FF7FF0000000000000001FFFFBE00000FF
:10DAC00000000000000FFFF9FFC000000000000090
:10DAD0000FFFF9FFF800000000000007FFF1FFFF53
:10DAE00000000000000003FC73FFFF800000000046
:10DAF0000001FE3FFFFF80000000000000FF1E0F3E
:10DB0000FF000000000000007FFE1FFC000000007E
:10DB10000000003FFFFFF8000000000000000FDFE2
:10DB2000FFE0000000000000001F19FFC00000001F
:10DB3000000000003F3CFF00000000000000007EED
:10DB40007CF800000000000000007FFE7C00000068
:10DB50000000000000FFFFFC0000000000000000CB
:10DB6000FFFFFE0000000000000000FFFFFE0000BD
:10DB7000000000000001FFEFFE00000000000000B8
:10DB800001FFCFFE0000000000000003FF07FE00C1
:10DB900000000000000003FC07FE00000000000081
:10DBA0000003F003FE00000000000000018000FE02
:10DBB000000000000000000000007E0000000000E7
:10DBC00000000000003E0000000000000000000017
:10DBD0000C000000000000078000FC000003C000F3
:10DBE0000000078001FC000003C000000007800166
:10DBF000FC000003C0000000078001E00000001EE0
:10DC0000000000078001E00000001E007FE3F79F96
:10DC1000F9FDE7787BDFC0FFF7FFBFFDFDFF787BF5
:10DC2000DFC0FFF7FFBFFDFDFF787BDFC0F0F787A8
:10DC3000BC3DE1FF787BDE00F0F787BC3DE1F0788A
:10DC40007BDE0000F787803DE1E0787BDE007FF738
:10DC5000879FFDE1E0787BDE00FFF787BFFDE1E015
:10DC6000787BDE00F0F787BC3DE1E0787BDE00F0FA
:10DC7000F787BC3DE1E0787BDE00F0F787BC3DE153
:10DC8000E0787BDE00FFF7FFBFFDE1E07FFBDFC058
:10DC9000FFF7FFBFFDE1E07FFBDFC07CF3F39F3DBB
:10DCA000E1E03E7BCFC0000000000000000000006B
:10DCB00000FFFFFFFFFFFFFFFFFFFFC0FFFFFFFFB2
:10DCC000FD68DB111A31C0FFFFFFFFFD2B5AFB6A15
:10DCD000EFC0FFFFFFFFFD4B5B3B1A33C0FFFFFFB1
:10DCE000FFFD6B5BDB6AFDC0DA0281FF0000000014
:10DCF00000000000897E0000B9810000715D000015
:10DD0000B56800003D89000031770000E57600002D
:10DD100019770000F1760000057700000176000019
:10DD20003177000059770000557700007D770000BB
:10DD3000D577000029780000357700008D78000045
:10DD40002D79000000000000003E5B4F5B3E3E6B03
:10DD50004F6B3E1C3E7C3E1C183C7E3C181C577D85
:10DD6000571C1C5E7F5E1C00183C1800FFE7C3E7D1
:10DD7000FF0018241800FFE7DBE7FF30483A060EE3
:10DD80002629792926407F050507407F05253F5A2A
:10DD90003CE73C5A7F3E1C1C08081C1C3E7F14229A
:10DDA0007F22145F5F005F5F06097F017F00668945
:10DDB000956A606060606094A2FFA29408047E048B
:10DDC0000810207E201008082A1C08081C2A0808B1
:10DDD0001E101010100C1E0C1E0C30383E38300671
:10DDE0000E3E0E06000000000000005F000000076D
:10DDF000000700147F147F14242A7F2A122313089B
:10DE0000646236495620500008070300001C224176
:10DE1000000041221C002A1C7F1C2A08083E08081A
:10DE200000807030000808080808000060600020CA
:10DE3000100804023E5149453E00427F40007249AD
:10DE40004949462141494D331814127F1027454551
:10DE500045393C4A49493141211109073649494967
:10DE600036464949291E00001400000040340000D5
:10DE7000000814224114141414140041221408023E
:10DE8000015909063E415D594E7C1211127C7F49B1
:10DE90004949363E414141227F4141413E7F494906
:10DEA00049417F090909013E414151737F08080832
:10DEB0007F00417F41002040413F017F0814224103
:10DEC0007F404040407F021C027F7F0408107F3E5D
:10DED0004141413E7F090909063E4151215E7F09CA
:10DEE000192946264949493203017F01033F404031
:10DEF000403F1F2040201F3F4038403F631408141C
:10DF00006303047804036159494D43007F41414153
:10DF10000204081020004141417F04020102044034
:10DF200040404040000307080020545478407F28B8
:10DF30004444383844444428384444287F385454AE
:10DF4000541800087E090218A4A49C787F080404D1
:10DF50007800447D40002040403D007F1028440070
:10DF600000417F40007C047804787C080404783801
:10DF700044444438FC1824241818242418FC7C0831
:10DF8000040408485454542404043F44243C4040AE
:10DF9000207C1C2040201C3C4030403C4428102861
:10DFA000444C9090907C4464544C440008364100AA
:10DFB0000000770000004136080002010204023C24
:10DFC0002623263C1EA1A161123A4040207A3854F3
:10DFD000545559215555794122545478422155546C
:10DFE000784020545579400C1E52721239555555BF
:10DFF00059395454545939555454580000457C41AA
:10E000000002457D420001457C407D1211127DF0E9
:10E01000282528F07C545545002054547C547C0A13
:10E02000097F4932494949323A4444443A324A48DC
:10E0300048303A4141217A3A42402078009DA0A0E0
:10E040007D3D4242423D3D4040403D3C24FF242432
:10E05000487E4943662B2FFC2F2BFF0929F620C051
:10E06000887E090320545479410000447D413048A2
:10E07000484A32384040227A007A0A0A727D0D19E5
:10E08000317D2629292F28262929292630484D4047
:10E0900020380808080808080808382F10C8ACBA43
:10E0A0002F102834FA00007B000008142A142222C2
:10E0B000142A14085500550055AA55AA55AAFF550B
:10E0C000FF55FF000000FF00101010FF0014141493
:10E0D000FF001010FF00FF1010F010F0141414FCDB
:10E0E000001414F700FF0000FF00FF1414F404FCF8
:10E0F000141417101F10101F101F1414141F0010D9
:10E100001010F0000000001F101010101F10101051
:10E1100010F010000000FF10101010101010101060
:10E12000FF10000000FF140000FF00FF00001F10A0
:10E13000170000FC04F414141710171414F404F45A
:10E140000000FF00F714141414141414F700F7144B
:10E150001414171410101F101F141414F41410109A
:10E16000F010F000001F101F0000001F140000003E
:10E17000FC140000F010F01010FF10FF141414FF36
:10E18000141010101F00000000F010FFFFFFFFFF31
:10E19000F0F0F0F0F0FFFFFF0000000000FFFF0FC5
:10E1A0000F0F0F0F3844443844FC4A4A4A347E0269
:10E1B000020606027E027E026355494163384444EA
:10E1C0003C04407E201E2006027E020299A5E7A59F
:10E1D000991C2A492A1C4C7201724C304A4D4D3010
:10E1E0003048784830BC625A463D3E494949007E35
:10E1F0000101017E2A2A2A2A2A44445F44444051CC
:10E200004A444040444A51400000FF0103E080FF7F
:10E21000000008086B6B083612362436060F090F0B
:10E2200006000018180000001010003040FF010127
:10E23000001F01011E00191D1712003C3C3C3C0050
:10E24000000000000D0AFFFF050E08090D0C06076F
:10E250000F0400130393050E08090D0C06070F04A5
:10E26000FFFFC585848687C4FFFF001303931A92BE
:10E2700017FFFFFF6FF07F030370037813F0800F29
:10E28000FBD070474008FE4340A004404408FE43D2
:10E2900044A004400018FE4300C004403000FE4388
:10E2A000309004403400FE43349004401C18FE4378
:10E2B0001CC004401018FE4310C004400818FE4360
:10E2C00008C004400C18FE430CC004400C10FE4370
:10E2D0000CB004401010FE4310B004401810FE4370
:10E2E00018B004401C10FE431CB004401410FE4340
:10E2F00014B004400418FE4304C004400010FE4360
:10E3000000B004400008FE4300A004400408FE439F
:10E3100004A004400C08FE430CA004400808FE437F
:10E3200008A004401418FE4314C004401818FE430B
:10E3300018C004400410FE4304B004400810FE431B
:10E3400008B004401400FE43149004404C08FE43FF
:10E350004CA004400420FE4304D004402410FE439B
:10E3600024B004402010FE4320B004402810FE4397
:10E3700028B004402C10FE432CB004400020FE4383
:10E3800000D004404808FE4348A004401000FE436B
:10E3900010900440090AFFFFFFFFFFFFFFFFFFFF90
:10E3A000FFFFFF0D00060807FFFF0E0FFF0CFFFF2A
:10E3B000FFFFFFFF0B05FFFF1519151900010000F6
:10E3C0000090FF1F12000000000200002C90FF1FB1
:10E3D0007300000000220100A090FF1F2100000038
:10E3E000002101008890FF1F0900000000030000C9
:10E3F000C490FF1F00000000010309041490FF1FD8
:10E400000000000002030904208EFF1F000000002E
:10E4100003030904C890FF1F000000000000000073
:10E42000000000000000000065787000FFFFFFFFA3
:10E43000000000000000E03F000000000000E0BF1E
:10E44000763C7935EF39EA3D763C7935EF39EABDEE
:10E450000000E0FE422EE63F0000E0FE422EE6BF56
:10E46000E090FF1FF8B500BFF8BC08BC9E4670479F
:10E47000E9C70000350400007D320000154A0000A5
:04E48000F8B500BF2C
:10E4840038B5084B1C681C6054B1074D94FAA4F3CA
:10E49400B3FA83F355F823309847631E1C40F5D133
:10E4A40038BD00BFA0D00440F08FFF1F38B5084B23
:10E4B4001C681C6054B1074D94FAA4F3B3FA83F3B7
:10E4C40055F823309847631E1C40F5D138BD00BF72
:10E4D400A0C00440D08FFF1F38B5084B1C681C60D7
:10E4E40054B1074D94FAA4F3B3FA83F355F82330E7
:10E4F4009847631E1C40F5D138BD00BFA0B004404E
:10E50400A08FFF1F38B5084B1C681C6054B1074D21
:10E5140094FAA4F3B3FA83F355F823309847631EAF
:10E524001C40F5D138BD00BFA0A00440508FFF1F90
:10E5340038B5084B1C681C6054B1074D94FAA4F319
:10E54400B3FA83F355F823309847631E1C40F5D182
:10E5540038BD00BFA0900440188FFF1F00000000CA
:10E564000020000032000000002000000020000015
:10E5740000100000AB0A000000080000660600005E
:10E584005505000092040000000400008E03000002
:10E5940033030000E8020000AB0200002400000086
:10E5A400002000000200020001000C00140500001D
:10E5B4000C0000000000F041000102070B010207FB
:10E5C4000B4A1400FBFFFFFF0000000000000000E6
:10E5D4000000000000000000000000000000000037
:10E5E40000000000000000000200FFFFFFFF000029
:10E5F400E4CC000074CD00008CCD00005CCD0000A4
:10E60400FCCC00000000000070D500005CD50000C8
:10E614006A89FF1F01001E000000000000000000C6
:10E624000000000000000000000000001CD60000F4
:10E634001CD600001C9AFF1F00000100010000000E
:10E6440000000000000000000000000000000000C6
:10E654007CD500005CD500006489FF1F01000C001C
:10E6640000000000000000000000000000000000A6
:10E674000000000001000000000000000000000095
:10E68400F0D50000F0D500005099FF1F00000900EC
:10E694000100000000000000000000000000000075
:10E6A4000000000088D500005CD50000A889FF1F89
:10E6B4000000040000000000000000000000000052
:10E6C40000000000208BFF1F9C8AFF1F648CFF1F2B
:10E6D40090D20000B08BFF1F4C8DFF1F0000000084
:10E6E400C8D50000C8D500002E9AFF1F00000C00FA
:10E6F4000000000000000000000000000000000016
:10E70400000000003CD700003CD70000E499FF1F44
:10E7140000000600000000000000000000000000EF
:10E724000000000001000000FC8AFF1F908DFF1F05
:10E734001C8CFF1FD48BFF1FD88DFF1F000000000F
:10E7440030D7000030D700004E9AFF1F00000100B0
:10E7540001000000000000000000000000000000B4
:10E7640000000000D4D50000D4D50000EC99FF1FB0
:10E774000000020001000000000000000000000092
:10E78400000000000000000034D6000034D6000071
:10E79400289AFF1F00007F00010000000000000015
:10E7A400000000000000000000000000FCD5000094
:10E7B400FCD50000209AFF1F00001E00010000008D
:10E7C4000000000000000000000000000000000045
:10E7D40028D6000028D600007099FF1F01000A0007
:10E7E4000100000000000000000000000000000024
:10E7F40000000000B0D50000B0D50000849AFF1FCF
:10E8040000004600000000000000000000000000BE
:10E8140000000000000000000CD700000CD700002E
:10E82400429AFF1F000001000100000000000000E8
:10E8340000000000000000000000000044D70000B9
:10E8440044D700008099FF1F00001800000000005A
:10E8540000000000000000000000000000000000B4
:10E8640018D7000018D70000049AFF1F0000010009
:10E874000100000000000000000000000000000093
:10E88400000000003CD500003CD50000829AFF1F28
:10E894000000010001000000000000000000000072
:10E8A4000000000000000000BCD50000BCD5000042
:10E8B4004C9AFF1F0000040001000000000000004B
:10E8C4000000000000000000FC8DFF1FECD30000DE
:10E8D400608AFF1F408CFF1F0C8AFF1FC489FF1F23
:10E8E400C88CFF1FEC8CFF1FF88BFF1FC08AFF1F13
:10E8F4002CD300006CD2000010D40000C0D2000061
:10E9040084D20000D8D200000000000064D50000CA
:10E914005CD500006689FF1F01000C0000000000A8
:10E9240000000000000000000000000000000000E3
:10E9340050D500005CD500007089FF1F01001E0047
:10E9440000000000000000000000000000000000C3
:10E954000000000040D6000040D600006299FF1F6E
:10E9640000000A0001000000000000000000000098
:10E974000000000048D2000094D3000024CE000020
:10E984009CD2000008D30000C8D30000000000009F
:10E99400A4D50000A4D500007C9AFF1F0000180035
:10E9A4000000000000000000000000000000000063
:10E9B400108DFF1F448BFF1F8C8BFF1FE889FF1FE7
:10E9C400B48DFF1FE4D20000688BFF1F3C8AFF1F39
:10E9D4000000000024D7000024D70000DC99FF1FAA
:10E9E4000000010001000000000000000000000021
:10E9F400000000000000000010D6000010D6000047
:10EA04004099FF1F00007F0001000000000000008B
:10EA140000000000000000000000000000D700001B
:10EA240000D700008C99FF1F0000030000000000C5
:10EA340000000000000000000000000000000000D2
:10EA440048D5000048D50000B299FF1F000001001E
:10EA540001000000000000000000000000000000B1
:10EA640016034E00750045005600490020004D0075
:10EA74004900440049000000A0D700000000000045
:10EA8400E8030000000000000060064058D70000C2
:10EA94000000000000000000000000000000000072
:10EAA4000000000000000000000000000000000062
:10EAB4000000000000000000000000000000000052
:10EAC4000000000000000000000000000000000042
:10EAD4000000000000000000000000000000000032
:10EAE40000000000A0D7000000000000E8030000C0
:10EAF400000000000070064078D70000000000000D
:10EB04000000000000000000000000000000000001
:10EB140000000000000000000000000000000000F1
:10EB240000000000000000000000000000000000E1
:10EB340000000000000000000000000000000000D1
:10EB440000000000000000000000000000000000C1
:10EB54000A040000B49FFF1FC9890000C98900008E
:10EB6400C9890000C9890000C9890000C989000059
:10EB7400C9890000C9890000C9890000C989000049
:10EB8400C9890000C9890000C9890000C989000039
:10EB9400C9890000C9890000C9890000C989000029
:10EBA400C9890000C9890000C9890000C989000019
:10EBB400C9890000C9890000C9890000C989000009
:10EBC400C9890000C9890000C9890000C9890000F9
:10EBD400C9890000C9890000C9890000C9890000E9
:10EBE400C9890000C9890000C9890000C9890000D9
:10EBF400C9890000C9890000C9890000C9890000C9
:10EC0400C9890000C9890000C9890000C9890000B8
:10EC1400C9890000C9890000C9890000C9890000A8
:10EC2400C9890000C9890000C9890000C989000098
:10EC3400C9890000C989000008000000FFFFFFFF28
:10EC44001201100100000040C01685047502010283
:10EC54000301000018035400650065006E00730092
:10EC640079006400750069006E006F00090273008A
:10EC7400020100C03209040000020103000007245D
:10EC840001000125000624020101000624020202FB
:10EC94000009240301030102010009240302040101
:10ECA40001010009050402400000000005250101DE
:10ECB4000109058302400000000005250101030944
:10ECC40004010002030000000921110100012221B6
:10ECD400000705810340000107050203200002002C
:10ECE40006C9FF0904A15C7508150026FF009540BC
:10ECF4000975810295200976910295040976B1027D
:10ED0400C0000000040309040C030000000000001C
:10ED140000000000000000000000000000000100EE
:10ED240000000000CC93FF1F3494FF1F9C94FF1F2E
:10ED340000000000000000000000000000000000CF
:10ED440000000000000000000000000000000000BF
:10ED540000000000000000000000000000000000AF
:10ED6400000000000000000000000000000000009F
:10ED7400000000000000000000000000000000008F
:10ED8400000000000000000000000000000000007F
:10ED9400000000000000000000000000000000006F
:10EDA400000000000000000000000000000000005F
:10EDB400000000000000000000000000000000004F
:10EDC400000000000000000001000000000000003E
:10EDD4000E33CDAB34126DE6ECDE05000B00000003
:10EDE400000000000000000000000000000000001F
:10EDF400000000000000000000000000000000000F
:10EE040000000000000000000000000000000000FE
:10EE140000000000000000000000000000000000EE
:10F144000000000000000000E090FF1F000000002D
:10F15400000000000C95FF1F0C95FF1F1495FF1F66
:10F164001495FF1F1C95FF1F1C95FF1F2495FF1F5F
:10F174002495FF1F2C95FF1F2C95FF1F3495FF1F0F
:10F184003495FF1F3C95FF1F3C95FF1F4495FF1FBF
:10F194004495FF1F4C95FF1F4C95FF1F5495FF1F6F
:10F1A4005495FF1F5C95FF1F5C95FF1F6495FF1F1F
:10F1B4006495FF1F6C95FF1F6C95FF1F7495FF1FCF
:10F1C4007495FF1F7C95FF1F7C95FF1F8495FF1F7F
:10F1D4008495FF1F8C95FF1F8C95FF1F9495FF1F2F
:10F1E4009495FF1F9C95FF1F9C95FF1FA495FF1FDF
:10F1F400A495FF1FAC95FF1FAC95FF1FB495FF1F8F
:10F20400B495FF1FBC95FF1FBC95FF1FC495FF1F3E
:10F21400C495FF1FCC95FF1FCC95FF1FD495FF1FEE
:10F22400D495FF1FDC95FF1FDC95FF1FE495FF1F9E
:10F23400E495FF1FEC95FF1FEC95FF1FF495FF1F4E
:10F24400F495FF1FFC95FF1FFC95FF1F0496FF1FFD
:10F254000496FF1F0C96FF1F0C96FF1F1496FF1FAA
:10F264001496FF1F1C96FF1F1C96FF1F2496FF1F5A
:10F274002496FF1F2C96FF1F2C96FF1F3496FF1F0A
:10F284003496FF1F3C96FF1F3C96FF1F4496FF1FBA
:10F294004496FF1F4C96FF1F4C96FF1F5496FF1F6A
:10F2A4005496FF1F5C96FF1F5C96FF1F6496FF1F1A
:10F2B4006496FF1F6C96FF1F6C96FF1F7496FF1FCA
:10F2C4007496FF1F7C96FF1F7C96FF1F8496FF1F7A
:10F2D4008496FF1F8C96FF1F8C96FF1F9496FF1F2A
:10F2E4009496FF1F9C96FF1F9C96FF1FA496FF1FDA
:10F2F400A496FF1FAC96FF1FAC96FF1FB496FF1F8A
:10F30400B496FF1FBC96FF1FBC96FF1FC496FF1F39
:10F31400C496FF1FCC96FF1FCC96FF1FD496FF1FE9
:10F32400D496FF1FDC96FF1FDC96FF1FE496FF1F99
:10F33400E496FF1FEC96FF1FEC96FF1FF496FF1F49
:10F34400F496FF1FFC96FF1FFC96FF1F0497FF1FF8
:10F354000497FF1F0C97FF1F0C97FF1F1497FF1FA5
:10F364001497FF1F1C97FF1F1C97FF1F2497FF1F55
:10F374002497FF1F2C97FF1F2C97FF1F3497FF1F05
:10F384003497FF1F3C97FF1F3C97FF1F4497FF1FB5
:10F394004497FF1F4C97FF1F4C97FF1F5497FF1F65
:10F3A4005497FF1F5C97FF1F5C97FF1F6497FF1F15
:10F3B4006497FF1F6C97FF1F6C97FF1F7497FF1FC5
:10F3C4007497FF1F7C97FF1F7C97FF1F8497FF1F75
:10F3D4008497FF1F8C97FF1F8C97FF1F9497FF1F25
:10F3E4009497FF1F9C97FF1F9C97FF1FA497FF1FD5
:10F3F400A497FF1FAC97FF1FAC97FF1FB497FF1F85
:10F40400B497FF1FBC97FF1FBC97FF1FC497FF1F34
:10F41400C497FF1FCC97FF1FCC97FF1FD497FF1FE4
:10F42400D497FF1FDC97FF1FDC97FF1FE497FF1F94
:10F43400E497FF1FEC97FF1FEC97FF1FF497FF1F44
:10F44400F497FF1FFC97FF1FFC97FF1F0498FF1FF3
:10F454000498FF1F0C98FF1F0C98FF1F1498FF1FA0
:10F464001498FF1F1C98FF1F1C98FF1F2498FF1F50
:10F474002498FF1F2C98FF1F2C98FF1F3498FF1F00
:10F484003498FF1F3C98FF1F3C98FF1F4498FF1FB0
:10F494004498FF1F4C98FF1F4C98FF1F5498FF1F60
:10F4A4005498FF1F5C98FF1F5C98FF1F6498FF1F10
:10F4B4006498FF1F6C98FF1F6C98FF1F7498FF1FC0
:10F4C4007498FF1F7C98FF1F7C98FF1F8498FF1F70
:10F4D4008498FF1F8C98FF1F8C98FF1F9498FF1F20
:10F4E4009498FF1F9C98FF1F9C98FF1FA498FF1FD0
:10F4F400A498FF1FAC98FF1FAC98FF1FB498FF1F80
:10F50400B498FF1FBC98FF1FBC98FF1FC498FF1F2F
:10F51400C498FF1FCC98FF1FCC98FF1FD498FF1FDF
:10F52400D498FF1FDC98FF1FDC98FF1FE498FF1F8F
:10F53400E498FF1FEC98FF1FEC98FF1FF498FF1F3F
:10F54400F498FF1FFC98FF1FFC98FF1F0499FF1FEE
:0CF554000499FF1F00000200FFFFFFFFF2
:00000001FF
